:100000000C94481E0C94881E0C94881E0C94881E18
:100010000C94881E0C94881E0C94881E0C94881EC8
:100020000C94881E0D944B200D944B200D944B2066
:100030000C94881E0C94881E0C94881E0C94881EA8
:100040000C94881E0C941A880C94881E0C94881E9C
:100050000C94881E0C947C850C94881E0D94DD1ED7
:100060000C94881E0C9499DD0C948FDD0C94881EE2
:100070000C94881E0C94881E0C94881E0C94881E68
:100080000C94881E0C94881E0C94881E0C94881E58
:100090000C94881E0C94881E0C94881E0D94271FA7
:1000A0000C94881E0C94881E0C94881E0C94881E38
:1000B0000C94881E0C94881E0C94881E0C94881E28
:1000C0000C94881E0C94881E0C94881E0C94881E18
:1000D0000C94881E0C94881E0C94881E0C94881E08
:1000E0000C94881E084AD73B3BCE016E84BCBFFDF2
:1000F000C12F3D6C74319ABD56833DDA3D00C77FF8
:1001000011BED9E4BB4C3E916BAAAABE0000008090
:100110003F05A84CCDB2D44EB93836A9020C50B91F
:10012000918688083CA6AAAA2ABE000000803F004B
:100130000C942C440C941F4E0D94C8090C94BE963C
:100140000C945E270C941C440C942D740C9418444D
:100150000D94B0180C9433CE0D940A1C0C9473605B
:100160000D9475070C94DA220C94EE340C94A230A2
:100170000C94462E0C946E260C9413CE0D94C30949
:100180000C9439470C94DE470C946E280C94879697
:100190000C942A250D94A8180C94AB960D945B072B
:1001A0000C943A2E0C9496260C94FC470C946A25D9
:1001B0000C94012E0D94251C0C94662D0D94D206E2
:1001C0000C940C440D9426090C9485270C940E482D
:1001D0000C94D7200C9428230C94C3960C94EFCD48
:1001E0000C9457CE0C941A480D94671C0C94092952
:1001F0000C94EB270C9424510C9406560C947628FE
:100200000D94E0090C94CD640D944B070C947E265C
:100210000C94FA480C9401320C9421240C94D32CA5
:100220000D942E090C946E760C94A7280C944A70A9
:100230000C943F960C943D750C94D92B0C94CC2BBC
:100240000C94BF270C94F5CB0C94C8260C94F1CBDE
:100250000C94432E0D94F0090C94F6470C94F32063
:100260000D94D1070C944D2E0D944C070C94583BD3
:100270000C94F21E0C9432280D948D180C94EF23DC
:100280000C9428440D94C3180C9459CE0C94BE5869
:100290000C9456260C944B2E0C94A5730C94C920E8
:1002A0000C9466260C9436470C94372E0D94BF2779
:1002B0000C94C76F0C9444270C94FA340D94CB180B
:1002C0000C94B0200C9435CE0C944D700D94D9182C
:1002D0000D94831C0C94145F0C942E270C948F2582
:1002E0000C944F750C9402480C94C6220C94A622D0
:1002F0000D94731C0C94A8530D94C41C0D940834D5
:100300000C94312E0C94F4340D94D6090D945C09A0
:100310000C94B2530C940B370C9486260C94501FFB
:100320000C9419390C9424440D94D1060C948E3BF2
:100330000C94FC220D94791C0C9408440C94062314
:100340000D9492180C9422C60C94EF570C940C5CEC
:100350000C94DD2B0C947A280C94532E0C94E126EB
:100360000C94E4470C945E260D94D1180C947228DA
:100370000C94EA470C94C8230C94AC270C94497055
:100380000C9492740C943F260C94502E0C94742868
:100390000C9433470C9493960C9492220C94D84767
:1003A0000C94111F0C948B250C944F450C94AD5359
:1003B0000C944D3E0D946E070D944C1D0C940CCC7A
:1003C0000D947F090D94A4180C94CFCD0D9446097B
:1003D0000C943A240C9408CC0C9408240C941448E3
:1003E0000D94B9180D94E9070C947C280D94AC1861
:1003F0000C9416350C940F350C9495750C9437CEDF
:100400000C944C450C940FCE0C9464630C94E8222D
:100410000D94D5180C9430290C9452450C94F36D1E
:100420000C9420440D94F1090C94F0470D94CD09DF
:100430000C94A1240C94AD740C9499270C94C3CD06
:100440000D945D080D94621C0D94BD180C945150D0
:100450000D94A1090C945BCE0C94BE1E0C94A69630
:100460000C944B270C9428280C948A1E0C949C25E1
:100470000C942DC50C94342E0C94B7530C9408484E
:100480000D9445080C9411CE0C94635A0C94E771AA
:100490000C9488730C948D2E0D94B3180C94AF2685
:1004A0000C9476260C94B0220C94142F0C94E52016
:1004B0000C94444B0C9410440C944E740C94A4244F
:1004C0000C9463250D948E1C0C94402E0C94924C2D
:1004D0000D94E3180C9471270C9478280C94013532
:1004E0000C942F960C94B5240D94DF180C947E2850
:1004F0000C9408350C94061F0C943D2E0C94EDCDF5
:100500000C9414230C94DF2C0D94D0060D94C71872
:100510000C94262E0C9414440D94A2074E414E497F
:100520004E495459494E46CDCCCC3D0AD7233C17B1
:10053000B7D13877CC2B329595E6241FB14F0A00FE
:100540000020410000C84200401C4620BCBE4CCAEE
:100550001B0E5AAEC59D741FE0201023102490106E
:10056000A011202210241037B00840048003001F7F
:10057000E02010211023101520112021102110310E
:10058000300840048003001FE03FF03CF03B701F48
:10059000601EE03DF03BF038700FC0078003001F85
:1005A000E03FF03EF03CF01AE01EE03EF03EF03E50
:1005B000F00FC007800300554E4C4F414420464980
:1005C0004C414D454E54004C4F41442046494C410E
:1005D0004D454E540046494C414D454E54204348EC
:1005E000414E47450041425300504C410045727214
:1005F0003A207574663820666F6E74206E6F7420B2
:10060000696E697469616C697A65642E00FFE0FF48
:10061000D140A0C8A6A22FF80023AC00AF10FFFE67
:10062000FF05FFD0FFE0FFC1FFD1E240A0C8A6A2B6
:100630002FF800238127AC00AFFFD0FF64FFD1A5C6
:10064000FFD0FF64FF64FFD1A4FFD0FF16FFFE427E
:10065000656400456E636C6F73757265002568751F
:100660003A25303268750025303268753A253032C7
:100670006875002530326875272530326875002589
:100680006875642025303268753A25303268750007
:1006900020202020202020002020202000657272B1
:1006A000006F0557059F0587053FFFF03800703044
:1006B000FC3020FC102078102030102C00D02E317F
:1006C000D02F7BD02F7BD02E31D02C00D0203010DB
:1006D00020781020FC1030FC303800703FFFF03FD5
:1006E000FFF03800703186302387102787902F87DE
:1006F000D02F03D020301020781020781020301018
:100700002F03D02F87D0278790238710318630384A
:1007100000703FFFF01FFFF81FFFF80410400208B1
:1007200020020820041040082080104100104100E1
:100730000820800410400000001FFFF81FFFF85041
:1007400072696E742041626F72746564004D323557
:1007500020500A4D32340050617573696E672E2E39
:100760002E004D3234004C6F6164202A004C6F61C2
:1007700064206D6D00556E6C6F6164202A00556EAB
:100780006C6F6164206D6D0046696C2E2044696158
:100790002E202A0046696C2E204469612E004520D7
:1007A000696E206D6D5E3300200820466163740021
:1007B0002008204D6178002008204D696E004F66AA
:1007C00066004F6E004175746F74656D70004D6901
:1007D0006E2054726176656C205370656564004DBF
:1007E000696E2056656C6F63697479004D6178207D
:1007F00040205370656564004D6178204520416359
:1008000063656C004D6178204020416363656C0036
:1008100054726176656C20416363656C0052657447
:100820007261637420416363656C00416363656C4E
:1008300000402073746570732F6D6D0041647661A4
:100840006E6365642053657474696E6773003F005E
:1008500043616E63656C00496E6974004D343238D3
:1008600000496E697469616C697A6520454550522A
:100870004F4D0046696C616D656E740054656D7016
:100880006572617475726500544D432044726976D7
:100890006572730053746570732F6D6D004A756EC9
:1008A0006374696F6E2044657600416363656C65AF
:1008B000726174696F6E004D617820537065656474
:1008C00020286D6D2F73290053657420486F6D6566
:1008D000204F66667365747300436F6E6669677553
:1008E000726174696F6E005A2052616973650032DB
:1008F0006E64204E6F7A7A6C652040004265640019
:100900004E6F7A7A6C650046616E2053706565643F
:1009100000436F6E66696775726174696F6E00522D
:100920006573746F72652044656661756C747300DD
:100930004C6F61642053657474696E6773005374FF
:100940006F72652053657474696E677300507265C9
:1009500068656174202420436F6E6600546F6F6C6D
:10096000204368616E676500546F6F6C204F666648
:100970007365747300416476616E636564205365CA
:100980007474696E6773004D61696E004D37303263
:1009900020542564004D36303020423020542564E8
:1009A000004D373032203B2564004D373031205424
:1009B0002564004368616E67652046696C616D65FA
:1009C0006E7400556E6C6F61642046696C616D6574
:1009D0006E74004C6F61642046696C616D656E7465
:1009E000005072656865617420437573746F6D00A3
:1009F000507265686561742024004261636B005524
:100A00006E6C6F6164202A004C6F6164202A004381
:100A100068616E67652046696C616D656E74202A39
:100A2000004D61696E00436F6E74696E75650050AC
:100A300075726765206D6F726500524553554D455F
:100A4000204F5054494F4E533A005052494E542073
:100A50005041555345440020204E6F7A7A6C653AD8
:100A600020005061726B696E672E2E2E00000057B9
:100A700061697420666F720066696C616D656E7481
:100A8000206368616E676500746F207374617274AF
:100A9000005761697420666F720066696C616D65EC
:100AA0006E7420756E6C6F616400004E6F7A7A6CA4
:100AB000652068656174696E6700506C6561736577
:100AC00020776169742E2E2E00005072657373209A
:100AD000627574746F6E00746F2068656174206E47
:100AE0006F7A7A6C650000496E736572742066696E
:100AF0006C616D656E7400616E64207072657373F5
:100B000020627574746F6E00746F20636F6E746909
:100B10006E7565005761697420666F720066696C56
:100B2000616D656E74206C6F616400005072657356
:100B30007320427574746F6E00746F2072657375E4
:100B40006D65207072696E7400005761697420666B
:100B50006F72207072696E7400746F2072657375A5
:100B60006D652E2E2E00005761697420666F72002D
:100B700066696C616D656E742070757267650000E2
:100B80004D36303020423020542569004D37303109
:100B900020542569004D37303220542569005669AC
:100BA0006F6C657400496E6469676F00426C7565AF
:100BB00000477265656E0059656C6C6F77004F7207
:100BC000616E67650052656400576869746500422C
:100BD0006C756520496E74656E736974790047722F
:100BE00065656E20496E74656E736974790052652F
:100BF0006420496E74656E73697479004C454420B5
:100C0000436F6E74726F6C00437573746F6D204C1C
:100C10006967687473004C69676874205072657303
:100C20006574730044656661756C74004F66660098
:100C30004F6E004C6967687473004D61696E003FC8
:100C4000004261636B0053746F70004E6F204D65FE
:100C5000646961005072696E742066726F6D204D18
:100C600065646961004368616E6765204D6564690C
:100C700061004D3231004C696768747300436861EC
:100C80006E67652046696C616D656E7400436F6EBA
:100C900066696775726174696F6E0054656D706521
:100CA000726174757265004D6F74696F6E00526584
:100CB00073756D65205072696E740054756E6500B1
:100CC00053746F70205072696E7400506175736553
:100CD000205072696E7400496E666F2053637265AE
:100CE000656E003F005374617274205072696E74B7
:100CF0000043616E63656C005072696E74004361FD
:100D00006E6E6F7420656E746572207375626469AF
:100D1000723A200002202E2E004D61696E004D6F48
:100D2000766520246D6D00302E303235004D6F76A3
:100D30006520302E316D6D004D6F766520316D6D03
:100D4000004D6F76652031306D6D002100486F7465
:100D5000656E6420746F6F20636F6C640042616322
:100D60006B0050726F63656564004D6F7665202A75
:100D7000004D6F7665204578747275646572004D1C
:100D80006F76652040004D6F74696F6E0044697323
:100D900061626C65205374657070657273004D38C4
:100DA00034004732385A004732385900486F6D6571
:100DB00020400047323858004175746F20486F6DED
:100DC0006500473238004D6F7665204178697300C1
:100DD0004D61696E0050726568656174202420421F
:100DE00065640050726568656174202420416C6CF4
:100DF0000050726568656174202420456E64207E11
:100E000000507265686561742024207E0054656D11
:100E1000706572617475726500E905E505436F6F71
:100E20006C646F776E005072656865617420240091
:100E300046616E205370656564207E0042656400E3
:100E40004E6F7A7A6C65207E004D61696E00453286
:100E5000004531005A005900580045320045310024
:100E60005A0059004F6666004F6E005800544D43BB
:100E7000204472697665727300537465616C74689E
:100E800043686F7020456E61626C656400537465E1
:100E90007070696E67204D6F646500447269766595
:100EA000722043757272656E7400416476616E6380
:100EB00065642053657474696E677300466C6F7760
:100EC000207E00466C6F770046616E20537065652A
:100ED00064207E00426564004E6F7A7A6C65207EE5
:100EE000005370656564004D61696E00000C0F0071
:100EF000FE07022503BB017FFE08FE08FE05080869
:100F000006000040F0C88888987810050808060098
:100F100000C0F88888888888F80505050600012043
:100F200030F830200508080600002070F820202046
:100F300020E00509090600FF2070A8A8B88888707D
:100F400020070505070001D86C366CD8050909068D
:100F500000FFF8A88888888888A8F8050A0A06008B
:100F6000FE205050505088A8A88870030303060044
:100F70000340A040FFFFFFFFFFFFFFFFFFFFFFFF5A
:100F8000FFFFFFFFFFFFFFFFFFFF0000000605FF61
:100F90000107070602008080808080008003030331
:100FA000060105A0A0A005060606000050F8505056
:100FB000F8500509090600FF2070A8A07028A87045
:100FC00020050707060000C8C810204098980507AC
:100FD0000706000040A0A040A89068010303060295
:100FE000058080800309090601FF20404080808041
:100FF0004040200309090601FF8040402020204096
:10100000408005070706000020A8702070A8200572
:1010100005050600012020F820200203030601FF39
:10102000C04080050101060003F80202020601002B
:10103000C0C00507070600000810102040408005CA
:101040000707060000708898A8C88870030707067D
:10105000010040C040404040E00507070600007026
:101060008808102040F8050707060000F80810302F
:1010700008887005070706000010305090F810101F
:10108000050707060000F880F008088870050707C4
:10109000060000304080F0888870050707060000D1
:1010A000F808101020202005070706000070888827
:1010B0007088887005070706000070888878081017
:1010C00060020505060100C0C000C0C00206060699
:1010D00001FFC0C000C0408003050506010120409B
:1010E000804020050303060002F800F8030505060A
:1010F000010180402040800507070600007088102D
:10110000202000200507070600007088B8A8B880D6
:1011100070050707060000708888F888888805072A
:1011200007060000F04848704848F0050707060029
:101130000070888080808870050707060000F048EE
:1011400048484848F0050707060000F88080F0800E
:1011500080F8050707060000F88080F08080800591
:1011600007070600007088808098887005070706CA
:101170000000888888F8888888030707060100E04F
:101180004040404040E005070706000038101010BE
:101190001090600507070600008890A0C0A0908806
:1011A000050707060000808080808080F80507071B
:1011B00006000088D8A888888888050707060000E8
:1011C0008888C8A89888880507070600007088885E
:1011D00088888870050707060000F08888F08080FE
:1011E0008005070706000070888888A890680507B2
:1011F00007060000F08888F0A09088050707060021
:101200000070888070088870050707060000F820C5
:10121000202020202005070706000088888888886D
:1012200088700507070600008888888850502005C8
:10123000070706000088888888A8A85005070706C1
:10124000000088885020508888050707060000881D
:10125000885020202020050707060000F8081020ED
:101260004080F80309090601FFE0808080808080CB
:1012700080E00507070600008040402010100803AA
:1012800009090601FFE020202020202020E005039E
:10129000030600052050880501010600FEF803033F
:1012A000030601058040200505050600007008784A
:1012B00088780507070600008080F0888888F00598
:1012C000050506000070808088700507070600008D
:1012D000080878888888780505050600007088F079
:1012E0008070050707060000304840E04040400598
:1012F00007070600FE7088888878087005070706CB
:1013000000008080F0888888880307070601004075
:1013100000C0404040E00409090601FE1000301002
:10132000101010906005070706000080808890E08C
:101330009088030707060100C04040404040E00598
:101340000505060000D0A8A8A8A805050506000008
:10135000B0C88888880505050600007088888870F0
:101360000507070600FEF0888888F08080050707DB
:101370000600FE78888888780808050505060000BC
:10138000B0C880808005050506000078807008F0F0
:101390000507070600002020F82020201805050575
:1013A000060000888888986805050506000088887A
:1013B0008850200505050600008888A8A850050566
:1013C0000506000088502050880507070600FE88A3
:1013D000888850204080050505060000F810204050
:1013E000F80309090601FF204040408040404020AA
:1013F0000109090602FF8080808080808080800350
:1014000009090601FF80404040204040408005031C
:101410000306000248A890FF486F6D696E6720467A
:1014200061696C6564006F70656E0054524947478E
:1014300045524544003A20007A5F6D696E00795F3D
:101440006D696E00785F6D6178005265706F7274BF
:10145000696E6720656E6473746F70207374617455
:1014600075730A000000184300009A4200001643FA
:101470000000E6C20000A8C20000000020746F6FE8
:10148000206C6F6E6720657874727573696F6E205B
:1014900070726576656E7465640A0020636F6C64B3
:1014A00020657874727573696F6E207072657665E9
:1014B0006E7465640A00000018430000A8C20000B2
:1014C00000005761726E696E673A20486F6D696EF1
:1014D000672042756D702044697669736F72203C95
:1014E00020310A00020204008085430000214300ED
:1014F0000016430000A0400000A040000000400093
:10150000000001000000010000800055555500005A
:1015100000400033333300AAAA2A00499224000075
:10152000002000C7711C0099991900D1451700557A
:101530005515003BB1130024491200111111000090
:101540000010000F0F0F00E3380E0043790D00CCA0
:10155000CC0C00C3300C00E8A20B0064210B00AAE5
:10156000AA0A00703D0A009DD80900427B0900923A
:10157000240900DCD3080088880800104208000015
:10158000000800F0C1070087870700755007007149
:101590001C07003EEB0600A1BC0600699006006631
:1015A000660600703E06006118060017F405007418
:1015B000D105005BB00500B29005006272050055D0
:1015C00055050078390500B81E0500050505004ED3
:1015D000EC040087D40400A1BD040090A7040049D6
:1015E000920400C17D0400EE690400C75604004463
:1015F0004404005C3204000821040041100400008F
:101600000004003FF00300F8E0030026D20300C30B
:10161000C30300CCB503003AA803000A9B030038BB
:101620008E0300C08103009F750300D06903005042
:101630005E03001D53030034480300913D03003353
:1016400033030016290300381F03009715030030E9
:101650000C0300030303000BFA020049F10200BA75
:10166000E802005CE002002DD802002DD0020059F3
:10167000C80200B0C0020031B90200DAB10200AA0B
:10168000AA0200A0A30200BC9C0200FA9502005C22
:101690008F0200DF88020082820200457C02002760
:1016A00076020027700200436A02007C640200D0C8
:1016B0005E02003F590200C8530200FFFDFCFAF829
:1016C000F6F4F2F0EEECEAE9E7E5E3E1E0DEDCDA9D
:1016D000D9D7D5D4D2D0CFCDCBCAC8C7C5C3C2C045
:1016E000BFBDBCBAB9B7B6B4B3B2B0AFADACAAA9BE
:1016F000A8A6A5A4A2A1A09E9D9C9A99989795940E
:101700009392908F8E8D8B8A89888786848382813D
:10171000807F7E7D7B7A797877767574737271704D
:101720006F6E6D6C6B6A6968676665646362616041
:101730005F5E5D5C5B5A5958585756555453525129
:1017400050504F4E4D4C4B4A4A49484746464544F7
:1017500043424241403F3E3E3D3C3B3B3A393838B4
:1017600037363535343332323130302F2E2E2D2C62
:101770002B2B2A2929282727262525242323222104
:101780002120201F1E1E1D1C1C1B1B1A1919181896
:10179000171616151514131312121111100F0F0E20
:1017A0000E0D0D0C0C0B0A0A09090808070706069E
:1017B0000505040403030202010000DB0FC93F45D5
:1017C000BCDA3F8FB30240FCF0274056946140FEE4
:1017D0004B9B4084A5D840E0231841346A5641E829
:1017E00059974164DBD5416E271742B4B75542CEB5
:1017F0001A9742C8AED542B5885A43D40684BFA6CC
:101800005FA7BF7443E0BF10B11AC01C2C58C0E8DA
:10181000F697C0B849D6C04E4E17C124D355C180E3
:101820002497C1A0B5D5C1121A17C244AE55C278CB
:101830001797C26CACD5C267885AC320746F6F20EB
:101840006C6F6E6720657874727573696F6E207047
:10185000726576656E7465640A0020636F6C64203F
:10186000657874727573696F6E2070726576656ED7
:101870007465640A0053657474696E6773205374E9
:101880006F72656400290A002062797465733B20D9
:10189000637263200053657474696E6773205374B8
:1018A0006F726564202800454550524F4D20496EA7
:1018B000697469616C697A65640A0048617264637D
:1018C0006F6465642044656661756C74205365744B
:1018D00074696E6773204C6F616465640020286DC5
:1018E0006D290020460020420020480020204D3174
:1018F00034352053004D6174657269616C206865F0
:101900006174757020706172616D657465727300C9
:1019100020204D39303600205431204500205430ED
:101920002045005374657070657220647269766535
:10193000722063757272656E740020204D353639E1
:1019400020533100543120450054302045002058A8
:1019500000447269766572207374657070696E6791
:10196000206D6F64650020204D3134392043203BC9
:1019700020556E69747320696E2043656C736975B8
:10198000730A0054656D70657261747572652055D7
:101990006E697473002020473231203B004C696E21
:1019A00065617220556E69747300454550524F4D04
:1019B000206461746173697A65206572726F722E3A
:1019C0000A00290A002062797465733B2063726300
:1019D00020002073746F7265642073657474696E7F
:1019E00067732072657472696576656420280020CB
:1019F0002863616C63756C6174656429210A002039
:101A0000213D2000454550524F4D20435243206D0B
:101A100069736D61746368202D202873746F72651B
:101A2000642920002053697A653A2000496E646574
:101A3000783A200000007A4300007A430000A04179
:101A40000000C8428747BC428747BC420000C843E9
:101A5000E78CC042E8030000E803000064000000D7
:101A600088130000204D61726C696E3D563836292E
:101A70000A00454550524F4D2076657273696F6E6E
:101A8000206D69736D617463682028454550524F1D
:101A90004D3D0024F4D43050C38E20C2A2401782A2
:101AA0008B7011127A910D816CD90AA861E108C777
:101AB000586607615143061E4B5D05C145A7041AD0
:101AC000411104093D9803713931034036DB026549
:101AD000339102D4305402802E1D02632CEE017526
:101AE0002AC501B028A001102781018F2564012B90
:101AF000244B01E0223401AC211F018D200D018017
:101B00001FFC00841EED00971DDF00B81CD200E60C
:101B10001BC600201BBC00641AB200B219A8000A40
:101B200019A0006A189900D117910040178B00B5D1
:101B300016840031167E00B31579003A157300C77C
:101B4000146F0058146A00EE1366008813630025B2
:101B5000135E00C7125B006C12570015125400C1CF
:101B600011510070114F0021114B00D61049008D0A
:101B70001047004610440002104200C00F40008091
:101B80000F3E00420F3C00060F3B00CB0E38009387
:101B90000E37005C0E3500270E3400F30D3200C105
:101BA0000D3100900D3000600D2E00320D2D00051E
:101BB0000D2C00D90C2B00AE0C2900850C29005CE3
:101BC0000C2700350C27000E0C2600E80B2400C45F
:101BD0000B2400A00B23007D0B23005A0B2100399E
:101BE0000B2100180B2000F80A1F00D90A1E00BBA9
:101BF0000A1E009D0A1D00800A1D00630A1C004782
:101C00000A1B002C0A1B00110A1A00F7091A00DD32
:101C1000091900C4091900AB091900920917007BC2
:101C2000091800630917004C091600360916002030
:101C30000916000A091500F5081500E0081400CC83
:101C4000081400B8081400A4081400900813007DBC
:101C50000812006B081300580812004608120034DE
:101C6000081100230811001208110001081100F0EA
:101C7000071000E0071000D0071000C0071000B0E8
:101C8000070F00A107100091070E0083070F0074D3
:101C9000070F0065070E0057070E0049070E003BAF
:101CA000070D002E070E0020070D0013070D00067C
:101CB000070D00F9060C00ED060D00E0060C00D43F
:101CC000060C00C8060C00BC060C00B0060C00A4F4
:101CD000060B0099060C008D060B0082060B0077A0
:101CE000060B006C060B0061060A0057060B004C41
:101CF000060A0042060A0038060A002E060A0024D8
:101D0000060A001A060A001006090007060A00FD66
:101D1000050900F4050900EB050900E2050900D9F1
:101D2000050900D0050900C7050900BE050900B571
:101D3000050800AD050800A50509009C05080094EC
:101D40000508008C050800840508007C050800745F
:101D50000508006C050700650508005D05070056CD
:101D60000508004E05070047050700400508003834
:101D7000050700310507002A050700230507001C99
:101D8000050600160507000F0507000805060002F6
:101D9000050700FB040600F5040700EE040600E852
:101DA000040600E2040700DB040600D5040600CFA9
:101DB000040600C9040600C3040600BD040600B7FB
:101DC000040600B1040500AC040600A6040600A049
:101DD0000405009B04060095040500900406008A93
:101DE00004050085040500800406007A04050075DA
:101DF000040500700405006B04050066040500611D
:101E00000405005C04050057040500520405004D5C
:101E100004050048040500430405003E0404003A9C
:101E200004050035040500300404002C04050027D7
:101E3000040400230405001E0404001A0404001610
:101E4000040500110404000D040400090405000445
:101E500004040000040400FC030400F8030400F47C
:101E6000030400F0030400EC030400E8030400E4AE
:101E7000030400E0030400DC030400D8030400D4DE
:101E8000030400D0030400CC030400C8030300C50E
:101E900003030024F404D9201BC40C5C0E9804C472
:101EA000095F0265077101F405F900FB04B30048FE
:101EB000048700C10369005803550003034500BEB1
:101EC000023A008402310053022A0029022500044C
:101ED000022000E4011C00C8011900AF011700989E
:101EE0000114008401130071011000610110005100
:101EF000010E0043010D0036010B002B010B0020E9
:101F0000010B00150109000C01090003010800FB89
:101F1000000800F3000800EB000700E4000600DE04
:101F2000000600D8000600D2000600CC000500C75D
:101F3000000500C2000500BD000400B9000400B5A2
:101F4000000400B1000400AD000400A9000400A5D5
:101F5000000300A20003009F0004009B0003009800
:101F60000003009500020093000300900003008D21
:101F70000002008B0003008800020086000200843B
:101F8000000300810002007F0002007D0002007B50
:101F90000002007900020077000100760002007460
:101FA00000020072000100710002006F0002006D6B
:101FB0000001006C0002006A000100690002006775
:101FC000000100660001006500010064000200627B
:101FD00000010061000100600001005F0002005D7F
:101FE0000001005C0001005B0001005A0001005983
:101FF0000001005800010057000100560001005583
:102000000001005400010053000000530001005281
:1020100000010051000100500001004F0001004E7E
:102020000000004E0001004D0001004C0001004B7B
:102030000000004B0001004A000100490001004877
:102040000000004800010047000100460000004673
:10205000000100450000004500010044000100436C
:102060000000004300010042000000420001004166
:1020700000000041000100400001003F0000003F5F
:102080000001003E0000003E0001003D0000003D58
:102090000001003C0000003C0000003C0001003B4F
:1020A0000000003B0001003A0000003A0001003946
:1020B000000000390001003800000038000000383E
:1020C0000001003700000037000100360000003634
:1020D000000000360001003500000035000000352A
:1020E000000100340000003400000034000100331F
:1020F0000000003300000033000100320000003215
:102100000000003200010031000000310000003109
:102110000001003000000030000000300001002FFE
:102120000000002F0000002F0000002F0001002EF3
:102130000000002E0000002E0001002D0000002DE8
:102140000000002D0000002D0001002C0000002CDC
:102150000000002C0000002C0001002B0000002BD0
:102160000000002B0000002B0001002A0000002AC4
:102170000000002A0000002A0001002900000029B8
:1021800000000029000000290000002900010028AB
:10219000000000280000002800000028000000289F
:1021A0000001002700000027000000270000002792
:1021B0000000002700010026000000260000002685
:1021C0000000002600000026000100250000002578
:1021D000000000250000002500000025000000256B
:1021E000000100240000002400000024000000245E
:1021F0000000002400010023000000230000002351
:102200000000002300000023000000230000002342
:102210000001002200000022000000220000002235
:102220000000002200000022000100210000002127
:10223000000000210000002100000021000000211A
:10224000000000210001002000000020000000200C
:1022500000000020000000200000002000000020FE
:10226000000000200001001F0000001F0000001FF0
:102270000000001F0000001F0000001F0000001FE2
:102280000001001E0000001E0000001E0000001ED5
:10229000000000393000003325000087190000B02D
:1022A0000F0000DB080000BD040000740200003FC6
:1022B00001000020436F756E7420583A00453200CB
:1022C000426564004531004500626564002C20735E
:1022D000797374656D2073746F7070656421204824
:1022E00065617465725F49443A20004572723A2014
:1022F0004D415854454D50004D415854454D502086
:102300007472696767657265640048656174696EB7
:1023100067204661696C65640048656174696E6731
:10232000206661696C6564004572723A204D494EC1
:1023300054454D50004D494E54454D5020747269DE
:1023400067676572656400544845524D414C2052A0
:10235000554E4157415900546865726D616C205269
:10236000756E6177617900202F0020400020424087
:102370003A0020403A00496E76616C6964206578C5
:102380007472756465720A004163746976652045EC
:10239000787472756465723A20000009121B242D4E
:1023A000363F48415A536C657E7719100B023D3415
:1023B0002F265158434A757C676E323B2029161FE1
:1023C000040D7A7368615E574C452B2239300F0635
:1023D0001D14636A7178474E555C646D767F404981
:1023E000525B2C253E3708011A137D746F665950D5
:1023F0004B42353C272E1118030A565F444D727B21
:1024000060691E170C053A3328214F465D546B62F4
:102410007970070E151C232A31384148535A656CD0
:10242000777E09001B122D243F3658514A437C7594
:102430006E671019020B343D262F737A6168575E60
:10244000454C3B3229201F160D046A6378714E47B4
:102450005C55222B3039060F141D252C373E010800
:10246000131A6D647F7649405B523C352E27181154
:102470000A03747D666F5059424B171E050C333AA0
:1024800021285F564D447B7269600E071C152A2374
:102490003831464F545D626B707900002110422044
:1024A00063308440A550C660E770088129914AA135
:1024B0006BB18CC1ADD1CEE1EFF1311210027332AC
:1024C0005222B5529442F772D662399318837BB385
:1024D0005AA3BDD39CC3FFF3DEE36224433420043C
:1024E0000114E664C774A44485546AA54BB52885D5
:1024F0000995EEE5CFF5ACC58DD55336722611168C
:102500003006D776F6669556B4465BB77AA7199724
:102510003887DFF7FEE79DD7BCC7C448E558866813
:10252000A7784008611802282338CCC9EDD98EE974
:10253000AFF9488969990AA92BB9F55AD44AB77AEB
:10254000966A711A500A333A122AFDDBDCCBBFFBC4
:102550009EEB799B588B3BBB1AABA66C877CE44CFB
:10256000C55C222C033C600C411CAEED8FFDECCD14
:10257000CDDD2AAD0BBD688D499D977EB66ED55ECB
:10258000F44E133E322E511E700E9FFFBEEFDDDF64
:10259000FCCF1BBF3AAF599F788F8891A981CAB1F0
:1025A000EBA10CD12DC14EF16FE18010A100C23022
:1025B000E3200450254046706760B9839893FBA3DD
:1025C000DAB33DC31CD37FE35EF3B1029012F32272
:1025D000D2323542145277625672EAB5CBA5A8952D
:1025E00089856EF54FE52CD50DC5E234C324A014C2
:1025F00081046674476424540544DBA7FAB79987BD
:10260000B8975FE77EF71DC73CD7D326F236910611
:10261000B01657667676154634564CD96DC90EF904
:102620002FE9C899E9898AB9ABA944586548067861
:102630002768C018E1088238A3287DCB5CDB3FEB1C
:102640001EFBF98BD89BBBAB9ABB754A545A376AB1
:10265000167AF10AD01AB32A923A2EFD0FED6CDDEC
:102660004DCDAABD8BADE89DC98D267C076C645C01
:10267000454CA23C832CE01CC10C1FEF3EFF5DCFFC
:102680007CDF9BAFBABFD98FF89F176E367E554E51
:10269000745E932EB23ED10EF01E7C3C3E5E2B3D0E
:1026A0003F2F5B5D3B2C2A225C0043616E6E6F7492
:1026B000206F70656E2073756264697220004D65CD
:1026C00064696120496E6974204661696C005344F5
:1026D0002063617264206F6B0A006F70656E526FC9
:1026E0006F74206661696C65640A00766F6C756D45
:1026F000652E696E6974206661696C65640A004EB6
:102700006F20534420636172640A000A4D32340022
:102710004D3233202573002E0A006F70656E2066DF
:1027200061696C65642C2046696C653A20004669D5
:102730006C652073656C65637465640A0020536979
:102740007A653A200046696C65206F70656E656435
:102750003A2000454E4420535542524F5554494E5D
:10276000450A002220706F73002220706172656E2E
:10277000743A2200535542524F5554494E45204316
:10278000414C4C207461726765743A220053756243
:1027900063616C6C204F766572666C6F770045786C
:1027A000636565646564206D617820535542524FBE
:1027B0005554494E452064657074683A00577269F3
:1027C00074696E6720746F2066696C653A200043F7
:1027D0004F4D4D554E49434154494F4E0044525977
:1027E00052554E004552524F525300494E464F00EB
:1027F0004543484F004572726F7220777269746961
:102800006E6720746F20454550524F4D210A00538A
:10281000544F505045442E20005072696E746572BA
:102820002073746F707065642064756520746F2008
:102830006572726F72732E20466978207468652005
:102840006572726F7220616E6420757365204D39F8
:10285000393920746F20726573746172742E202868
:1028600054656D706572617475726520697320724C
:10287000657365742E2053657420697420616674D5
:1028800065722072657374617274696E67290A00DB
:102890004E6F20436865636B73756D20776974684C
:1028A000206C696E65206E756D6265722C204C61BE
:1028B0007374204C696E653A20004E6F2043686542
:1028C000636B73756D2077697468206C696E652021
:1028D0006E756D6265722C204C617374204C696E4C
:1028E000653A2000636865636B73756D206D69736D
:1028F0006D617463682C204C617374204C696E6543
:102900003A20004C696E65204E756D6265722069D3
:1029100073206E6F74204C617374204C696E652057
:102920004E756D6265722B312C204C617374204C96
:10293000696E653A20004D3131300053657269612E
:102940006C20737461747573206D69736D61746349
:10295000680A0053442072656164206572726F7268
:102960000A004B494C4C20627574746F6E2F70696D
:102970006E0A002121204B494C4C20636175736520
:10298000642062792000746F6F206D756368206920
:102990006E6163746976652074696D65202D2063AE
:1029A000757272656E7420636F6D6D616E643A202E
:1029B000002121204B494C4C2063617573656420D4
:1029C00062792000627573793A207061757365646D
:1029D00020666F7220696E7075740A006275737973
:1029E0003A2070617573656420666F722075736537
:1029F000720A00627573793A2070726F636573733F
:102A0000696E670A004D656469612052656D6F7675
:102A10006564004D6564696120496E736572746513
:102A20006400506C65617365205265736574005075
:102A300052494E5445522048414C54454400255378
:102A40003A202553004B494C4C45442E20005072EF
:102A5000696E7465722068616C7465642E206B69A0
:102A60006C6C28292063616C6C6564210A00006528
:102A700063686F3A004572726F723A00486F74650E
:102A80006E6420746F6F20636F6C640A005072650F
:102A9000737320627574746F6E20746F2072657327
:102AA000756D650A00496E736572742066696C61A4
:102AB0006D656E7420616E64207072657373206240
:102AC0007574746F6E0A005072657373206275744A
:102AD000746F6E20746F2068656174206E6F7A7AEF
:102AE0006C650A004C4F570048494748004F4B005F
:102AF0004572726F723A20416C6C200020636F6ED9
:102B00006E656374696F6E2E2E2E2000546573748B
:102B1000696E6720004C4F570048494748004F4BAB
:102B2000004572726F723A20416C6C200020636F16
:102B30006E6E656374696F6E2E2E2E200054657361
:102B400074696E6720004C4F570048494748004F52
:102B50004B004572726F723A20416C6C200020630A
:102B60006F6E6E656374696F6E2E2E2E2000546535
:102B70007374696E6720004C4F57004849474800FE
:102B80004F4B004572726F723A20416C6C200020EE
:102B9000636F6E6E656374696F6E2E2E2E20005407
:102BA000657374696E6720004C4F57004849474869
:102BB000004F4B004572726F723A20416C6C2000DE
:102BC00020636F6E6E656374696F6E2E2E2E20000B
:102BD00054657374696E672000544D4320434F4E13
:102BE0004E454354494F4E204552524F52002044C7
:102BF0000020204D32303020540020204D32303023
:102C0000205300202844697361626C6564293A008E
:102C100046696C616D656E742073657474696E6766
:102C2000730020204D3230312058004D6178204112
:102C30006363656C65726174696F6E2028756E6977
:102C400074732F7332290020204D32303320580006
:102C50004D617820666565647261746573202875BE
:102C60006E6974732F73290020520020204D32307A
:102C700034205000416363656C65726174696F6EE6
:102C80002028756E6974732F7332292028503C7088
:102C900072696E742D616363656C3E20523C72658F
:102CA00074726163742D616363656C3E20543C747F
:102CB000726176656C2D616363656C3E2900204A04
:102CC0000020540020530020204D32303520420097
:102CD000416476616E6365642028423C6D696E5F75
:102CE0007365676D656E745F74696D655F75733E5E
:102CF00020533C6D696E5F66656564726174653E04
:102D000020543C6D696E5F74726176656C5F6665B8
:102D10006564726174653E204A3C6A756E635F64E7
:102D200065763E290020204D32313700546F6F6C9C
:102D30002D6368616E67696E670020204D323138FF
:102D4000205400486F74656E64206F666673657406
:102D5000730020440020490020204D3330312050A2
:102D600000486F74656E6420504944004F46460029
:102D70004F4E0020204D61783A2000200020204D49
:102D8000696E3A2000203B200020204D3231312056
:102D90005300536F667420656E6473746F707300B4
:102DA000203B00205500204C0020204D36303320A1
:102DB000540046696C616D656E74206C6F61642FA0
:102DC000756E6C6F616400737072656164437963E2
:102DD0006C6500737465616C746843686F70002083
:102DE000647269766572206D6F64653A090073706C
:102DF000726561644379636C6500737465616C74BA
:102E00006843686F700020647269766572206D6F28
:102E100064653A09007370726561644379636C6537
:102E200000737465616C746843686F70002064722D
:102E300069766572206D6F64653A0900737072651A
:102E400061644379636C6500737465616C74684395
:102E5000686F700020647269766572206D6F6465BA
:102E60003A09007370726561644379636C6500733D
:102E70007465616C746843686F7000206472697671
:102E80006572206D6F64653A0900202E6873747254
:102E9000743A2000202E68656E643A200020636832
:102EA0006F70706572202E746F66663A2000202E57
:102EB00068737472743A2000202E68656E643A203C
:102EC000002063686F70706572202E746F66663ABA
:102ED0002000202E68737472743A2000202E6865DA
:102EE0006E643A20002063686F70706572202E74E3
:102EF0006F66663A2000202E68737472743A200060
:102F0000202E68656E643A20002063686F707065DB
:102F100072202E746F66663A2000202E68737472D9
:102F2000743A2000202E68656E643A2000206368A1
:102F30006F70706572202E746F66663A20003F5382
:102F4000206F7574206F662072616E67652028316E
:102F50002E2E38290A003F50206F7574206F66208E
:102F600072616E676520282D332E2E3132290A00BA
:102F70003F4F206F7574206F662072616E67652009
:102F800028312E2E3135290A003B200020496E764B
:102F9000616C69642065787472756465722000479D
:102FA000322F47332062616420706172616D6574F5
:102FB0006572730A00536C6565702E2E2E00436C8B
:102FC00069636B20746F20526573756D652E2E2EAC
:102FD000004E6F204D6F76652E00456E6420666949
:102FE0006C65206C6973740A00426567696E2066BF
:102FF000696C65206C6973740A004E6F206D65649E
:1030000069610A00286E6F2066696C652900437546
:103010007272656E742066696C653A2000534420B4
:103020007072696E74696E67206279746520004EF3
:103030006F74205344207072696E74696E670A0061
:103040002E0A0044656C6574696F6E206661696C58
:1030500065642C2046696C653A200046696C6520E1
:1030600064656C657465643A005072696E742074AE
:10307000696D653A20000A53746174733A20466999
:103080006C616D656E7420757365643A20002C2048
:103090004C6F6E67657374206A6F623A2000546FDC
:1030A00074616C2074696D653A20005374617473A7
:1030B0003A20002C204661696C65643A20002C207F
:1030C00046696E69736865643A20005072696E746F
:1030D000733A200053746174733A20006F6B006F71
:1030E000666600F027EB27E427DD27CF274445421B
:1030F00055473A004D3131322053687574646F770B
:103100006E004D3131332053004D616B6572626F3B
:1031100074205265706C696361746F72204F46460B
:103120002E002F2F004D31343520533C696E6465DD
:10313000783E206F7574206F662072616E6765201F
:1031400028302D31290A003F4A206F7574206F66A0
:103150002072616E67652028302E303120746F2018
:10316000302E33290A0046523A0020466C6F773AD7
:103170002000496E76616C696420657874727564AC
:1031800065720A0064697300656E0043290A006174
:10319000626C656420286D696E2074656D70200016
:1031A000436F6C6420657874727564657320617216
:1031B0006520004F666673657473204170706C699A
:1031C0006564004572723A20546F6F206661722107
:1031D00000546F6F206661722066726F6D20726599
:1031E000666572656E636520706F696E740A00456E
:1031F0004550524F4D204F4B0A002064726976654E
:10320000722063757272656E743A20002064726970
:103210007665722063757272656E743A2000206460
:1032200072697665722063757272656E743A2000F9
:10323000206472697665722063757272656E743A85
:103240002000206472697665722063757272656E03
:10325000743A200020204D323036205800486F6DDF
:1032600065206F6666736574004361703A00434F72
:103270004E4649475F4558504F5254004D454154C2
:103280005041434B00434F4F4C45525F54454D50C6
:1032900045524154555245004348414D4245525FC5
:1032A00054454D50455241545552450042414259B2
:1032B0005354455050494E470041524353004D4FDF
:1032C00054494F4E5F4D4F44455300544845524D6D
:1032D000414C5F50524F54454354494F4E0045585E
:1032E00054454E4445445F4D323000435553544F8E
:1032F0004D5F4649524D574152455F55504C4F41E5
:1033000044004C464E5F5752495445004C4F4E477F
:103310005F46494C454E414D45004155544F52453D
:10332000504F52545F53445F5354415455530053CC
:10333000445F575249544500524550454154004D51
:10334000554C54495F564F4C554D450053444341ED
:1033500052440050524F4D50545F535550504F52AD
:103360005400484F53545F414354494F4E5F434FBD
:103370004D4D414E445300454D455247454E4359EE
:103380005F50415253455200434153455F4C4947BA
:1033900048545F4252494748544E45535300544F96
:1033A00047474C455F4C494748545300534F465498
:1033B000574152455F504F574552004255494C4482
:1033C0005F50455243454E54004C4556454C494E7E
:1033D000475F44415441005A5F50524F42450052AA
:1033E000554E4F5554004155544F4C4556454C0091
:1033F0005052494E545F4A4F420050524F47524537
:103400005353004155544F5245504F52545F544509
:103410004D50004155544F5245504F52545F504FFC
:103420005300564F4C554D45545249430045455065
:10343000524F4D0042494E4152595F46494C455FFB
:103440005452414E534645520053455249414C5FF8
:10345000584F4E5F584F4646004649524D574152CD
:10346000455F4E414D453A4D61726C696E20322E7A
:10347000302E392E352028417072203131203230E3
:1034800032342031373A30343A31392920534F55CC
:103490005243455F434F44455F55524C3A67697408
:1034A0006875622E636F6D2F4D61726C696E46692F
:1034B000726D776172652F4D61726C696E2050522A
:1034C0004F544F434F4C5F56455253494F4E3A313C
:1034D0002E30204D414348494E455F545950453A9E
:1034E0004D616B6572626F74205265706C696361C7
:1034F000746F722045585452554445525F434F559E
:103500004E543A3220555549443A636564653261F8
:1035100032662D343161322D343734382D396231F1
:10352000322D6335356336326633363766660A00C8
:1035300020204D3235302043004C434420436F6EF1
:103540007472617374004D383400446F6E6520707E
:1035500072696E74696E672066696C650A004D3722
:1035600037004D3331002569730025696D202569C9
:1035700073002569682025696D2025697300256918
:1035800064202569682025696D20256973002569F7
:103590007920256964202569682025696D202569C1
:1035A0007300436F6F6C696E672E2E2E0045256386
:1035B0002025530042656420436F6F6C696E672E4F
:1035C0002E2E004265642048656174696E672E2E58
:1035D0002E00206661696C65642120426164206868
:1035E00065617465722069640A0050494420417520
:1035F000746F74756E650023646566696E6520443A
:10360000454641554C545F004B6420004B692000F7
:103610004B7020002066696E6973686564212050D4
:10362000757420746865206C617374204B702C2055
:103630004B6920616E64204B6420636F6E7374610C
:103640006E74732066726F6D2062656C6F7720698F
:103650006E746F20436F6E66696775726174696F0F
:103660006E2E680A00504944204175746F74756E5F
:103670006500206661696C6564212074696D656F01
:1036800075740A00504944204175746F74756E65F5
:1036900000206661696C6564212054656D706572F7
:1036A000617475726520746F6F20686967680A00BD
:1036B000504944204175746F74756E6500504944DB
:1036C000204379636C65730025532025692F256994
:1036D00000204B643A2000204B693A2000204B70B8
:1036E0003A200020436C6173736963205049442081
:1036F0000A002054753A2000204B753A2000206DB6
:1037000061783A2000206D696E3A200020643A20EA
:103710000020626961733A200048656174696E67D0
:103720002E2E2E002073746172740A0050494420BA
:103730004175746F74756E6500206661696C6564AF
:10374000212054656D706572617475726520746FA7
:103750006F20686967680A00504944204175746F9A
:1037600074756E6500504944204175746F74756EB0
:1037700065004572723A207574663820666F6E7403
:10378000206E6F7420696E697469616C697A656412
:103790002E004572723A207574663820666F6E741A
:1037A000206E6F7420696E697469616C697A6564F2
:1037B0002E00667265736800646F696E670020662C
:1037C000696C653A20004E6F7720002F6175746F29
:1037D00025632E670000002100240027002A002D09
:1037E000003000330001010000040107010A01005C
:1037F000000A0B02090C0D0E08070304010000006B
:1038000000000000000000000000000000000000B8
:103810000000000000000000000000121110000075
:103820000000000000000000000000000000000098
:1038300000000000006D61726C696E66772E6F7219
:103840006700322E302E392E35001FFFFFFFFFFF9D
:10385000FF600000000001FF400000000000FF804A
:1038600000000000007F83CF00000C303F87FF8006
:10387000000C301F867980000C000F8C30C7838CC1
:1038800030E78C30CFC7CC31F38C30DCECEC33B983
:103890008C30D86C6C33198C30D06C0C33198C3064
:1038A000D86C0C33198C30DC6C0E3B198C30CF7C0F
:1038B000079F198C30C77C038F194000000000005F
:1038C00002600000000000061FFFFFFFFFFFF8700E
:1038D000012C0190012701B0012201C0011D01F05E
:1038E0000118011002130130020E0160020901905B
:1038F000020401C002FF000003FA004003F500804B
:1039000003F000D003EB002004E6007004E100E0C7
:1039100004DC004005D700C005D2004006CD00D031
:1039200006C8008007C3003008BE00F008B900C018
:1039300009B400B00AAF00B00BAA00D00CA500007B
:103940000EA000500F9B00C0109600501291000076
:10395000148C00C0158700B0178200B0197D00D00C
:103960001B7800001E730040206E0090226900F05A
:1039700024640040275F0090295A00E02B55001076
:103980002E500020304B0010324600E033410090B2
:10399000353C001037370070383200A0392D00B0A8
:1039A0003A2800A03B2300603C1E00103D19009007
:1039B0003D1400103E0F00703E0A00C03E0500009E
:1039C0003F0000403FFBFF803FF6FFC03FF1FF207C
:1039D00020506C616E6E65724275666665724279E2
:1039E0007465733A20002046726565204D656D6FE1
:1039F00072793A200020436F6D70696C65643A20DB
:103A000041707220313120323032340A00204C6152
:103A1000737420557064617465643A2032303232B8
:103A20002D30372D3239207C20417574686F723A01
:103A3000204D2E2042616B65720A004D61726C69E7
:103A40006E20322E302E392E350A0020536F6674C8
:103A5000776172652052657365740A00205761743E
:103A60006368646F672052657365740A0020427250
:103A70006F776E206F75742052657365740A00202D
:103A800045787465726E616C2052657365740A00C6
:103A9000506F77657255700A0073746172740A0012
:103AA000473237004D31303031006F6B0065727234
:103AB0006F722077726974696E6720746F2066690F
:103AC0006C650A00446F6E6520736176696E6720CD
:103AD00066696C652E0A004D323900456E64737458
:103AE0006F707300255320256320256320256320F4
:103AF000256300205A3A0020593A0020583A0065C0
:103B00006E6473746F7073206869743A20000000EB
:103B100020002300260029002C002F003200000185
:103B20000000030106010901000022002500280011
:103B30002B002E00310034000201000005010801B5
:103B40000B01050505050705080808080202020221
:103B50000A0A080804040404010101010101010129
:103B60000303030303030303040707070C0C0C0CF4
:103B70000C0C0C0C020202020606060606060606DD
:103B80000B0B0B0B0B0B0B0B01021020200808106A
:103B900020401020408002010201080402010102BD
:103BA0000408102040808040201008040201800496
:103BB00002018040201008040201080402010102F1
:103BC000040810204080010204081020408001FFFA
:103BD000FF496E736572742066696C616D656E7401
:103BE00020616E6420707265737320627574746FE7
:103BF0006E0A00220A00556E6B6E6F776E20636F3F
:103C00006D6D616E643A202200204500205A00202C
:103C1000590020204D3932205800537465707320AC
:103C200070657220756E697400486F6D652025732C
:103C3000257325732046697273740020453A00206D
:103C40005A3A0020593A00583A004D616B65726249
:103C50006F74205265706C696361746F7220526575
:103C60006164792E005072696E74696E672E2E2E13
:103C7000005072696E7420506175736564006F6BDB
:103C80000A00526573656E643A20000056017E0199
:103C900011241FBECFEFD1E2DEBFCDBF00E00CBFCD
:103CA00084B780930F1914BE0FB6F894A89580912D
:103CB0006000886180936000109260000FBE13E086
:103CC000A0E0B2E0ECE5F4E802E00BBF02C0079030
:103CD0000D92AA3FB107D9F729E1AAEFB3E001C0DD
:103CE0001D92AF30B207E1F71EE1C7E4DEE100E06C
:103CF00006C021970109802FFE010F945C41C63454
:103D0000D10780E00807A9F70F943E2A0D941C42C2
:103D10000C9400000F931F93CF93DF93809147097A
:103D200090E0EC01CC0FDD1FCC0FDD1F8E010A5D92
:103D30001D4F880F991FFC01EE5DFD4F6081718161
:103D4000072E000C880B990B0F94B8392AE037ED39
:103D500043E25CE30F94173ACA54DA4F2881398161
:103D60004A815B810F94173AF801608371838283E3
:103D70009383DF91CF911F910F9108950F931F931C
:103D8000CF93DF938091510990E0EC01CC0FDD1FC0
:103D9000CC0FDD1F8E010A5D1D4F880F991FFC019E
:103DA000EE5DFD4F60817181072E000C880B990B31
:103DB0000F94B8392AE037ED43E25CE30F94173AE9
:103DC000CA54DA4F288139814A815B810F94173AAE
:103DD000F8016083718382839383DF91CF911F9178
:103DE0000F910895CF93DF93EC01CB01BA010F94AB
:103DF000B8392DEC3CEC4CEC5DE30F94023F0F9492
:103E00007B3F79836883DF91CF910895E0914709E3
:103E1000E23030F4F0E0EE52FA4F809136098083C0
:103E20000895809197178823C1F081508093971748
:103E3000E4EAF4E1882351F08150990B2BE1289FAB
:103E4000F001299FF00D1124E757F94E8BE1A9E805
:103E5000B4E101900D928A95E1F720919717211115
:103E600005C08091A21780648093A21781E090E042
:103E7000A0E0B0E0211103C080E090E0DC0180937D
:103E80003B0990933C09A0933D09B0933E091092E1
:103E9000A10581E080939F0583E0809375020895DA
:103EA000CF93DF93EC01CB01BA010F94B8390F9493
:103EB0007B3F6883DF91CF91089581E080934E0925
:103EC000089582E080934E0908958F929F92AF9259
:103ED000BF92CF92DF92EF92FF92CF936B017C0162
:103EE00020E030E0A9010F94B13987FFA3C06DEB4A
:103EF00077E386E095EBA70196010F94083E6B01EE
:103F00007C0120E030E040E251E40F94173A20E0D9
:103F100030E048EC52E40F94173A4B015C0120E08A
:103F200030E040E251ECC701B6010F94B1391816E8
:103F300054F420E030E048EC52E4C701B6010F949D
:103F4000684087FD8BC020E030E0A901C701B601C1
:103F50000F94B13987FF73C060E070E080EA90ECA5
:103F6000A50194010F94083E20E030E040E251E4C6
:103F70000F94023F0F94743F6B017C01F7FC64C007
:103F800020E137E240E050E00F94C63DCA01B9019C
:103F90002AE030E040E050E00F94C63D605D609361
:103FA000A305C701B60128EE33E040E050E00F94CE
:103FB000C63D9AE0892E912CA12CB12CCA01B901E1
:103FC000A50194010F94C63D605D6093A405C701EF
:103FD000B60124E630E040E050E00F94C63DCA014F
:103FE000B901A50194010F94C63D605D6093A505DC
:103FF0008EE28093A605C701B601A50194010F9436
:10400000C63DC62FCA01B901A50194010F94C63D52
:10401000605D6093A705C05DC093A80583EA95E045
:10402000CF91FF90EF90DF90CF90BF90AF909F9097
:104030008F9008956DEB77E386E095E35CCF60E0C9
:1040400070E080EA90E48CCFF094E094D094C09437
:10405000C11CD11CE11CF11C6DE2A1CF20E030E0BD
:10406000A901C701B6010F94B13987FF6AC060E0AA
:1040700070E080EA90ECA50194010F94083E20E0E6
:1040800030E040E251E40F94023F0F94743F4B0143
:104090005C0120E030E0A901C701B6010F9468403F
:1040A00087FD0BC020E030E040E251E4C701B601DB
:1040B0000F94B13960E287FD13C0B7FC47C0C5015A
:1040C000B40128EE33E040E050E00F94C63DCA0151
:1040D000B9012AE030E040E050E00F94C63D605D59
:1040E0006093A405C501B40124E630E040E050E04F
:1040F0000F94C63D8AE0C82ED12CE12CF12CCA01C8
:10410000B901A70196010F94C63D605D6093A505B6
:104110008EE28093A605C501B401A70196010F9414
:10412000C63DC62FCA01B901A70196010F94C63D2D
:10413000605D6093A705C05DC093A80584EA95E023
:104140006FCF60E070E080EA90E495CFB094A094E7
:1041500090948094811C911CA11CB11C6DE2C0CF75
:10416000CF93DF93EC01CB01BA010F94B83929EC5E
:1041700038EC48EC5EE30F94023F20E030E040E092
:104180005FE30F94083E0F947B3F6883DF91CF91EC
:104190000895CF93DF93EC01CB01BA010F94B839A6
:1041A000688379838A839B83DF91CF910895CF932E
:1041B000DF93EC01CB01BA010F94B839688379839E
:1041C0008A839B83DF91CF910895E091470986E030
:1041D000E802F0011124EE50FA4F8091360990E088
:1041E00095838483089580915109882369F0809193
:1041F000E4088770873041F482EC9DE09093F308E7
:104200008093F2081092510908958F929F92AF9275
:10421000BF92CF92DF92EF92FF92CF936B017C011E
:1042200020E030E0A9010F94B13987FDC3C06DEBE8
:1042300077E386E095E3A70196010F94083E6B01B2
:104240007C0120E030E0A9010F94B13987FFB7C0AD
:10425000C701B601905820E030E040E251E40F94ED
:10426000173A20E030E040E251E40F94173A20E0A2
:1042700030E040EA50E40F94083E20E030E040E2B5
:1042800051E40F94023F0F94743F6B017C0160E294
:1042900080EAC81686E8D80681E0E806F1048CF0CA
:1042A000C701B60120EA36E841E050E00F94C63D70
:1042B000CA01B9012AE030E040E050E00F94C63D69
:1042C000605D6093A20560E280E1C81687E2D806CF
:1042D000E104F1048CF0C701B60120E137E240E0CF
:1042E00050E00F94C63DCA01B9012AE030E040E039
:1042F00050E00F94C63D605D6093A30560E288EED8
:10430000C81683E0D806E104F1048CF0C701B601B9
:1043100028EE33E040E050E00F94C63DCA01B901F9
:104320002AE030E040E050E00F94C63D605D6093CD
:10433000A40560E284E6C816D104E104F1048CF01F
:10434000C701B60124E630E040E050E00F94C63DDE
:10435000CA01B9012AE030E040E050E00F94C63DC8
:10436000605D6093A5058AE0882E912CA12CB12C6C
:10437000C701B601A50194010F94C63DC62FCA011D
:10438000B901A50194010F94C63D605D6093A60537
:104390008EE28093A705C05DC093A80582EA95E0F0
:1043A000CF91FF90EF90DF90CF90BF90AF909F9014
:1043B0008F9008956DEB77E386E095EB3CCF20E09E
:1043C00030E040E251E4C701B60149CF8F929F929D
:1043D000AF92BF92CF92DF92EF92FF92CF936B0199
:1043E0007C0120E030E0A9010F94B13987FD93C032
:1043F0006DEB77E386E095E3A70196010F94083E05
:104400006B017C0120E030E040E251E40F94173A68
:1044100020E030E04AE754E40F94173A4B015C0186
:1044200020E030E0A901C701B6010F94B13920E0C6
:1044300030E040EA50E487FF04C020E030E040EA8A
:1044400050ECC501B4010F94083E20E030E040E29A
:1044500051E40F94023F0F94743F6B017C01C1142F
:10446000D104E104F10409F45BC0F7FE59C0F094F3
:10447000E094D094C094C11CD11CE11CF11C8DE2CD
:104480008093A305C701B60128EE33E040E050E079
:104490000F94C63D8AE0882E912CA12CB12CCA0124
:1044A000B901A50194010F94C63D605D6093A40518
:1044B0008EE28093A505C701B60124E630E040E016
:1044C00050E00F94C63DCA01B901A50194010F94B3
:1044D000C63D605D6093A605C701B601A5019401C4
:1044E0000F94C63DC62FCA01B901A50194010F94CE
:1044F000C63D605D6093A705C05DC093A80583EAD3
:1045000095E0CF91FF90EF90DF90CF90BF90AF906C
:104510009F908F9008956DEB77E386E095EB6CCFDD
:1045200080E2AECFCF93DF93EC01CB01BA010F94C1
:10453000B83920E030E040E251E40F94023F688354
:1045400079838A839B83DF91CF9108950F94B83943
:1045500020E030E040E251E40F94023F0C9405214A
:10456000CF93DF93EC01CB01BA010F94B8392AE065
:1045700037ED43E25DE30F94023F0F947B3F688386
:1045800079838A839B83DF91CF910895CF93DF93C3
:10459000EC01CB01BA010F94B8392AE037ED43E2C0
:1045A0005DE30F94023F688379838A839B83DF9165
:1045B000CF910895CF93DF93EC01CB01BA010F9413
:1045C000B839688379838A839B83DF91CF9108957B
:1045D000CF93DF93EC01CB01BA010F94B83920E0FF
:1045E00030E048EC52E40F94023F688379838A8379
:1045F0009B83DF91CF9108950F94B83920E030E08C
:1046000048EC52E40F94023F0C94651FCF93DF9364
:10461000EC01CB01BA010F94B8390F94743F798340
:104620006883DF91CF910895CF93DF93EC01CB01A5
:10463000BA010F94B83920E030E04AE754E40F940F
:10464000023F688379838A839B83DF91CF910895AA
:104650000F94B83920E030E04AE754E40F94023F69
:104660000C94E621282F8FEF80931B0210924509AE
:1046700080913B0990913C09A0913D09B0913E0980
:10468000B7FF08C010923B0910923C0910923D09F7
:1046900010923E0980919705882331F080913B0963
:1046A0008093A00510929F0580919E051816FCF43A
:1046B000082E000C990B821B91092091A005022E57
:1046C000000C330B2817390794F097FF02C090E0D5
:1046D00080E08093A005092E000CAA0BBB0B8093F1
:1046E0003B0990933C09A0933D09B0933E0980910A
:1046F000A0056623A9F09091A105891714F4809371
:10470000A1052091A105022E000C330B2C5F3F4F19
:10471000482F082E000C550B241735071CF4845025
:104720008093A10508950F931F93522F2091431654
:10473000309144162817390741F1109201049093E3
:104740004416809343168B0130E020E000933B0930
:1047500010933C0920933D0930933E094093A105F5
:1047600050939E058D5C944621F41092400910925E
:104770008F0582E08093750281E080939F051092FF
:10478000940580931B0210923A091F910F9108958E
:1047900020E040E070E060E08FE095E30C9493232C
:1047A000CF93C1E0C0934009FC0180819181A28137
:1047B000B38180931C0290931D02A0931E02B093BC
:1047C0001F0220E040E070E060E080919C05909145
:1047D0009D050E949323C0930104CF910895CF9328
:1047E000DF9300D01F92CDB7DEB78DEC9CECACEC24
:1047F000BCE389839A83AB83BC83CE0101960E947C
:10480000D0230F900F900F900F90DF91CF910895CC
:10481000CF93DF9300D01F92CDB7DEB78DEC9CEC29
:10482000ACECBDE389839A83AB83BC83CE01019654
:104830000E94D0230F900F900F900F90DF91CF9197
:104840000895CF93DF9300D01F92CDB7DEB780E0FD
:1048500090E0A0E8BFE389839A83AB83BC83CE0159
:1048600001960E94D0230F900F900F900F90DF9130
:10487000CF910895CF93DF9300D01F92CDB7DEB7CD
:1048800080E090E0A0E2B1E489839A83AB83BC83AB
:10489000CE0101960E94D0230F900F900F900F90A1
:1048A000DF91CF910895E0918F05E63028F581E002
:1048B0008E0F80938F0540913B0950913C09609188
:1048C0003D0970913E092091A10590919E0580912E
:1048D000400939E0E39FF0011124E65BFA4FA09113
:1048E0004316B0914416B183A083428353836483FB
:1048F00075832683978380870895CF93DF93EC0198
:104900000E94532420E040E070E060E0CE01DF919F
:10491000CF910C949323FC01A081B1811C92A281C0
:10492000B3818C918F5F8C930280F381E02D908115
:104930008CE0989F800D1124E5E4F6E113AE84AF7E
:104940000895FC0184910895FC01808108950097E9
:1049500051F0FC0180E09191992331F0907C9038E6
:10496000D1F38F5FF8CF80E0089590E080E0089564
:10497000CF92DF92EF92FF92CF93C82F833011F442
:1049800060932F050F941E1D6B017C0124EA30E714
:104990004DE75FE360911C0270911D0280911E0241
:1049A00090911F020F94B13987FD18C08AEF90E0F3
:1049B000A0E0B0E08C0D9D1DAE1DBF1D80933005A5
:1049C00090933105A0933205B0933305C093100244
:1049D000CF91FF90EF90DF90CF90089580E090E02E
:1049E000DC01E8CFCF92DF92EF92FF920F931F93FB
:1049F0000F941E1D009106051091070520910805D2
:104A0000309109056B017C01C01AD10AE20AF30A50
:104A10009701860137FD11C020910505209520934F
:104A200005056A547C4F8F4F9F4F60930605709326
:104A30000705809308059093090581E0909105058D
:104A4000911101C080E01F910F91FF90EF90DF90D6
:104A5000CF900895CF92DF92EF92FF920F94B839E2
:104A60006B017C0120E030E0A9010F94B1392DEBFE
:104A700037E346E055E387FF04C02DEB37E346E01C
:104A800055EBC701B6010F94083E6B017C0120E095
:104A900030E0A9010F94B13920E030E040E05FE35D
:104AA00087FF04C020E030E040E05FEBC701B601C3
:104AB0000F94083E0F94743FCB01FF90EF90DF906E
:104AC000CF900C9492BD0F94B8390F94743FCB01E2
:104AD0000C9492BD0F94B83929EC38EC48EC5EE3A5
:104AE0000F94023F20E030E040E05FE30F94083E87
:104AF0000F947B3F862F0C942ABECF93DF93CDB7C4
:104B0000DEB720E2488559856F818E810F941E158E
:104B1000DF91CF910895809147090C949ACC0F941E
:104B2000B8392DEC3CEC4CEC5DE30F94023F0F9454
:104B30007B3FCB010C94C7BDAF92BF92CF92DF9267
:104B4000EF92FF920F931F93CF93DF9361E081E089
:104B50000E943223C091A10505E00C0FD1E086E24E
:104B6000E82E8AE0F82E12E01C1B9FE2C92E9AE084
:104B7000D92EBD2EBC1AAC2EA194C1112EC0DD239E
:104B8000D9F08091A0051816BCF040913B095091D6
:104B90003C0960913D0970913E094F5F5F4F6F4F37
:104BA0007F4F40933B0950933C0960933D097093BC
:104BB0003E098F5F8093A00580917502882331F0B4
:104BC00041E06AE37AE08A2D0F949314CF5F0C13CF
:104BD000D4CF83E080939E051FC0C13041F59091F2
:104BE000A005913069F0809175028823C9F11F9268
:104BF000DF92CF92BF9281E0913051F180E028C0E6
:104C000080913F0910923F09882369F3C0934E09B0
:104C100080919F05882339F3DF91CF911F910F91E8
:104C2000FF90EF90DF90CF90BF90AF900895C2308B
:104C300069F69091A0059230A9F0809175028823C1
:104C400079F01F92FF92EF921F9381E09230B1F6BC
:104C50008F930E947D250F900F900F900F900F90D3
:104C6000D0E0B4CF80913F0910923F09882329F307
:104C7000C0934E0980919F058823F9F2CDCF809192
:104C80007502882341F0609190057091910541E093
:104C900081E00D94931408950D9421120D9419122E
:104CA0000D9411120D9409120D9401126091F814D3
:104CB0007091F9148FEB94E10D940F2160913415EC
:104CC000709135158BEF94E10D940F216091701563
:104CD0007091711587E395E10D940F216091AC15EA
:104CE0007091AD1583E795E10D940F216091E81562
:104CF0007091E9158FEA95E10D940F2160914709B4
:104D000080913609909137090C94DCCC809151093F
:104D10000E940CCD882341F020E040E070E060E08C
:104D200086E996E20C9493230C94C823EF92FF92A9
:104D30000F931F938BE4E82E8DE0F82E10E000E037
:104D40002DE43DE048EC53E26DE57DE082E69DE038
:104D50000F941D241F910F91FF90EF900895EF92F3
:104D6000FF920F931F938FE3E82E8CE0F82E10E054
:104D700000E020EC3CE04DE45EE361E47CE086E4AE
:104D80009CE00F941D241F910F91FF90EF900895C8
:104D9000EF92FF920F931F938EE4E82E88E0F82E97
:104DA00010E000E021E638E043E55EE260E578E00F
:104DB00087E598E00F941D241F910F91FF90EF90CD
:104DC0000895CF92DF92EF92FF920F931F93CF93AC
:104DD000DF93CDB7DEB7CDB6DEB68091FC1169E7C3
:104DE0007FE0882311F06CEF71E1FB01019000205E
:104DF000E9F7CF01861B970B01962DB73EB7281B0D
:104E0000390B0FB6F8943EBF0FBE2DBF0DB71EB7BE
:104E10000F5F1F4F80E2EDB7FEB78183C801019697
:104E20000F94ED4183EEE82E8CE0F82E25EE3CE069
:104E300041E05EE261EF7CE088EF9CE00F941D248E
:104E40000FB6F894DEBE0FBECDBEDF91CF911F919D
:104E50000F91FF90EF90DF90CF9008950F948E10F8
:104E600010924F09109274020E9473CD882351F062
:104E70008091A21782FD06C082E697E09093F30826
:104E80008093F2080C94A6BB0F94B8390F947B3F23
:104E9000862F0C9408BECF93DF9300D0CDB7DEB73A
:104EA0008FEF89838A838B83CE0101960E94F6CA95
:104EB0000F900F900F90DF91CF910895CF93DF93D4
:104EC00000D0CDB7DEB78FEF89831A821B82CE0167
:104ED00001960E94F6CA0F900F900F90DF91CF912C
:104EE0000895CF93DF9300D0CDB7DEB78FEF8983DE
:104EF00089E18A831B82CE0101960E94F6CA0F9037
:104F00000F900F90DF91CF910895CF93DF9300D052
:104F1000CDB7DEB78FEF89838BE48A831B82CE0106
:104F200001960E94F6CA0F900F900F90DF91CF91DB
:104F30000895CF93DF9300D0CDB7DEB719821A82E0
:104F40008FEF8B83CE0101960E94F6CA0F900F90CF
:104F50000F90DF91CF910895CF93DF9300D0CDB71D
:104F6000DEB719828FEF8A838B83CE0101960E9470
:104F7000F6CA0F900F900F90DF91CF910895CF93C5
:104F8000DF9300D0CDB7DEB78FEF89831A828B8392
:104F9000CE0101960E94F6CA0F900F900F90DF91FC
:104FA000CF910895CF93DF9300D01F92CDB7DEB796
:104FB0000F947B3F0F94B63969837A838B839C83EC
:104FC000CE0101960E9414BC0F900F900F900F908D
:104FD000DF91CF9108950F94B8392AE037ED43E27D
:104FE0005DE30F94023F0C94D227CF92DF92EF92B1
:104FF000FF92CF93DF9300D01F92CDB7DEB76B0146
:105000007C0120E030E0A9010F94B13987FD1BC07D
:105010006DEB77E386E095E3A70196010F94083ED8
:1050200069837A838B839C83CE0101960E9414BC92
:105030000F900F900F900F90DF91CF91FF90EF9016
:10504000DF90CF9008956DEB77E386E095EBE4CFAA
:105050000F94B8392AE037ED43E25DE30F94023F45
:105060000C94F5270F94B8390C94F527CF92DF9262
:10507000EF92FF926B017C0120E030E0A9010F94D8
:10508000B13987FD26C06DEB77E386E095E3A70194
:1050900096010F94083E6B017C0120E030E0A901ED
:1050A0000F94B13920E030E040E05FE387FF04C0B7
:1050B00020E030E040E05FEBC701B6010F94083E0E
:1050C0000F94743FCB01FF90EF90DF90CF900C9442
:1050D00013BD6DEB77E386E095EBD9CF0F94B8392C
:1050E0000C9436280C945B8F0C945B8F0C940D8F72
:1050F0000C940D8F0C940D8F0C940D8FEF92FF92EA
:105100000F931F93CF93DF93EC018B017A018A8574
:105110009B858617970731F0888199810F9419250F
:105120001B870A87B701888199810F948B152E817F
:105130003F81820F932F911D9F838E8390E080E0AB
:10514000DF91CF911F910F91FF90EF9008959F9263
:10515000AF92BF92CF92DF92EF92FF920F931F9385
:10516000CF93DF93EC018B01942EA52E8A859B852E
:105170008617970731F0888199810F9419251B872D
:105180000A8788859985019649F5BC800A818E81B8
:10519000080FC880D980D6015596ED91FC91C601C3
:1051A0001995B80EE92CFA2C10E0F70121917F0136
:1051B000211127C08E819F81810F911D9F838E8336
:1051C00090E080E0DF91CF911F910F91FF90EF90E1
:1051D000DF90CF90BF90AF909F9008950E811F8178
:1051E000692D7A2D888199810F948B15800F912FCD
:1051F000911D288539852817390738F681E090E018
:10520000E1CF4B2D602FC6010F947125080F180FA9
:10521000CCCFDF92EF92FF920F931F93CF93DF9348
:10522000EC01D62E1CAD0BAD7C0184E0E80EF11C28
:10523000E98DFA8DC7011995412F480F2D2D602F4B
:10524000C7010F9471259BAD890F8BAF81E090E072
:10525000DF91CF911F910F91FF90EF90DF90089514
:10526000AF92BF92DF92EF92FF920F931F93CF9373
:10527000DF938C01EB01D42E79018FE0481709F4FC
:1052800088C0A5E14A17C1F1BAE04B130EC0EC810A
:10529000FD8130E020E042E061E0C801199542E282
:1052A00056E0BE01C8010F941C260A80DB81C02D88
:1052B000F2E3DF1609F4E4C0FD1508F493C085E1BC
:1052C000D81609F4E2C0A7E1DA1609F4FCC0B4E18B
:1052D000DB127DC0EE81FF818D8190E0880F991FE8
:1052E0008E0F9F1F11928E179F07E1F71A828881F8
:1052F00081508B831C826BC0AA80BB804DE056E03E
:10530000C8010F941C26F5014481440F406BBE0177
:10531000C8010F94042641E0BE01C8010F940C2679
:10532000D50116962D913C911797EC81FD8115962C
:105330004C9166E0C801199540E0BE01C8010F9488
:1053400014264DE056E0BE01C8010F941C26F5015D
:105350004481440F4F5F406BBE01C8010F94042687
:1053600041E0BE01C8010F940C26D50115964C9161
:10537000159716962D913C91240F311DEC81FD81DE
:1053800066E0C801199540E0BE01C8010F941426DB
:105390008CCF41E0C8010F94142640E0BE01C80143
:1053A0000F940C2641E8BE01C8010F940426F701B2
:1053B000408150E05595479555954795BE01C801E8
:1053C0000F94042640E0BE01C8010F94142681E02A
:1053D000DF91CF911F910F91FF90EF90DF90BF90E1
:1053E000AF900895E6E4DE1609F47CC0F7E4DF161A
:1053F00009F47CC08BE3D812EACFD70111969C91B7
:10540000119713968C9138E0390F813031F0833049
:1054100011F0392F02C0392F985021E04B814917E4
:1054200008F420E041E0391708F040E091E05A81AB
:10543000351708F490E0322F342B932311F42423F2
:1054400031F2F701128100E0D12C843048F490E071
:10545000FC01EC55FD4FD08080569D4FDC010C9136
:1054600017FF04C0B701CE010F941222F70180810B
:105470008D0D80838181800F8183110F89F7A7CFE4
:10548000B701CE010F941222A2CF88819A81980F82
:105490009A832981921770F59C819F5F9C839B81E1
:1054A000890F821710F08FEF820F8B83EE81FF81BF
:1054B0008D8190E0880F991F8E0F9F1F11928E177C
:1054C0009F07E1F784CFD7011C928A8111968C93B4
:1054D00011978D81815012968C9312978B81139620
:1054E0008C9375CF8D81F701808371CF8981D7012E
:1054F0008C936DCF80E06CCF8F929F92AF92BF92D2
:10550000CF92DF92EF92FF920F931F93CF93DF938F
:10551000CDB7DEB760970FB6F894DEBF0FBECDBF34
:105520008B0140E050E068EC72E449875A876B8752
:105530007C8740E050E060EA70E44D875E876F87CB
:10554000788B8130B9F1823009F462C020E030E01C
:1055500040E050E460917E0270917F028091800271
:10556000909181020F94083E4B017C0120E030E0D5
:1055700046E153E40F946840181634F4812C912CC2
:1055800086E1E82E93E4F92EF801A084B184C28468
:10559000D3849401A701B501C6010F946840181681
:1055A00014F054016701C501D60189839A83AB8346
:1055B000BC8351C0BE01635F7F4FC80108960E9443
:1055C000C4B488E0F801DE01119601900D928A952D
:1055D000E1F7AE01475F5F4FBE016B5F7F4FCE01CA
:1055E00001960E94A2B40E94BBB860960FB6F894D0
:1055F000DEBF0FBECDBFDF91CF911F910F91FF9006
:10560000EF90DF90CF90BF90AF909F908F900895D4
:10561000F801208531854285538560917E02709125
:105620007F0280918002909181020F94083E6B016D
:105630007C0120E030E046E153E40F94B13987FD6E
:1056400006C0C12CD12C26E1E22E23E4F22EC98221
:10565000DA82EB82FC82BE01635F7F4FCE0101964E
:10566000AECF0F931F930F941E1D0091CB08109186
:10567000CC082091CD083091CE08011511052105E7
:105680003105D9F5209131162223A1F1E0912F1691
:1056900021502093311621E02E0F20932F163091A8
:1056A0003216231302C010922F1624E0E29FF0015D
:1056B0001124ED5CF94E0081118122813381009328
:1056C000C7081093C8082093C9083093CA08600F10
:1056D000711F811D911D6093CB087093CC0880933E
:1056E000CD089093CE088091C9089091CA08892B63
:1056F00009F0409A1F910F910895601B710B820B66
:10570000930B97FDF7CF40981092CB081092CC08DE
:105710001092CD081092CE08EDCF0F931F93CF9328
:10572000DF938C01EB019091311620913216921388
:1057300005C00E94312B0E94A591F5CF80913016B3
:1057400034E0839FF0011124ED5CF94E1183008356
:10575000D383C2839F5F909331168F5F281739F0F0
:1057600080933016DF91CF911F910F910895109281
:105770003016F8CF63E972E084E690E00E948D2B4A
:1057800070E060E08AE090E00E948D2B6AEB72E0AE
:1057900084E690E00C948D2B0E947CB90C94BA2B7B
:1057A00081110C94BA2B68E270E080E991E00C94CE
:1057B0008D2B0E94648B0C94D02B0E940FC50C94EF
:1057C000D02B4FE350E0BC0184EF98E00D940242EF
:1057D0000F931F93CF93DF93CDB7DEB72C970FB600
:1057E000F894DEBF0FBECDBF80914709282F082E49
:1057F000000C330B3F938F9385E99BE09F938F932E
:105800008E010F5F1F4F1F930F930F944839C801EC
:105810000E94E12B0F900F900F900F900F900F9020
:105820002C960FB6F894DEBF0FBECDBFDF91CF919F
:105830001F910F9108950C94E82B0F931F93CF9312
:10584000DF93CDB7DEB72C970FB6F894DEBF0FBE4F
:10585000CDBF80914709282F082E000C330B3F93B2
:105860008F938CE89BE09F938F938E010F5F1F4F68
:105870001F930F930F944839C8010E94E12B0F909A
:105880000F900F900F900F900F902C960FB6F894EA
:10589000DEBF0FBECDBFDF91CF911F910F91089555
:1058A0000C941D2C0F931F93CF93DF93CDB7DEB7CE
:1058B0002F970FB6F894DEBF0FBECDBF809147097A
:1058C000282F082E000C330B3F938F9380E89BE02A
:1058D0009F938F938E010F5F1F4F1F930F930F9412
:1058E0004839C8010E94E12B0F900F900F900F9044
:1058F0000F900F902F960FB6F894DEBF0FBECDBF5E
:10590000DF91CF911F910F9108950C94522CEF923B
:10591000FF920F931F93CF93DF9300D000D000D05E
:105920001F921F92CDB7DEB77C0120919205422FC6
:10593000022E000C550B80919305833089F1843041
:1059400041F185E999E05F932F939F938F938E01A7
:105950000F5F1F4F1F930F930F944839609192056B
:10596000C7010E94DCCCC8010E94E12B0F900F9070
:105970000F900F900F900F902B960FB6F894DEBFFC
:105980000FBECDBFDF91CF911F910F91FF90EF9090
:10599000089581EA99E027FDD6CF8CE899E0D3CF2E
:1059A0008AEA99E0D0CFE091470986E0E802F00169
:1059B0001124EE50FA4F808191810C94872CE09154
:1059C000470987E1E89FF0011124E15CF94F8085E8
:1059D00091850C94872C2F923F924F925F926F92F9
:1059E0007F928F929F92AF92BF92CF92DF92EF926F
:1059F000FF920F931F93CF93DF9300D000D0CDB7CA
:105A0000DEB71C017A8369832B833C834D835E83DD
:105A10002701380181E080939F050E94532483E091
:105A20008093750230928E0520928D0589819A812E
:105A300090938C0580938B058B819C81AD81BE8179
:105A40008093870590938805A0938905B0938A0574
:105A50004092830550928405609285057092860578
:105A6000F12CE12CC0923B09D0923C09E0923D0917
:105A7000F0923E09B0924416A0924316909282058D
:105A8000809281058C8D8093800526960FB6F894C0
:105A9000DEBF0FBECDBFDF91CF911F910F91FF9061
:105AA000EF90DF90CF90BF90AF909F908F907F90BE
:105AB0006F905F904F903F902F90089520E040E0CE
:105AC00070E060E08DEC94E60C9493230E9497CDF7
:105AD0000E94B4850C945E2DCF93DF93782FC62F50
:105AE000D42F67FD36C086E06802F0011124EE5025
:105AF000FA4F408151811416150684F4E72FF0E027
:105B0000EE0FFF1FE054FD4F808191810F974817E2
:105B100059070CF4CA01672F0E94DCCCD7FF1BC0C9
:105B2000E0915109E23008F0E0E0F0E0EE52FA4F87
:105B300086E0C802D0011124AE50BA4F14968D9160
:105B40009C918F3F910519F010F08FEF90E08083CA
:105B50001AC047FD18C086E0D802F0011124EE50AB
:105B6000FA4F82819381181619065CF484369105E8
:105B700014F084E690E090933706809336060E94F6
:105B800022C6C7FFCDCFDF91CF910C945E2D0F932E
:105B90001F93CF93DF93C6E3D9E0E88186E0E80264
:105BA000F0011124EE50FA4F0081118160E0C8012C
:105BB0000E94DCCC61E0C8010E94DCCC48816FEF20
:105BC00080E0DF91CF911F910F910C946C2D0C947C
:105BD000C72D60913609462F809147090C946C2D92
:105BE0000C94E92D4FEF60913609809147090C9490
:105BF0006C2D0C94F22D409136096FEF80E00C94DF
:105C00006C2D89E79FE00E949B790E945E2D0D9488
:105C10008E10611160931A02409300048C3008F0DA
:105C20003AC0E82F880FFF0B8827E65EF14D8F4FB3
:105C30000D945C414D2E262E312E502E342E372EB3
:105C40003A2E462E3D2E4B2E402E432E8CE094E4D1
:105C500021E02093400920E040E070E060E00C94F7
:105C6000932384E194E4F4CF88E194E4F1CF8CE1D0
:105C700094E4EECF80E294E4EBCF84E294E4E8CFC6
:105C800088E294E4E5CF8CE294E4E2CF10924E09EE
:105C90008CE995E2DDCF0C945E2D88E094E4D8CFBA
:105CA00080E194E4D5CFCF930E947CB90E94648BAD
:105CB000C82F882319F080E00E942E8A8C2F0E9422
:105CC000D02BCF910C945E2D8CE598E09093F30847
:105CD0008093F2080C945E2DCF93DF93C0918F05D3
:105CE000CC23B9F0C150C0938F0589E0C89FE00173
:105CF0001124C65BDA4F6A817B812F814E818881B6
:105D000099810E949323888580934009DF91CF91E8
:105D10000895DF91CF910C945E2DEF92FF920F9337
:105D20001F93CF93DF9361E081E00E943223C09103
:105D3000A10585E0F82EFC0ED2E0DC1B11E01C1B57
:105D4000EC2EE194C1112BC00091A0050023A1F01D
:105D500080917502882349F081E0011180E024E000
:105D60004AEA5EE06E2D0F941E15CF5FFC12EACF5B
:105D700083E080939E050CC080913F0910923F09FB
:105D8000882331F30E946C2E80919F05882301F3B4
:105D9000DF91CF911F910F91FF90EF900895C13047
:105DA00001F50091A005013069F08091750288230A
:105DB000E1F281E0013009F080E023E04BE95EE0B0
:105DC000612FD1CF80913F0910923F09882369F359
:105DD00084E49BE40E947D2480919F05882329F31D
:105DE000D7CFC23011F60091A005023071F080913A
:105DF0007502882309F4B9CF81E0023009F080E010
:105E000023E04DE85EE06D2FAECF80913F09109208
:105E10003F09882361F382E99CE40E947D248091FC
:105E20009F05882321F3B4CF2F923F924F925F9228
:105E30006F927F928F929F92AF92BF92CF92DF929A
:105E4000EF92FF920F931F93CF93DF9300D01F9297
:105E5000CDB7DEB70091360961E081E00E943223C0
:105E60002091A1052B8310E0000F111F075E114F39
:105E7000422E2B5F2983842D81958A8341E0E42E75
:105E80004EE0F42E51EFC52E5DE0D52E63EEA62E2A
:105E90006DE0B62E85E0582E541875ED872E7DE006
:105EA000972E2B81211114C08091A0058C8388230B
:105EB00009F4E3C080917502882351F081E09C8150
:105EC000911180E024E04DE05EE06A810F941E15A0
:105ED000612C21E02C833B8034188B819C818913B9
:105EE0002DC0E0913609F0E0EE0FFF1FE75EF14FA5
:105EF000859194916092470990934B0980934A0948
:105F000010924909109248097090A0052B817216D1
:105F100009F4D8C080917502882381F01F92FF9206
:105F2000EF923F9281E09C81791280E08F930E94F2
:105F30007D250F900F900F900F900F907C80872DF4
:105F40008F5F2B8182132CC0E0913609F0E0EE0FB9
:105F5000FF1FE75EF14F85919491609247099093FE
:105F60004B0980934A0910924909109248092090E0
:105F7000A005221609F4B5C080917502882381F02E
:105F80001F92DF92CF923F9281E09B81291280E0A5
:105F90008F930E947D250F900F900F900F900F9080
:105FA00063942C812E5F2C83253009F096CF8B8152
:105FB000853041F5F80185919491109247099093AD
:105FC0004B0980934A09109249091092480990910F
:105FD000A0059C83953009F493C0809175028823B5
:105FE00089F01F92BF92AF925F9281E02C812530A1
:105FF00009F080E08F930E947D250F900F900F9005
:106000000F900F9083E0870D9B8189132BC0F801BF
:10601000859194911092470990934B0980934A0976
:1060200010924909109248092091A0052C838B8178
:10603000281709F474C080917502882399F01F9283
:106040009F928F928B8184198F9381E09C812B8109
:10605000921380E08F930E947D250F900F900F90F8
:106060000F900F908B818F5F8B839981891319CF4C
:1060700084E0870D80939E050EC080913F091092A9
:106080003F09882309F416CF0E946C2E80919F054A
:10609000882309F40FCF0F900F900F900F90DF918E
:1060A000CF911F910F91FF90EF90DF90CF90BF9015
:1060B000AF909F908F907F906F905F904F903F90A8
:1060C0002F90089580913F0910923F09882309F489
:1060D00021CF0E94E92D80919F05882309F41ACFD2
:1060E000DACF80913F0910923F09882309F444CF09
:1060F0000E94F22D80919F05882309F43DCFCBCFDC
:1061000080913F0910923F09882309F466CF0E94CD
:10611000C72D80919F05882309F45FCFBCCF809164
:106120003F0910923F09882309F485CF4091360931
:106130006FEF80E00E946C2D80919F05882309F409
:106140007ACFA9CF6F927F928F929F92AF92BF9298
:10615000CF92DF92EF92FF920F931F93CF93DF9333
:1061600061E081E00E943223C091A1059C2E85E070
:10617000C82ECC0E9EE9A92E9DE0B92ED6E0DC1BE0
:10618000EE24E39422E0D22E15E01C1B04E00C1B4D
:1061900083E0F82EFC1A8D2C8C1A7E2C7C1AC111EF
:1061A00034C06090A0056620A9F080917502882314
:1061B00051F0692D619581E0611080E024E040EDAF
:1061C0005DE00F941E15CF5FCC11E9CF87E080937F
:1061D0009E050CC080913F0910923F09882329F346
:1061E0000E946C2E80919F058823F9F2DF91CF9158
:1061F0001F910F91FF90EF90DF90CF90BF90AF90E5
:106200009F908F907F906F900895C13001F56090BE
:10621000A00581E0681661F080917502882399F2EB
:1062200081E0681280E023E046EC5DE0672DC9CF95
:1062300080913F0910923F09882371F381E092E336
:106240000E947D2480919F05882331F3CFCFC230F7
:1062500009F0B9C09091A005923071F0809175025B
:10626000882309F4B0CF81E0923009F080E020E289
:1062700048EB5DE0682DA5CF80913F0910923F0962
:10628000882361F322EC3DE03093F3082093F20879
:1062900080919F05882311F3A9CF1092470910928E
:1062A0004B0910924A09109249091092480990919D
:1062B000A005933071F080917502882309F483CF93
:1062C00081E0933009F080E020E24CEA5DE06F2D40
:1062D00078CF80913F0910923F09882361F323EB27
:1062E0003DE03093F3082093F20880919F058823C6
:1062F00011F37CCFE092470910924B0910924A09A2
:1063000010924909109248099091A005943071F0BB
:1063100080917502882309F456CF81E0943009F00A
:1063200080E020E24CEA5DE0602F4BCF80913F0996
:1063300010923F09882361F327EA3DE03093F30888
:106340002093F20880919F05882311F34FCFD092BC
:10635000470910924B0910924A091092490910926C
:1063600048099091A005953071F0809175028823BD
:1063700009F429CF81E0953009F080E020E24CEA71
:106380005DE0612F1ECF80913F0910923F09882365
:1063900061F322EA3DE03093F3082093F208809104
:1063A0009F05882311F322CF80913F0910923F0966
:1063B0008823C9F0B092F308A092F20880919F055B
:1063C000882389F013CFC33009F467CFC43009F4B0
:1063D00091CFC53009F4BBCFC63009F0F4CE90910F
:1063E000A005963009F380917502882309F4EBCE5D
:1063F00081E0963009F080E020E24DE85DE06D2F0D
:10640000E0CE8F929F92AF92BF92CF92DF92EF92A7
:10641000FF920F931F93CF93DF9361E081E00E947F
:106420003223C091A10585E0B82EBC0ED1E016E064
:106430001C1B05E00C1B84E0F82EFC1A92E0D92E00
:1064400083E0E82EEC1AAD2CAC1A9D2E9C1A8C2EF3
:106450008194C11131C0C090A005CC20A1F08091E1
:106460007502882349F081E0C11080E024E046E80D
:106470005DE0682D0F941E15CF5FCB11EACF87E04A
:1064800080939E050CC080913F0910923F0988239C
:1064900031F30E946C2E80919F05882301F3DF91D8
:1064A000CF911F910F91FF90EF90DF90CF90BF9011
:1064B000AF909F908F900895C13051F51092470989
:1064C00010924B0910924A091092490910924809FA
:1064D000C090A00581E0C81661F080917502882304
:1064E00059F281E0C81280E023E04FE75DE0692DBA
:1064F000C1CF80913F0910923F09882371F388E052
:1065000095E30E947D2480919F05882331F3C7CFB6
:10651000C23009F0B5C0D093470910924B091092D0
:106520004A091092490910924809C090A00592E0CA
:10653000C91671F080917502882309F49DCF81E01E
:1065400092E0C91280E023E04FE75DE06A2D92CF30
:1065500080913F0910923F09882361F381E095E320
:106560000E947D2480919F05882321F398CFD092AB
:10657000470910924B0910924A091092490910924A
:106580004809C090A00583E0C81671F0809175029B
:10659000882309F471CF81E093E0C91280E023E001
:1065A0004FE75DE06E2D66CF80913F0910923F0965
:1065B000882361F38AEF94E30E947D2480919F05F4
:1065C000882321F36CCFC090A00584E0C81671F039
:1065D00080917502882309F44FCF81E094E0C912BD
:1065E00080E023E041E75DE06F2D44CF80913F09DB
:1065F00010923F09882361F386E896E20E947D2489
:1066000080919F05882321F34ACF10924709109269
:106610004B0910924A091092490910924809C090FA
:10662000A00585E0C81671F080917502882309F4F1
:1066300023CF81E095E0C91280E023E04AE65DE0E7
:10664000602F18CF80913F0910923F09882361F392
:1066500084EF94E30E947D2480919F05882321F399
:106660001ECF80913F0910923F09882321F18EEEC1
:1066700094E30E947D2480919F058823E1F00FCF51
:10668000C33009F474CFC43009F49DCFC53009F488
:10669000BCCFC63009F0F0CED093470910924B0919
:1066A00010924A091092490910924809C090A00519
:1066B00086E0C816B1F280917502882309F4DCCE19
:1066C00081E096E0C91280E023E04AE65DE0612FB8
:1066D000D1CE7F928F929F92AF92BF92CF92DF9254
:1066E000EF92FF920F931F93CF93DF93F82E842E98
:1066F00070939D0560939C0561E081E00E943223C8
:10670000C091A10585E0982E9C0ED1E007E21DE026
:1067100085E0E82EEC1A84E0D82EDC1A83E0C82E3F
:10672000CC1A82E0B82EBC1A7D2E7C1AAC2EA19415
:1067300083E0F81609F44EC0C11196C0F0924709E3
:1067400010924B0910924A09109249091092480977
:10675000DD23D9F08091A0051816BCF040913B09CB
:1067600050913C0960913D0970913E094F5F5F4F28
:106770006F4F7F4F40933B0950933C0960933D0915
:1067800070933E098F5F8093A005809175028823E6
:1067900031F043E06FE77DE08A2D0F94931482E09F
:1067A000F8125BC0C530A1F41092470910934B0951
:1067B00000934A091092490910924809D091A00506
:1067C000D53009F4D9C0809175028111E6C0D0E0BE
:1067D00086E044C08091820290918302A09184025D
:1067E000B09185028093980590939905A0939A059E
:1067F000B0939B05C11138C08092470910924B0994
:1068000010924A091092490910924809DD23D9F0E3
:106810008091A0051816BCF040913B0950913C09AD
:1068200060913D0970913E094F5F5F4F6F4F7F4F01
:1068300040933B0950933C0960933D0970933E0996
:106840008F5F8093A00580917502882331F043E02B
:106850006AE67DE08A2D0F94931485E0CF5F9C1249
:1068600067CF80939E0522C0C13071F5D091A005FD
:10687000D13081F080917502882351F081E0D130D0
:1068800009F080E024E046EC5DE0672D0F941E15D2
:10689000D0E085CF80913F0910923F09882351F3C2
:1068A0000E946C2E80919F05882321F3DF91CF9168
:1068B0001F910F91FF90EF90DF90CF90BF90AF901E
:1068C0009F908F907F900895C23009F071C0D09151
:1068D000A005D23069F0809175028823C9F281E069
:1068E000D23009F080E023E041E45DE06B2DCECFB3
:1068F00080913F0910923F09882369F38AE394E26B
:106900000E947D2480919F05882329F3CFCF809119
:106910003F0910923F09882309F452C081E294E2B2
:106920000E947D2480919F05882309F449C0BECF31
:10693000C43009F034CFD091A005D43071F08091EB
:106940007502882309F4A4CF81E0D43009F080E0F7
:1069500023E04DE25DE06D2D99CF80913F091092CB
:106960003F09882361F388E094E20E947D248091AE
:106970009F05882321F39ACF80913F0910923F0908
:10698000882309F420CF8FEE93E20E947D2480912A
:106990009F05882309F417CF89CF81E0D53009F00E
:1069A00080E023E04EE15DE06E2D0F941E150FCFC9
:1069B000C33009F0BDCFD091A005D33009F4A7CFE3
:1069C00080917502882309F463CF81E0D33009F008
:1069D00080E023E048E35DE06C2D58CF41E06CE4BB
:1069E00075E483E00C94693340E06FE475E483E080
:1069F0000C9469334091510963E377E482E00C948D
:106A000069334091510966E377E481E00C9469337E
:106A10004091510969E377E480E00C946933409137
:106A2000510962E575E483E00C9469332F923F923B
:106A30004F925F926F927F928F929F92AF92BF928E
:106A4000CF92DF92EF92FF920F931F93CF93DF933A
:106A500000D000D01F92CDB7DEB70E9462CD482E85
:106A600061E081E00E9432237090A105572C25E05F
:106A7000270D298382E087198A8381E087198B8318
:106A8000872D81958C8309ED1BE29EE3E92E99E029
:106A9000F92E2CECC22E2BE2D22E3FE1A32E39E0B0
:106AA000B32E4DED842E4BE2942E711000C19091C7
:106AB000A0059D83992309F4D3C080917502882392
:106AC00009F4A3C181E02D81211180E024E047E891
:106AD00059E06C810F941E1582E041103AC183E0A9
:106AE0008D838D81871115C09091A0059E83981785
:106AF00009F437C180917502882359F0672D651913
:106B000081E02E81271180E023E04CE559E00F94CD
:106B10001E156D8063941F821E82272C2518761007
:106B200025C0EE81FF81EE0FFF1FE75EF14F8591DB
:106B300094912E812093470990934B0980934A09A1
:106B400010924909109248093090A005371409F4B1
:106B50001EC180917502882349F081E0361080E0E3
:106B600023E04DE459E0622D0F941E15362C662467
:106B70006394630C8E819F81019709F003C16710B4
:106B80001EC08091A005871509F412C1809175027D
:106B90008823A9F01F930F93FF92EF92872D8519F9
:106BA0008F9381E09091A005971180E08F930E94D0
:106BB0007D250F900F900F900F900F900F9082E017
:106BC000830D411046C0871120C08091A005871514
:106BD00009F4FDC0809175028823B9F09F928F92CD
:106BE00080E399E09F938F93872D85198F9381E0A0
:106BF0009091A005971180E08F930E947D250F90C2
:106C00000F900F900F900F900F9083E0830D8711DE
:106C10001EC08091A005871509F4E8C08091750217
:106C20008823A9F0DF92CF92BF92AF92872D85196A
:106C30008F9381E09091A005971180E08F930E943F
:106C40007D250F900F900F900F900F900F9084E084
:106C5000830D73949981971128CF80939E050EC060
:106C600080913F0910923F09882309F426CF0E94A2
:106C70006C2E80919F05882309F41FCF27960FB6AD
:106C8000F894DEBF0FBECDBFDF91CF911F910F9162
:106C9000FF90EF90DF90CF90BF90AF909F908F903C
:106CA0007F906F905F904F903F902F90089591E06C
:106CB000791214C02091A0052D83213001F180911B
:106CC0007502882359F081E09D81913009F080E0C0
:106CD00023E045E759E06B810F941E1541103BC03E
:106CE00022E072123BC08091A0058D838230B1F00A
:106CF00080917502811121C093E09D830ACF80911C
:106D00003F0910923F098823D1F287EB93E50E9457
:106D10007D2480919F05882391F2B0CF80913F0917
:106D200010923F09882321F386E096E50E947D2496
:106D300080919F058823E1F2A1CF81E02D8122304F
:106D400009F080E023E048E659E06A810F941E15BF
:106D500083E08D83DECE92E09D83C3CE23E02D833E
:106D6000C0CE80913F0910923F09882309F4C2CE1A
:106D70008FEE97E50E947D2480919F05882309F47A
:106D8000B9CE7CCF81E090E09F838E83C8CE809186
:106D90003F0910923F09882309F4DBCE8EEB98E57A
:106DA0000E947D2480919F05882309F4D2CE66CF6E
:106DB00080913F0910923F09882309F4E7CE0E9491
:106DC000D92B80919F05882309F4E0CE57CF80917D
:106DD0003F0910923F09882309F4FCCE0E94DD2B65
:106DE00080919F05882309F4F5CE48CF80913F0913
:106DF00010923F09882309F411CF0E94CC2B809177
:106E00009F05882309F40ACF39CF442009F474CFB1
:106E100022E02D837ECE2F923F924F925F926F920F
:106E20007F928F929F92AF92BF92CF92DF92EF921A
:106E3000FF920F931F93CF93DF9300D0CDB7DEB7B0
:106E40000E9481CD8111EEC082E0809336090E94BC
:106E500062CD682E61E081E00E9432232091A1057D
:106E60002A83722E2B5F2983572C51949FE0C92EC1
:106E70009AE0D92E28E0A22E2AE0B22E3FEF832EF0
:106E800039E0932E8A81811114C09091A0059B83D3
:106E9000992309F4C9C080917502882351F081E0DB
:106EA000EB81E11180E024E041E25AE0652D0F948E
:106EB0001E150FE316E07801F1E0FB834A804A9447
:106EC0003A803718F701808591850E94F7CC882396
:106ED00009F4E2C0FA812B81F2131DC040924709E8
:106EE00010924B0910924A091092490910924809D0
:106EF0002090A0052F1609F4BEC08091750288234A
:106F000051F081E09A81291280E023E04FE05AE0BD
:106F1000632D0F941E158B818F5F97E1E90EF11C95
:106F2000EB81E23009F0A4C0611073C08B838FE362
:106F3000E82E86E0F82E412C3A803718F70180853C
:106F400091850E94F7CC882309F4F1C0FA812B8146
:106F5000F2131DC04092470910924B0910924A0942
:106F600010924909109248092090A0052F1609F4A3
:106F7000CDC080917502882351F081E09A81291259
:106F800080E023E048E05AE0632D0F941E158B81CA
:106F90008F5F97E1E90EF11CEB81EF5FEB83F1E08E
:106FA0004F12B1C08B83F12CEA80E718F80180857D
:106FB00091850E94F7CC882309F404C1FA812B81C2
:106FC000F2131DC0F092470910924B0910924A0922
:106FD00010924909109248094090A0054F1609F4F3
:106FE000E0C080917502882351F081E09A814912B6
:106FF00080E023E04FEF59E06E2D0F941E158B813A
:107000008F5F095E1F4F9B819F5F9B83E1E0FE12B4
:10701000C5C0FA81FF5FFA8329812F1333CF809394
:107020009E0510C081E011CF80913F0910923F0969
:10703000882309F430CF0E946C2E80919F0588230D
:1070400009F429CF0F900F900F90DF91CF911F91EE
:107050000F91FF90EF90DF90CF90BF90AF909F90F7
:107060008F907F906F905F904F903F902F900895FA
:1070700022E02B8327CF80913F0910923F0988237C
:1070800009F43BCF82EB93E50E947D2480919F051C
:10709000882309F432CFD6CFEA81FB81EF133BCFAF
:1070A0004092470910924B0910924A0910924909DF
:1070B000109248098091A0058E17C1F08091750249
:1070C000882309F428CF1F92DF92CF923F9281E06C
:1070D0009091A0052A81921380E08F930E947D25D4
:1070E0000F900F900F900F900F9015CF80913F0948
:1070F00010923F09882311F30E94522C80919F0522
:107100008823E1F29FCF4424439418CF80913F0914
:1071100010923F09882309F42CCF8DEA93E50E9451
:107120007D2480919F05882309F423CF8BCFEA81AA
:10713000FB81EF132CCF4092470910924B0910921C
:107140004A0910924909109248098091A0058E17AA
:10715000C1F080917502882309F419CF1F92BF9264
:10716000AF923F9281E09091A0052A81921380E036
:107170008F930E947D250F900F900F900F900F908E
:1071800006CF80913F0910923F09882311F30E9496
:107190001D2C80919F058823E1F254CFFF24F394A6
:1071A00005CF80913F0910923F09882309F419CF38
:1071B00088EA93E50E947D2480919F05882309F445
:1071C00010CF40CFEA81FB81EF1319CFF09247092E
:1071D00010924B0910924A091092490910924809DD
:1071E0008091A0058E17C1F080917502882309F463
:1071F00006CF1F929F928F92EF9281E09091A0050F
:107200002A81921380E08F930E947D250F900F902A
:107210000F900F900F90F3CE80913F0910923F098D
:10722000882311F30E94E82B80919F058823E1F2C7
:1072300009CF8F929F92AF92BF92CF92DF92EF923F
:10724000FF920F931F93CF93DF9361E081E00E9441
:107250003223C091A1051C2F85E0882E8C0ED1E031
:107260009FEBC92E97E2D92E09E00C1B88E0F82E7F
:10727000FC1A87E0E82EEC1A86E0B82EBC1A85E0EE
:10728000A82EAC1A84E0982E9C1AC1112FC0DD23C1
:10729000D9F08091A0051816BCF040913B0950919F
:1072A0003C0960913D0970913E094F5F5F4F6F4F00
:1072B0007F4F40933B0950933C0960933D09709385
:1072C0003E098F5F8093A00580917502882339F075
:1072D00043E066E17CE0812F81950F949314CF5FAA
:1072E0008C12D3CF8AE080939E0523C0C13071F504
:1072F000D091A005D13089F080917502882359F092
:1073000061E0611B81E0D13009F080E024E04CEFC6
:107310005BE00F941E15D0E0E2CF80913F09109200
:107320003F09882349F30E946C2E80919F05882392
:1073300019F3DF91CF911F910F91FF90EF90DF90A4
:10734000CF90BF90AF909F908F900895C23009F07A
:1073500029C18091A0058230B9F0809175028823FF
:10736000D1F28BE497E29F938F9389EC9BE09F93FC
:107370008F9382E0811B8F9381E09091A0059230E2
:1073800009F42EC180E02CC180913F0910923F0981
:10739000882319F30E944B2780919F058823E9F2E7
:1073A000C8CF80913F0910923F09882309F402C198
:1073B0000E945E2780919F05882309F4FBC0B9CF06
:1073C000C43029F58091A0058430A1F08091750228
:1073D000882309F4A0CF81E797E29F938F938EEBE8
:1073E0009BE09F938F939F9281E09091A0059430B2
:1073F00049F6F6C080913F0910923F09882331F386
:107400000E94712780919F05882301F392CFC53098
:1074100031F58091A0058530A9F08091750288230F
:1074200009F479CF85E897E29F938F9387EB9BE0F0
:107430009F938F93AF9281E09091A005953009F0D2
:10744000A1CFCEC080913F0910923F09882329F334
:107450000E94852780919F058823F9F26ACFC63064
:1074600051F58091A0058630A9F08091750288239E
:1074700009F451CF85EF9BEC9F938F9381EB9BE0B9
:107480009F938F93BF9281E09091A005963009F071
:1074900079CFA6C080913F0910923F09882329F334
:1074A00085EF9BEC892B11F00E94F5CB80919F0515
:1074B0008823D9F23ECFC73031F58091A0058730BF
:1074C000A9F080917502882309F425CF89E997E214
:1074D0009F938F938CEA9BE09F938F93EF9281E031
:1074E0009091A005973009F04DCF7AC080913F0967
:1074F00010923F09882329F30E94992780919F05C4
:107500008823F9F216CFC83031F58091A005883074
:10751000A9F080917502882309F4FDCE8CEA97E2E8
:107520009F938F9385EA9BE09F938F93FF9281E0D7
:107530009091A005983009F025CF52C080913F0965
:1075400010923F09882329F30E94AC2780919F0560
:107550008823F9F2EECEC93009F0C1CE8091A005A2
:10756000893099F080917502882309F4D4CEDF9296
:10757000CF928EE99BE09F938F930F9381E0909140
:10758000A005993009F0FECE2BC080913F091092E2
:107590003F09882339F30E94BF2780919F058823E4
:1075A00009F3C7CEC33009F00BCF8091A00583301B
:1075B00009F4F7CE80917502882309F4ACCE8EE5EC
:1075C00097E29F938F9385EC9BE09F938F9383E04B
:1075D000811B8F9381E09091A005933009F0D2CE6A
:1075E0008F930E947D250F900F900F900F900F901A
:1075F0000F9091CECF93DF93CDB7DEB78E81282F3A
:10760000082E000C330B909144129217130609F0C8
:107610008CF4809344129E01275F3F4F4F81588521
:107620006AE270E089E192E10F94783910921812C1
:1076300010921712DF91CF9108950F931F93CF935C
:10764000DF938C016F3F19F41092441260E0209197
:107650004412862F062E000C990B2817190609F0E4
:1076600014F560934412C8010F94FE38800F911FE7
:10767000EC01C01BD10BCB32D1053CF00197FC01D2
:107680002491207C2038D1F3F3CFDD27AE01B8015F
:1076900089E192E10F941F39C75EDD4E1882109286
:1076A000181210921712DF91CF911F910F91089528
:1076B000CF9380914205811109C087E597E09093AF
:1076C00091058093900581E0809342050E945324A8
:1076D00020E040E070E060E08FE396E20E949323B8
:1076E000C1E0C09340090E947F8F109240090E9420
:1076F0006C2EC093400960E081E79CE30E941D3B33
:107700004091510961E080E00E94092E8DE497E0EC
:107710009093F3088093F208CF9108952F923F92AF
:107720004F925F926F927F928F929F92AF92BF9291
:10773000CF92DF92EF92FF920F931F93CF93DF933D
:1077400000D000D01F92CDB7DEB780919A06412CB1
:10775000811103C00E944FCD482E8091A21784FB57
:10776000222720F92983312C84FF03C00E9473CD86
:10777000382E61E081E00E9432238091A1058E8342
:10778000582E8B5F8A8380E00EEA1CE091E0792E10
:107790007518952D91959B8398E5E92E9BE3F92E1D
:1077A0002BECC22E2CE0D22E92E095199C8393E014
:1077B00095199D833BE4A32E3CE0B32E42E7842E33
:1077C0004CE0942E9A812E81921709F463C22223F1
:1077D00039F1411079C00E9481CD882309F4B2C1EA
:1077E0008E81813009F47DC192E09F832E818F814B
:1077F000281398C12090A005221609F4A5C18091F4
:107800007502882309F48EC16E81651981E09E811D
:10781000291280E023E047EA5CE00F941E1582C144
:107820006090A005662059F180917502882389F245
:1078300081E0611080E024E047ED5CE06B810F9413
:107840001E15442041F224E02F838F819E818913ED
:107850005EC02090A005281609F487C180917502AA
:10786000882309F454C06E81651981E02E812212AB
:1078700080E023E04BE95CE00F941E1548C0809146
:107880003F0910923F09882379F20E946C2E809163
:107890009F05882349F227960FB6F894DEBF0FBEE6
:1078A000CDBFDF91CF911F910F91FF90EF90DF90AF
:1078B000CF90BF90AF909F908F907F906F905F9090
:1078C0004F903F902F9008958E81813009F4A8C089
:1078D000823009F4D0C09E81933009F0B4CF8091FA
:1078E000A0058F83833009F4EBC080917502882353
:1078F00009F4A9CF81E09F81933009F080E023E073
:107900004BEB5CE06D810F941E1524E02F838F817B
:107910008F5F9E81891314C02090A005291609F459
:1079200035C180917502882359F06E81651981E017
:107930002E81221280E023E04DE85CE00F941E15BA
:107940008F818E5F9E81891314C02090A005291617
:1079500009F42DC180917502882359F06E81651953
:1079600081E02E81221280E023E04DE75CE00F945D
:107970001E158F818D5F9E81891314C02090A005F4
:10798000291609F425C180917502882359F06E816A
:10799000651981E02E81221280E023E046E75CE059
:1079A0000F941E158F818C5F9981992309F444C12E
:1079B000311032C02E81821314C09091A00592170D
:1079C00009F417C180917502882359F06E816519F9
:1079D00081E02E81921380E020E245E65CE00F9486
:1079E0001E158F818B5F9E81891314C02090A00586
:1079F000291609F410C180917502882359F06E810F
:107A0000651981E02E81221280E023E044E55CE0EC
:107A10000F941E158F818A5F9E819F5F9E83D2CEB9
:107A20008091A0058130D1F080917502882309F4FE
:107A30000ACFFF92EF92DF92CF927F9281E09091F6
:107A4000A005913009F080E08F930E947D250F9072
:107A50000F900F900F900F900F90F5CE80913F09EF
:107A600010923F09882301F30E94583B80919F05A3
:107A70008823D1F210CF2091A0052F83223089F0E6
:107A800080917502882309F4DECE81E09F819230D7
:107A900009F080E023E040EC5CE06C810F941E155F
:107AA000D2CE80913F0910923F09882349F38FEA93
:107AB00096E20E947D2480919F05882309F3EBCEF6
:107AC00080913F0910923F09882309F40ECF8AEF75
:107AD00098E40E947D2480919F05882309F405CFB6
:107AE000DACE8091A005813001F180917502882362
:107AF00009F47ACE8EE297E29F938F931F930F93B0
:107B00007F9281E09091A005913009F080E08F9301
:107B10000E947D250F900F900F900F900F900F9067
:107B200082E08F832F812F5F8FCE80913F0910924B
:107B30003F098823D1F20E942E2780919F05882338
:107B4000A1F2A9CE91E051CE80913F0910923F0958
:107B5000882309F454CE82EA90E30E947D24809128
:107B60009F05882309F44BCE96CE80913F09109251
:107B70003F09882309F472CE8FE19EE40E947D24A0
:107B800080919F05882309F469CE85CE80913F09B5
:107B900010923F09882309F4C4CE86E195E30E9440
:107BA0007D2480919F05882309F4BBCE74CE8091FB
:107BB0003F0910923F09882309F4CCCE8BE097E36C
:107BC0000E947D2480919F05882309F4C3CE63CE53
:107BD00080913F0910923F09882309F4D4CE84E2B2
:107BE00091E50E947D2480919F05882309F4CBCEE6
:107BF00052CE80913F0910923F09882309F4E2CECA
:107C00009092F3088092F20880919F05882309F4EE
:107C1000D9CE8E8101CF80913F0910923F098823F0
:107C200009F4E9CE83EF9DE60E947D2480919F05B3
:107C3000882309F4E0CEEDCF9E8189131DC0909179
:107C4000A0052E819217D9F0809175028823A1F0AA
:107C50001F921F92BF92AF928E8185198F9381E000
:107C60002E81921380E08F930E947D250F900F90BC
:107C70000F900F900F900F908F818B5FCDCE8091E2
:107C80003F0910923F098823F9F280919F058823CC
:107C9000D9F2BFCF80939E05FECD10924F0910926E
:107CA00074020E9473CD9091A21780FB97F9909374
:107CB000A21760E08FE397E00E941D3B0C945E2DBD
:107CC0000F931F930F941E1D00913E0510913F05C9
:107CD0002091400530914105601B710B820B930B85
:107CE00097FD0BC086B18295817091E08927369B04
:107CF0008260329B84608093FF038091FF038170D8
:107D00009091FF0391FD826090913D05981749F095
:107D1000813029F148F0823089F08330A1F08093DE
:107D20003D051F910F910895913089F09230B9F778
:107D300090913C0520911B02921B0EC0992339F0B3
:107D40009330B1F3ECCF913099F3923041F79091A9
:107D50003C0520911B02920F90933C05E0CF9923A4
:107D600039F39330E1F6F3CFFC0180E0309749F02E
:107D70009491992331F0907C903809F08F5F31967F
:107D8000F7CF0895AF92BF92CF92DF92EF92FF921A
:107D90000F931F93CF93DF93EC015B018A01FB01EB
:107DA000199587FD16C0C82ED12CF12CE12C2196F7
:107DB000F801C082D182E282F382CE01DF91CF91BD
:107DC0001F910F91FF90EF90DF90CF90BF90AF90F9
:107DD0000895982F907E903CA9F48F7190E0B0E0C8
:107DE000A0E06C017D0156E0CC0CDD1CEE1CFF1CFC
:107DF0005A95D1F7CE010196F50119958F73C82ACE
:107E00002296D6CF982F907F903E11F58F7090E0FC
:107E1000B0E0A0E06C017D0136E0CC0CDD1CEE1C76
:107E2000FF1C3A95D1F7CE010196F50119958F7394
:107E3000C82A46E0CC0CDD1CEE1CFF1C4A95D1F78D
:107E4000CE010296F50119958F73C82A2396B0CFFB
:107E5000982F987F903F79F5877090E0B0E0A0E090
:107E60006C017D0186E0CC0CDD1CEE1CFF1C8A95AC
:107E7000D1F7CE010196F50119958F73C82A96E0C6
:107E8000CC0CDD1CEE1CFF1C9A95D1F7CE0102969E
:107E9000F50119958F73C82A26E0CC0CDD1CEE1C69
:107EA000FF1C2A95D1F7CE010396F50119958F7322
:107EB000C82A24967DCF982F907C903841F4807CFE
:107EC000803869F42196CE01F5011995F8CF8E7F9F
:107ED0008D3F28F02196CE01F5011995F8CFC12CE0
:107EE000D12C760165CF9CE0899F802D112491E0F3
:107EF000980F909304052CE0280F2093460930E05A
:107F00002E5F3F4F40917D164217130619F014F073
:107F100080E0089520917F169217D0F7662341F0F4
:107F20008E5F0F947423809146098E5F0F947423A3
:107F30008091460990917D16891750F320917F1604
:107F400090910405291720F31092801680938116D2
:107F500081E0089520910205022E000C330B821758
:107F6000130641F0809302056CEE7EE089E496E111
:107F70000D94192508951F93CF93DF931F92CDB7CA
:107F8000DEB710912E0280918216811105C081E02A
:107F9000809382160F94492260914B1670914C1673
:107FA00019839E012F5F3F4F4FE089E496E10F94C4
:107FB00045220F90DF91CF911F910895CF9380912B
:107FC000030581114FC010928016109281161092F5
:107FD000821610924E1610924D1610925016109254
:107FE0004F161092521681E08093511682E28093D0
:107FF00053161092581610925716ECE6F6E12AE73F
:1080000036E18FEF81932E173F07E1F7C1E0C09370
:10801000691622E132E030935F1620935E16C0931A
:108020006016109261161092621690E49093631697
:10803000109264162AE231E030937B1620937A1670
:1080400028E032E030934C1620934B1691E1909348
:108050006E1690E190936D1680936C160F944922E2
:10806000C0930305099A11988FE19EE40197F1F7F7
:1080700000C00000119A8FE19EE40197F1F700C063
:108080000000C1E0C09382160F9449228FEF8093C5
:108090002E020E94BB3FC093FA038DE096E09093BE
:1080A000880F8093870F10928A0F1092890FCF91BB
:1080B00008950E94DE3F3C98449A3E98469A3A982A
:1080C000429A0E94603E10923C050D948E10EF92F1
:1080D000FF920F931F93CF93DF93CDB7DEB72C970B
:1080E0000FB6F894DEBF0FBECDBFFC016081718179
:1080F000828193816F3F71058105910509F0C0F47C
:1081000085E496E10E940929E0914D16F0914E1602
:108110003196849190E02C960FB6F894DEBF0FBE96
:10812000CDBFDF91CF911F910F91FF90EF900895F8
:1081300010918016009181162091FA0321110FC031
:108140004DEE55E0602F812F0F94DD2590E080E00B
:10815000180F10938016009381169927DCCFE090BA
:108160004D16F0904E1629E436E13A832983212FEB
:1081700030E03C832B83202F30E03E832D83188614
:108180001F822FEF3FEF3A8729871C861B8627EA3D
:1081900038E2AE014F5F5F4FBF01C7010F948B0FF5
:1081A000B70189E496E10F9419258F819885D0CF86
:1081B0004F925F926F927F928F929F92BF92CF92D7
:1081C000DF92EF92FF920F931F93CF93DF9300D034
:1081D00000D01F921F92CDB7DEB77C016A01490122
:1081E000FB0190818CE0989F800D1124982FF7015E
:1081F0002081822F880F820F880F809380169093A2
:1082000081164115510579F1FA82E9827C836B83ED
:10821000011122C0AE014B5F5F4FB401C6010E9445
:10822000C23E6C018D819E81AF81B885892B8A2BDE
:108230008B2BC9F0CE0105960E946740F701808123
:108240008F5F8083853130F3CE0101960E948B24AD
:10825000E1CFB12C860129C08A01B12C26C0452866
:1082600046284728B1F728960FB6F894DEBF0FBE10
:10827000CDBFDF91CF911F910F91FF90EF90DF90D5
:10828000CF90BF909F908F907F906F905F904F9016
:108290000895B39407C0B1102EC001151105C9F29D
:1082A0000F5F1F4F01151105A9F2AE014B5F5F4F24
:1082B000B401C6010E94C23E6C014D805E806F8099
:1082C00078844114510461047104A9F0F0E24F165E
:1082D000510461047104F9F2D301C2018D97A1091F
:1082E000B1090297A105B10530F04BE244165104E3
:1082F0006104710471F6F7018081482F4B0D5527F9
:10830000551F4631510534F0853020F0CE010196DD
:108310000E948B2481E0411451046104710409F42A
:1083200080E0B80EF70180818B0D8083BB2009F4BB
:1083300096CFBA94AE014B5F5F4FB401C8010E9463
:10834000C23E8C01CE0105960E946740EFCF6F922E
:108350007F928F929F92AF92BF92CF92DF92EF92D5
:10836000FF920F931F93CF93DF9300D000D01F9203
:108370001F92CDB7DEB77C01162F5A014901862F17
:10838000660F990B9C0124563D4F690186E0682ECB
:10839000712C10160CF046C0AE014B5F5F4F61EAC6
:1083A00074E2C7010E94C23E7C018D819E81AF8133
:1083B000B8850097A105B105A9F18D339105A105F7
:1083C000B10509F480C08E379105A105B10509F406
:1083D0007AC08A329105A105B105D1F517FF12C007
:1083E00083E596E01E3F11F08FE496E036E003024D
:1083F000B00111240E947FC766E070E00F944841ED
:10840000061B9BC085E490E0A0E0B0E089839A83DE
:10841000AB83BC83CE0101960E946740015009F0F6
:1084200054C000E0802F28960FB6F894DEBF0FBE30
:10843000CDBFDF91CF911F910F91FF90EF90DF9013
:10844000CF90BF90AF909F908F907F906F90089546
:1084500084329105A105B105D1F48114910461F034
:10846000E6E00E02B0011124C4010E947FC7B301EF
:108470000F944841061B8DCFA114B104F1F0F6E032
:108480000F02B0011124C5010E94DDC7F0CF803476
:108490009105A105B10589F40150F6018081082EEE
:1084A000000C990BAA0BBB0B89839A83AB83BC830B
:1084B000CE0101960E9467406CCFCE0105960E94C6
:1084C0006740015066CF17FD8BCF81E04D815E8103
:1084D0006F8178854D3351056105710509F480E0A0
:1084E000810F8A30CCF001506AE00F942641D92EDA
:1084F000082E000C990BC096092E000CAA0BBB0B82
:1085000089839A83AB83BC83CE0101960E94674026
:10851000002309F486CF8D2D082E000C990BC096F0
:10852000092E000CAA0BBB0B89839A83AB83BC83F7
:10853000CE0101960E9467400150002309F471CFDB
:1085400086E00802B0011124C7010E947FC766E0DF
:1085500070E00F944841061B65CF6FEF7FEF0C94DE
:10856000DDC72F923F924F925F926F927F928F92D0
:108570009F92AF92BF92CF92DF92EF92FF920F93B2
:108580001F93CF93DF9300D000D01F92CDB7DEB7FB
:108590004C010F94FE3801966401C80ED91EC60125
:1085A0000F94FE3801961601280E391ED601EC9064
:1085B00001E0E11001C000E0F101408077247394F4
:1085C000411001C0712C11E0E11010E060E085E085
:1085D0000E9432235090A105F52C9EE0A92EB12CCB
:1085E000F52DF195FF83812F90E00196080F192F4B
:1085F000111D9801270D311D3E832D83F1101BC0E5
:1086000080917502882391F0E0911A02E2506AE4A9
:108610007AE0E33038F4F0E0EE0FFF1FE654FD4F50
:108620006081718143E08F810F94931401E0E11028
:1086300011C002E00FC002E0E11001E00F110AC01A
:1086400080917502882331F041E0B401802F8519B3
:108650000F94931411E0100F7F2C7518EE2069F021
:108660001F1109C080917502882329F041E0B601ED
:10867000872D0F94931412E0100F442061F01F1106
:1086800009C080917502882329F041E0B101872D4E
:108690000F9493141F5F4D815E81433051050CF49C
:1086A0001F5F1F1190C080917502882309F488C054
:1086B00042E067E57AE0872D0F9493149EEF9A0DC0
:1086C00080917D168A151B0411F00CF079C0209161
:1086D0007F1683EF8A0D821708F072C000910004A4
:1086E00025E430E040E050E029833A834B835C830B
:1086F0003EE33093801690938116CE0101960E943E
:10870000674081E3800F082E000C990BAA0BBB0B6E
:1087100089839A83AB83BC83CE0101960E94674014
:1087200080E290E0A0E0B0E089839A83AB83BC83D1
:10873000CE0101960E946740602E712C97E1969DB4
:10874000F001979DF00D1124E15CF94F20E030E03D
:1087500040E05FE364817581868197810F94083ED4
:108760000F94743FCB010E9492BD0E94AD422FE254
:1087700030E040E050E029833A834B835C83CE01B4
:1087800001960E9467400E94F22481110BC035E0DF
:10879000369DF001379DF00D1124E25EF94F848182
:1087A00081110EC047E1469DF001479DF00D112457
:1087B000E15CF94F808591850E9492BD0E94AD4297
:1087C00052E0509375028CE0A80EB11CF3949AE429
:1087D000A916B10409F012CF1F5F10939E052796CA
:1087E0000FB6F894DEBF0FBECDBFDF91CF911F91C2
:1087F0000F91FF90EF90DF90CF90BF90AF909F9040
:108800008F907F906F905F904F903F902F90089542
:1088100082E69AE00C94B1428FE69AE00C94B14261
:1088200081E99AE00C94B1428CE29BE00C94B14255
:1088300087EE9AE00C94B14284E19BE00C94B14243
:1088400087E69BE00C94B1428AE49BE00C94B14231
:108850008AEC9AE00C94B1428BEA9AE00C94B14213
:108860008F929F92AF92BF92CF92DF92EF92FF9240
:108870000F931F93CF93DF9300D01F92CDB7DEB736
:108880004C016B0181E080931B02C4010E94B43E45
:10889000A82EC6010E94A724B12C23E130E0790163
:1088A000E81AF10815E2EA14FB040CF41FE1812F29
:1088B00090E09C012E5F3F4F40917D1642171306BA
:1088C00011F00CF04AC0099720917F16281719065D
:1088D0000CF443C020914A0930914B09409148095A
:1088E00050914909609147091092801610938116A2
:1088F00005E1C4010E94A74101E0C114D104E1F0E7
:108900008AE390E0A0E0B0E089839A83AB83BC83E4
:10891000CE0101960E946740EA14FB0404F5145F3F
:1089200080917D16181740F020917F16412F4950F5
:10893000550B24171506ACF40F900F900F900F9065
:10894000DF91CF911F910F91FF90EF90DF90CF902B
:10895000BF90AF909F908F90089500E0CECF0023FE
:1089600059F380E290E0A0E0B0E089839A83AB8382
:10897000BC838E2D880FE80EEE0CE09280161093CB
:108980008116CE0101960E946740C6010E94AD4249
:10899000D3CF1F93CF93DF9300D01F92CDB7DEB715
:1089A000182F80913F0910923F09882361F010929F
:1089B00040090E946C2E0F900F900F900F90DF9146
:1089C000CF911F91089560913B0970913C0980916E
:1089D0003D0990913E09611571058105910569F187
:1089E0000F94B83920911C0230911D0240911E0253
:1089F00050911F020F94173A209182023091830206
:108A000040918402509185020F94083E6093820247
:108A1000709383028093840290938502612F83E098
:108A20000E94B82481E08093750210923B09109255
:108A30003C0910923D0910923E09809175028823ED
:108A400009F4B9CF1093470910924B0910924A09C3
:108A50001092490910924809209198053091990582
:108A600040919A0550919B0560918202709183021A
:108A700080918402909185020F94073E69837A83E6
:108A80008B839C83CE0101960E9497BCBC018AE631
:108A90009DE00E9430448FCF81E00C94C94480E077
:108AA0000C94C944809151090C94C9443F924F924F
:108AB0005F926F927F928F929F92AF92BF92CF926E
:108AC000DF92EF92FF920F931F93CF93DF9300D02B
:108AD00000D000D01F92CDB7DEB7382E80913F096D
:108AE00010923F098823E1F0109240090E946C2EF9
:108AF0002A960FB6F894DEBF0FBECDBFDF91CF919F
:108B00001F910F91FF90EF90DF90CF90BF90AF90AB
:108B10009F908F907F906F905F904F903F900895BF
:108B200060913B0970913C0980913D0990913E090B
:108B3000611571058105910509F459C0209137022D
:108B4000222309F4B9C0209138022111B5C021E0D7
:108B5000321609F48FC0A2E03A1609F49CC0C09006
:108B60003902D0903A02E0903B02F0903C024090F3
:108B700045025090460260904702709048020F9460
:108B8000B83920911C0230911D0240911E02509173
:108B90001F020F94173A6F83788789879A87B4E00A
:108BA0003B9E80011124F801EA58FD4FFE83ED83BE
:108BB00020813181428153810F94083E4B015C0139
:108BC000A3019201C701B6010F94B139811183C08D
:108BD000F801EA58FD4F80829182A282B3826091AF
:108BE0005109832D0E94B82481E080937502109270
:108BF0003B0910923C0910923D0910923E09809168
:108C00007502882309F474CF30924709F4E03F9E3F
:108C1000C0011124FC01EA58FD4F8359904FDC013B
:108C20002D913D914D915C91608171818281938103
:108C30000F94083E6B017C01C982DA82EB82FC82D0
:108C40002DEC3CEC4CEC5DE360911C0270911D023C
:108C500080911E0290911F020F94684087FD66C0AC
:108C6000CE0101960E9497BCBC018FE79DE00E9457
:108C700030443ECFC0903D02D0903E02E0903F0293
:108C8000F09040024090490250904A0260904B029E
:108C900070904C0274CFC0904102D0904202E0909C
:108CA0004302F090440240904D0250904E0260907A
:108CB0004F027090500263CF412C20E5522E23ECDE
:108CC000622E27E4722EC12C30E5D32E33ECE32E36
:108CD00037ECF32E54CF20E030E0A9016F81788586
:108CE00089859A850F94B13987FF10C0A701960135
:108CF000C501B4010F94B13987FF6ACFAD81BE8140
:108D0000CD92DD92ED92FC92139769CFA30192016F
:108D1000C501B4010F94684018160CF059CFED81CD
:108D2000FE81408251826282738259CF20E030E01E
:108D300040E251E4C701B6010F94173A20E030E059
:108D40004AE754E40F94173A4B015C0120E030E00D
:108D5000A901C701B6010F94B13920E030E040EA23
:108D600050E487FF04C020E030E040EA50ECC50149
:108D7000B4010F94083E20E030E040E251E40F944B
:108D8000023F0F94743F6B017C01F7FC62C020EA44
:108D900036E841E050E00F94C63DCA01B9012AE02F
:108DA00030E040E050E00F94C63D605D6093A20566
:108DB000C701B60120E137E240E050E00F94C63D24
:108DC0008AE0882E912CA12CB12CCA01B901A501F1
:108DD00094010F94C63D605D6093A305C701B60181
:108DE00028EE33E040E050E00F94C63DCA01B901DF
:108DF000A50194010F94C63D605D6093A4058EE2C9
:108E00008093A505C701B60124E630E040E050E0BC
:108E10000F94C63DCA01B901A50194010F94C63D46
:108E2000605D6093A605C701B601A50194010F948A
:108E3000C63D162FCA01B901A50194010F94C63D84
:108E4000605D6093A705105D1093A80582EA95E028
:108E50000BCFF094E094D094C094C11CD11CE11CC1
:108E6000F11C6DE2A3CF82E00C94564581E00C9496
:108E7000564580E00C9456450F931F93CF93DF9394
:108E8000FC01EB0180913B0990913C09A0913D09C7
:108E9000B0913E09B7FF08C010923B0910923C09FF
:108EA00010923D0910923E098091830590918405AE
:108EB000A0918505B091860540913B0950913C09F0
:108EC00060913D0970913E0984179507A607B70781
:108ED00044F480933B0990933C09A0933D09B093DF
:108EE0003E09809175028823E1F060913B09709101
:108EF0003C0980913D0990913E09009187051091B0
:108F000088052091890530918A05600F711F821FA5
:108F1000931F1995BC0180918D0590918E050E943B
:108F2000304480913F09811108C0809180058823D9
:108F3000D1F1809175028823B1F180918B059091D8
:108F40008C050097B1F040913B0950913C0960912C
:108F50003D0970913E090091870510918805209187
:108F6000890530918A05400F511F621F731FFE0152
:108F70001995E0918105F0918205309741F080913B
:108F80008005811103C080913F098111199580915D
:108F90003F0910923F09882331F0DF91CF911F9153
:108FA0000F910C946C2EDF91CF911F910F9108952A
:108FB00062EF7EE18FE895E20C943C4760E57FE14B
:108FC00084E497E20C943C4760EB70E28AE695E219
:108FD0000C943C4767ED70E28AE295E20C943C47C2
:108FE00068EE72E28CEF92E20C943C4762E972E226
:108FF00086EA92E20C943C4760EB72E28BEE97E2D9
:109000000C943C4766EC72E288E298E20C943C4790
:109010006AED72E282E398E20C943C4766E073E208
:1090200083E695E20C943C4769EC70E28EE698E2A8
:109030000C943C4764E173E288E293E20C943C4771
:109040004F925F926F927F928F929F92AF92BF9258
:10905000CF92DF92EF92FF920F931F93CF93DF9304
:10906000CDB7DEB72C970FB6F894DEBF0FBECDBFDD
:10907000982F862F5A017901D02E692F0E94733FB5
:10908000882309F49CC01091FA03C701002309F456
:1090900041C00E94B43EC82E80904D1690904E164E
:1090A000111155C01FEF03E10C1920914A093091AD
:1090B0004B09409148095091490960914709C50100
:1090C0000E94A741CC2009F47AC0B6E08B9F5001E2
:1090D00011248AE390E0A0E0B0E089839A83AB8317
:1090E000BC83CE0101960E94674080E2482E512C3D
:1090F000612C712C57E0A516B10408F445C04982D3
:109100005A826B827C82CE0101960E946740A81A27
:10911000B90AF0CF0E94A724C82E80904D169090D7
:109120004E16112309F4BECFFE0133968AE0DF010B
:109130001D928A95E9F789E496E19A8389830EE77F
:1091400018E29E012F5F3F4F44EA54E212C0FE0135
:1091500033968AE0DF011D928A95E9F789E496E16A
:109160009A8389830EE718E29E012F5F3F4F41EA01
:1091700054E2B701C4010F945010B40189E496E1A0
:109180000F9419251F818FCF40914609212F30E080
:10919000A6E0CA9EC00111242E5F3F4F2817390751
:1091A0000CF49C0180E8821B80938016409381160A
:1091B000DD20E1F06FEF7FEFC7010E947FC72C96A3
:1091C0000FB6F894DEBF0FBECDBFDF91CF911F91D8
:1091D0000F91FF90EF90DF90CF90BF90AF909F9056
:1091E0008F907F906F905F904F900895C7010E947D
:1091F000AD42E5CF6F927F928F929F92AF92BF92D6
:10920000CF92DF92EF92FF920F931F93CF93DF9352
:1092100061E081E00E943223C091A105DC2FF5E0DE
:10922000AF2EAC0E81E0D82EDC1A9C2E9194A7E1D3
:10923000BA2E8824839484E0C82ECC1AC11142C16E
:109240001091A005112309F420C180917502882393
:1092500049F081E0111180E024E047EE5EE0692DE5
:109260000F941E15F12CE12CE2E07E2E6C2E6D1A6F
:10927000C7112BC0E092470910924B0910924A097E
:1092800010924909109248098091A0058C1709F4A1
:1092900051C1809175028823C1F011E08091A00531
:1092A000871110E0BE9CF001BF9CF00D1124E15C21
:1092B000F94F808591850E9492BD00E09C0148EDA8
:1092C0005EE0662D812F0E942048872D9FEFE91ACE
:1092D000F90A63E0762E833059F6C430E9F48091C0
:1092E000A005843009F44DC1809175028823A1F056
:1092F00011E08091A005843009F010E080913606DD
:10930000909137060E9492BD00E09C0144ED5EE022
:109310006C2D812F0E9420488091D20580933609C0
:10932000C53031F51092470910924B0910924A0945
:1093300010924909109248098091A005853009F4DE
:109340003BC180917502882399F0FC2EFD1A11E033
:109350008091A0058C1310E0809136090E942ABEEE
:1093600000E09C0148EC5EE06F2D812F0E942048B8
:109370008091D30580933609C63031F58092470934
:1093800010924B0910924A0910924909109248090B
:109390008091A005863009F424C18091750288234C
:1093A00099F0FC2EFD1A11E08091A0058C1310E0BD
:1093B000809136090E942ABE00E09C0148EC5EE0E4
:1093C0006F2D812F0E942048C73019F58091A0058C
:1093D000873009F41BC1809175028823D1F0FC2EDF
:1093E000FD1A11E08091A0058C1310E0E091510965
:1093F000F0E0EE0FFF1FEE5DFD4F808191810E9436
:1094000092BD00E09C0143EC5EE06F2D812F0E9435
:10941000204838E0732EF12CE12C6C2E6D1AC71108
:1094200029C0E092470910924B0910924A09109204
:109430004909109248098091A0058C1709F408C1C8
:10944000809175028823B1F011E08091A005871109
:1094500010E0F701EE0FFF1FEE5DFD4F808191815F
:109460000E9492BD00E09C014CEB5EE0662D812FD6
:109470000E9420487394EA94EF2809F0E5C0CF5F7A
:10948000AC12DCCE70929E050EC080913F09109206
:109490003F09882309F4D9CE0E946C2E80919F0544
:1094A000882309F4D2CEDF91CF911F910F91FF90C5
:1094B000EF90DF90CF90BF90AF909F908F907F9074
:1094C0006F900895C13009F0CDCE8091A005813014
:1094D000D1F080917502882309F4C4CE11E0809107
:1094E000A005813009F010E08091200290912102C6
:1094F0000E9492BD00E09C0141EE5EE06D2D812F47
:109500000E942048AFCE80913F0910923F098823E6
:1095100001F310E000E027EE33E04AE050E060E2C3
:1095200072E081EE9EE00F94CC1680919F05882317
:1095300081F2B9CF80913F0910923F09882309F445
:10954000A8CE0F94BF15F701EE0FFF1FE054FD4F9B
:10955000208131812F503109BE9CB001BF9C700D1C
:109560001124695B794F0BE815E250E040E088ED8B
:109570009EE00F94CC1680919F05882309F489CE34
:1095800092CF80913F0910923F09882309F4ACCE15
:109590000F94BF1502E216EC24E630E050E040E004
:1095A00066E376E084ED9EE00F94CC1680919F05F3
:1095B000882309F499CE77CF80913F0910923F0913
:1095C000882309F4BECE0F94BF1566E07FE188ECD6
:1095D0009EE00F94A41780919F05882309F4B1CED3
:1095E00062CF80913F0910923F09882309F4D5CEBC
:1095F0000F94BF1566E07FE188EC9EE00F94A417FE
:1096000080919F05882309F4C8CE4DCF80913F09F2
:1096100010923F09882309F4DECE6091510970E071
:10962000660F771F6E5D7D4F0EEB1EE127EE33E078
:109630004AE050E083EC9EE00F94CC1680919F05A9
:10964000882309F4C8CE2FCFEE24E394F12CE7CE83
:1096500080913F0910923F09882309F4F1CEB701A8
:10966000660F771F6E5D7D4F0AE81EE127EE33E03F
:109670004AE050E08CEB9EE00F94CC1680919F0561
:10968000882309F4DDCE0FCFAF92BF92CF92DF9245
:10969000EF92FF920F931F93CF93DF9361E081E0EE
:1096A0000E943223C091A10585E0B82EBC0ED5E002
:1096B000DC1B14E01C1B83E0F82EFC1A82E0E82E71
:1096C000EC1A81E0D82EDC1AAC2EA194C1112FC067
:1096D000C090A005CC20A1F080917502882349F0AC
:1096E00081E0C11080E024E04DE65EE06A2D0F9439
:1096F0001E15CF5FCB11EACF86E080939E050CC08C
:1097000080913F0910923F09882331F30E946C2E0B
:1097100080919F05882301F3DF91CF911F910F91D5
:10972000FF90EF90DF90CF90BF90AF900895C13041
:1097300089F58091A0058130D1F080917502882350
:10974000C1F2CC24C3948091A005813009F0C12CD2
:109750008091E8159091E9150E94C7BD00E09C0139
:1097600048E55EE06D2D8C2D0E942048C2CF80918F
:109770003F0910923F09882301F346E756E268EE5D
:1097800075E188E59EE00F94141880919F05882369
:10979000A1F2C2CFC23009F0A0C08091A0058230F2
:1097A000C1F080917502882309F4A3CFCC24C3941F
:1097B0008091A005823009F0C12C8091AC15909168
:1097C000AD150E94C7BD00E09C0146E55EE06E2D30
:1097D000CACF80913F0910923F09882311F34EE6CA
:1097E00056E26CEA75E186E59EE00F9414188091CC
:1097F0009F058823B1F290CF8091A0058330C1F0FE
:1098000080917502882309F474CFCC24C39480918D
:10981000A005833009F0C12C8091701590917115CD
:109820000E94C7BD00E09C0144E55EE06F2D9BCF28
:1098300080913F0910923F09882311F346E656E2D2
:1098400060E775E184E59EE00F94141880919F0510
:109850008823B1F261CF8091A0058430C1F080915E
:109860007502882309F445CFCC24C3948091A005C8
:10987000843009F0C12C80913415909135150E94E7
:10988000C7BD00E09C0141E55EE0612F6CCF809197
:109890003F0910923F09882311F34EE556E264E335
:1098A00075E181E59EE00F94141880919F0588234F
:1098B000B1F232CF80913F0910923F098823D1F055
:1098C00046E556E268EF74E18EE49EE00F941418CA
:1098D00080919F05882371F01FCFC33009F48CCF8E
:1098E000C43009F4B8CFC53009F003CF8091A0058A
:1098F000853001F380917502882309F4FACECC24D7
:10990000C3948091A005853009F0C12C8091F81492
:109910009091F9140E94C7BD00E09C014EE45EE006
:109920006D2F21CF7F928F929F92AF92BF92CF9255
:10993000DF92EF92FF920F931F93CF93DF9361E03B
:1099400081E00E943223C091A1059C2E85E0A82EC3
:10995000AC0ED1E011E093E0F92E86E0E82EEC1A8F
:1099600085E0D82EDC1A84E0C82ECC1A8F2C8C1AF5
:1099700082E0B82EBC1A7D2E7C1AC1112FC0DD23C7
:10998000D9F08091A0051816BCF040913B09509188
:109990003C0960913D0970913E094F5F5F4F6F4FE9
:1099A0007F4F40933B0950933C0960933D0970936E
:1099B0003E098F5F8093A00580917502882339F05E
:1099C00041E069E77EE0892D81950F949314CF5F84
:1099D000AC12D3CF87E080939E0522C0C13071F5D1
:1099E000D091A005D13081F080917502882351F08B
:1099F00081E0D13009F080E024E04DE65EE0672DA3
:109A00000F941E15D0E0E3CF80913F0910923F09DB
:109A1000882351F30E946C2E80919F05882321F3A7
:109A2000DF91CF911F910F91FF90EF90DF90CF903A
:109A3000BF90AF909F908F907F900895C23009F0B3
:109A4000DEC08091A0058230C9F080917502882324
:109A5000C9F281E09091A005923009F080E09091E8
:109A6000EA1528E63EE0911102C024E63EE001E05E
:109A70004BE65EE06B2D0E942048C4CF80913F09E9
:109A800010923F09882309F38091EA15812780937A
:109A9000EA15F09275020E94542680919F05882352
:109AA000A1F2BECF80913F0910923F09882309F4AB
:109AB000AEC08091AE1581278093AE15C09375021C
:109AC0000E94522680919F05882309F4A0C0A8CF48
:109AD000C43081F58091A0058430C1F08091750279
:109AE000882309F48FCF81E09091A005943009F08C
:109AF00080E09091721528E63EE0911102C024E6C4
:109B00003EE001E040E65EE06C2DB5CF80913F097C
:109B100010923F09882311F3809172158127809359
:109B20007215F09275020E94502680919F0588233D
:109B3000A9F276CFC53081F58091A0058530C1F0BE
:109B400080917502882309F45DCF81E09091A00592
:109B5000953009F080E09091361528E63EE09111AD
:109B600002C024E63EE001E04DE55EE06D2D83CFCE
:109B700080913F0910923F09882311F38091361597
:109B8000812780933615F09275020E944E268091AF
:109B90009F058823A9F244CFC63009F018CF8091E1
:109BA000A0058630C1F080917502882309F42ACF80
:109BB00081E09091A005963009F080E09091FA1430
:109BC00028E63EE0911102C024E63EE001E04AE5CD
:109BD0005EE06E2D50CF80913F0910923F0988239F
:109BE00011F38091FA1481278093FA14F092750290
:109BF0000E944C2680919F058823A9F211CFC33083
:109C000009F066CF8091A005833009F44BCF809195
:109C10007502882309F4F6CE81E09091A005933077
:109C200009F080E09091AE1528E63EE0911102C067
:109C300024E63EE001E042E65EE0682D1CCF2F9274
:109C40003F924F925F926F927F928F929F92AF92CC
:109C5000BF92CF92DF92EF92FF920F931F93CF9319
:109C6000DF9300D0CDB7DEB78091470690914806CC
:109C700077247394892B39F480915E0690915F0666
:109C8000892B09F4712C61E081E00E9432238091DC
:109C9000A1058A838B83982F9B5F9983382E3194FB
:109CA00083E0582EEA815E1A55E0452E66E6A62E20
:109CB0006DE2B62E7DE1872E7EE0972EFA81F111BE
:109CC00012C01091A005112309F43DC180917502C5
:109CD000882349F081E0111180E024E049E45EE04E
:109CE000632D0F941E154FE3C42E46E0D42EF12CA5
:109CF000E12C662463942A808B81281AF6018085E2
:109D000091859093370980933609FA81F61126C020
:109D1000E092470910924B0910924A0910924909A2
:109D2000109248098091A0058F1709F430C18091E5
:109D30007502882399F011E08091A005861110E04A
:109D400080913609909137090E9492BD00E09C01F4
:109D500040E45EE0622D812F0E942048862D9FEF17
:109D6000E91AF90AE7E1CE0ED11C22E0622E823018
:109D700029F6FA81F330E9F48091A005833009F4E3
:109D800028C1809175028823A1F011E08091A0057F
:109D9000833009F010E080913606909137060E94DA
:109DA00092BD00E09C014CE35EE0652D812F0E9496
:109DB00020488091D205809336098A81843041F50C
:109DC0001092470910924B0910924A0910924909C2
:109DD000109248098091A005843009F415C1809142
:109DE00075028823A9F0FA809B81F91A11E080910D
:109DF000A005EA818E1310E0809136090E942ABEE8
:109E000000E09C0140E35EE06F2D812F0E9420481E
:109E10008091D30580933609FA814F1229C081E0E1
:109E20008093470910924B0910924A0910924909F0
:109E3000109248098091A005841509F4FAC0809118
:109E400075028823A9F0FA809B81F91A11E08091AC
:109E5000A005EA818E1310E0809136090E942ABE87
:109E600000E09C0140E35EE06F2D812F0E942048BE
:109E700096E0F92E09E11EE0E12CDA80FB81DF1A81
:109E8000E09236098A818F1120C0F8018591949162
:109E90001092470990934B0980934A0910924909FF
:109EA00010924809C090A0059A81C91609F4D9C03A
:109EB00080917502882349F081E0CF1080E023E093
:109EC00046E25EE06D2D0F941E15CF2CF3940E5FCD
:109ED0001F4FE1E0EE12C2C0809136069091370626
:109EE000892B11F4772031F1FA81FF121EC01091F5
:109EF000A0051F1709F4C6C0809175028823A9F038
:109F0000BF92AF929F928F928A819B81891B8F9380
:109F100081E0EA811E1380E08F930E947D250F90DF
:109F20000F900F900F900F900F9082E0F82EFC0C86
:109F300077247394FA81FF5FFA838981F813BECE88
:109F4000F0929E050EC080913F0910923F09882330
:109F500009F4BCCE0E946C2E80919F05882309F4E1
:109F6000B5CE0F900F900F90DF91CF911F910F9171
:109F7000FF90EF90DF90CF90BF90AF909F908F9029
:109F80007F906F905F904F903F902F9008958091B9
:109F90003F0910923F09882309F4C9CE0F94BF15D9
:109FA000F701EE0FFF1FE054FD4F208131812F504C
:109FB00031090EE716E250E040E066E379E080E424
:109FC0009EE00F94CC1680919F05882309F4AFCEB4
:109FD000C8CF80913F0910923F09882309F4D1CE60
:109FE0000F94BF1502E216EC24E630E050E040E0AA
:109FF00066E376E08CE39EE00F94CC1680919F059B
:10A00000882309F4BECEADCF80913F0910923F095D
:10A01000882309F4E4CE0F94BF1566E07FE180E366
:10A020009EE00F94A41780919F05882309F4D7CE52
:10A0300098CF80913F0910923F09882309F4FFCE01
:10A040000F94BF1566E07FE180E39EE00F94A417B4
:10A0500080919F05882309F4F2CE83CFEE24E39408
:10A060000FCF80913F0910923F09882309F420CF38
:10A0700084E19FE20E947D2480919F05882309F45A
:10A0800017CF6FCF80913F0910923F09882309F4C1
:10A0900033CF0E94662D80919F05882309F42CCF31
:10A0A00060CFCF92DF92EF92FF920F931F93CF93E7
:10A0B000DF9361E081E00E943223C091A10585E039
:10A0C000D82EDC0ED3E0DC1B12E01C1B81E0F82E46
:10A0D000FC1ACC2EC194C1112DC0E090A005EE2039
:10A0E000A1F080917502882349F081E0E11080E0C1
:10A0F00024E04CEF5BE06C2D0F941E15CF5FCD116B
:10A10000EACF84E080939E050CC080913F091092B5
:10A110003F09882331F30E946C2E80919F0588238C
:10A1200001F3DF91CF911F910F91FF90EF90DF909E
:10A13000CF900895C13069F58091A0058130C1F0BC
:10A14000809175028823D1F2EE24E3948091A005DA
:10A15000813009F0E12C809183160E9408BE00E056
:10A160009C014EEE5BE06F2D8E2D0E942048C6CFE5
:10A1700080913F0910923F09882311F363E876E14B
:10A180008EEE9BE00F94E81780919F058823C1F223
:10A19000C8CFC230E1F58091A0058230B1F0809146
:10A1A0007502882309F4AACFEE24E3948091A005D8
:10A1B000823009F0E12C809184160E9408BE00E0F4
:10A1C0009C014EED5BE0612FCFCF80913F09109253
:10A1D0003F09882321F364E876E18EED9BE00F943C
:10A1E000E81780919F058823D1F29BCF80913F098A
:10A1F00010923F09882391F065E876E18FEC9BE0AF
:10A200000F94E81780919F05882341F08ACFC330CF
:10A2100009F074CF8091A005833041F380917502DD
:10A22000882309F46BCFEE24E3948091A00583305A
:10A2300009F0E12C809185160E9408BE00E09C0187
:10A240004FEC5BE06D2F90CF5F926F927F928F9279
:10A250009F92AF92BF92CF92DF92EF92FF920F93B5
:10A260001F93CF93DF9361E081E00E943223C0917E
:10A27000A1056C2E85E0782E7C0ED4E0DC1B93E0EB
:10A28000892E582C5C1A21EFE22E2BECF22E34E2B0
:10A29000C32E3CE0D32E12E01C1B4CE0A42E4CEC51
:10A2A000B42E81E0982E9C1AC11113C00091A00514
:10A2B000002329F180917502882309F4DFC0662DFF
:10A2C000619581E0011180E024E04AE35CE00F94B5
:10A2D0001E1580910B0680933609C13009F055C0D8
:10A2E0009091A005913039F180917502811138C0AB
:10A2F000CF5F7C12D9CF85E080939E050CC0809102
:10A300003F0910923F098823A9F20E946C2E809188
:10A310009F05882379F2DF91CF911F910F91FF90D4
:10A32000EF90DF90CF90BF90AF909F908F907F90F5
:10A330006F905F90089590913F0910923F09992383
:10A3400099F28C278093360980927502A114B1048A
:10A3500011F00E940CCC80919F05882329F2DBCF5D
:10A3600081E09091A005913009F080E0909136094C
:10A3700020E33CE0911102C02CE23CE001E043E329
:10A380005CE0692D0E942048B3CFC23071F5809106
:10A39000A0058230D1F080917502882309F4A8CFFE
:10A3A000FF92EF92DF92CF921F9381E09091A005F0
:10A3B000923009F080E08F930E947D250F900F90DE
:10A3C0000F900F900F900F9093CF80913F091092B4
:10A3D0003F09882301F3E114F10411F00E94F1CB4D
:10A3E00080919F058823B9F296CFC33091F50091F3
:10A3F000A005033081F080917502882309F478CF9D
:10A4000081E0033009F080E023E046E15CE0652D67
:10A410000F941E156DCF80913F0910923F0988233C
:10A4200051F389E199E30E947D2480919F0588235F
:10A4300011F371CF80913F0910923F09882381F079
:10A4400081E590E50E947D2480919F05882341F05D
:10A4500062CFC43009F04CCF0091A005043051F315
:10A4600080917502882309F443CF81E0043009F01C
:10A4700080E023E048E05CE06D2FCACF80910B06BE
:10A480008093360935CF2F923F924F925F926F9211
:10A490007F928F929F92AF92BF92CF92DF92EF9274
:10A4A000FF920F931F93CF93DF9300D000D01F92A2
:10A4B000CDB7DEB7482E662E809393056093920544
:10A4C00020914709298361E081E00E943223709046
:10A4D000A10527E1362D3202C0011124AC01495BF0
:10A4E000594F6A01572C55E0570D5A833324339442
:10A4F000832D87198D8333EDA32E3CE2B32E40EFDD
:10A50000842E49E0942EE62CF12CEE0CFF1CF70172
:10A51000E054FD4F7F01562D5203A0011124495BE9
:10A52000594F5F834E8371107FC03320D9F08091E3
:10A53000A0051816BCF040913B0950913C09609170
:10A540003D0970913E094F5F5F4F6F4F7F4F4093C2
:10A550003B0950933C0960933D0970933E098F5F1E
:10A560008093A00580917502882389F083E063EDD4
:10A5700079E0481639F094E063EC79E0491611F07F
:10A5800063EB79E043E0852D81950F94931409E105
:10A590001EE022E0222EFEEFF70DFB83272D25196A
:10A5A0002C83721018C0F801859194913B813093EF
:10A5B000470990934B0980934A09109249091092D8
:10A5C00048098091A005871509F46BC08091750238
:10A5D000811176C0312C822D0E5F1F4F93E0292E02
:10A5E0008330F9F654E0751214C060924709109256
:10A5F0004B0910924A09109249091092480980911A
:10A60000A005843009F471C08091750281118AC05F
:10A61000312C7394FA81F71186CF85E080939E05E3
:10A6200029812093470919C0E1E07E12B0CF109133
:10A63000A005113031F080917502811127C0312CB5
:10A64000A6CF80913F0910923F098823A1F30E9471
:10A650006C2E80919F05882371F327960FB6F8948E
:10A66000DEBF0FBECDBFDF91CF911F910F91FF9045
:10A67000EF90DF90CF90BF90AF909F908F907F90A2
:10A680006F905F904F903F902F90089581E0113030
:10A6900009F080E024E04AEF59E06D810F941E1527
:10A6A000CECF80913F0910923F09882309F48ECFC5
:10A6B0000E94D32C80919F05882309F487CFCDCFAA
:10A6C000BF92AF929F928F924C814F9381E0909175
:10A6D000A005921180E08F930E947D250F900F902E
:10A6E0000F900F900F900F9075CF80913F091092AF
:10A6F0003F09882309F488CF0F94BF15F701208103
:10A7000031812F5031090FED1CE24AEA50E0B601C9
:10A7100081EE99E00F94CC1680919F05882309F46F
:10A7200073CF9BCF11E08091A005843009F010E039
:10A73000EE81FF81808191810E9492BD64E0651964
:10A7400000E09C0141EE59E0812F0E94204860CF3B
:10A750006091470984E00C9443526091470983E07B
:10A760000C9443526091470982E00C9443522F921B
:10A770003F924F925F926F927F928F929F92AF9291
:10A78000BF92CF92DF92EF92FF920F931F93CF93DE
:10A79000DF9300D000D0CDB7DEB70E9462CD482E47
:10A7A00061E081E00E9432232091A1052D834420A5
:10A7B00069F185E08E837D80272D2B5F298385E0DD
:10A7C00087198A8384E087198B8383E087198C83B8
:10A7D00082E0682E671881E0582E5718272C2194A4
:10A7E0002D8121113BC01091A005112391F0809182
:10A7F0007502882309F451C081E0111180E024E042
:10A8000049ED58E0622D0F941E1547C096E09E83D7
:10A81000D2CF80913F0910923F09882341F30E94D3
:10A820006C2E80919F05882311F326960FB6F8941D
:10A83000DEBF0FBECDBFDF91CF911F910F91FF9073
:10A84000EF90DF90CF90BF90AF909F908F907F90D0
:10A850006F905F904F903F902F9008958D81813041
:10A8600009F096C01091A005113009F47CC08091C8
:10A870007502882391F01F9288EC98E09F938F9344
:10A880005F9281E0113009F080E08F930E947D2576
:10A890000F900F900F900F900F904110B1C02D812D
:10A8A000253009F0ADC01091A005153009F402C1A2
:10A8B0008091750281110FC116E081E0810F9D81A9
:10A8C000891314C03090A005391609F42CC1809169
:10A8D0007502882359F06D81671981E02D8132124C
:10A8E00080E023E04CE758E00F941E1582E0810FD2
:10A8F0009D81891314C03090A005391609F424C134
:10A9000080917502882359F06D81671981E02D814E
:10A91000321280E023E043E758E00F941E1583E0F5
:10A92000810F9D81891315C09091A0052D819217EB
:10A9300009F41BC180917502882359F06D81671954
:10A9400081E02D81921380E023E041E658E00F94EE
:10A950001E158D818F5F8D839981981341CF1C5F68
:10A9600010939E0562CF80913F0910923F09882382
:10A9700009F47DCF8CE598E09093F3088093F2087A
:10A980000E945E2D80919F05882309F470CF4DCFE2
:10A990008D81823009F012C11091A005123071F042
:10A9A00080917502882309F478CF81E0123009F094
:10A9B00080E023E047EB58E0662D25CF80913F09EA
:10A9C00010923F09882361F383E69AE50E947D2473
:10A9D00080919F05882321F328CF1091A005133083
:10A9E000F1F080917502882309F457CF81E013308C
:10A9F00009F080E023E04AEA58E06C810F941E15CC
:10AA00008E819D81891309C01091A005181709F442
:10AA10006DC08091750281117AC01E814ECF8091E8
:10AA20003F0910923F098823E1F28CE09CE50E94E7
:10AA30007D2480919F058823A1F2F7CE80913F0964
:10AA400010923F09882309F4C6C020E030E04AE7AD
:10AA500054E46091FE057091FF058091000690918D
:10AA600001060F94173A20E030E040E85FE30F94CE
:10AA7000073E0F947B3F1F92912C812C8AE1A82ED8
:10AA800088E4B82E6B011BE2E12EFF24F39400E072
:10AA900010E021E030E040E050E06EEF75E08DE93D
:10AAA00098E00E94EB2C0F9080919F05882309F479
:10AAB00092C0BBCE80913F0910923F09882309F4D0
:10AAC000F7CE84E19FE50E947D2480919F05882335
:10AAD00009F4EECEAACE81E0153009F080E023E043
:10AAE00044E958E06A810F941E15E6CE80913F0933
:10AAF00010923F09882309F48CCF8DE89EE20E94D2
:10AB00007D2480919F05882309F483CF8ECE6D81AB
:10AB1000671981E02D81121380E023E048E858E0B6
:10AB20000F941E157ACF80913F0910923F09882318
:10AB300009F4CDCE84E693E60E947D2480919F05A2
:10AB4000882309F4C4CE71CE80913F0910923F0949
:10AB5000882309F4D5CE83E790E60E947D24809176
:10AB60009F05882309F4CCCE60CE80913F091092D6
:10AB70003F09882309F4DECE0E94532420E040E000
:10AB800070E060E088EC96E226960FB6F894DEBF9F
:10AB90000FBECDBFDF91CF911F910F91FF90EF902E
:10ABA000DF90CF90BF90AF909F908F907F906F90ED
:10ABB0005F904F903F902F900C9493232D812330E2
:10ABC00009F40BCF243009F068CE3090A00594E052
:10ABD000391609F433CF80917502882309F45DCECC
:10ABE0006091FE057091FF0580910006909101062D
:10ABF0000E94E6219C0181E094E0391280E000E0AF
:10AC00004DE958E06B810E942048FACE2F923F9286
:10AC10004F925F926F927F928F929F92AF92BF926C
:10AC2000CF92DF92EF92FF920F931F93CF93DF9318
:10AC300000D0CDB7DEB761E081E00E9432232091E1
:10AC4000A1052A832B5F298384E09A81891B8B834A
:10AC500066246394B2E05B2E83E0782E791A452C4B
:10AC6000491A362C391A292E21942A8121113DC0E6
:10AC70001091A0051123B9F080917502882349F045
:10AC800081E0111180E024E041E159E0622D0F9450
:10AC90001E159A819F5F9A8329819213E6CF85E0E2
:10ACA00080939E050CC080913F0910923F09882334
:10ACB00019F30E946C2E80919F058823E9F20F9072
:10ACC0000F900F90DF91CF911F910F91FF90EF9018
:10ACD000DF90CF90BF90AF909F908F907F906F90BC
:10ACE0005F904F903F902F9008958A81813009F0B6
:10ACF0006BC01092470910924B0910924A091092AA
:10AD00004909109248098091A0058130F1F08091A5
:10AD10007502882309F4BDCF11E08091A005813030
:10AD200009F010E060917A0670917B0680917C06B4
:10AD300090917D060E94651F00E09C014FEE58E057
:10AD4000632D812F0E942048A4CF80913F0910924B
:10AD50003F098823E1F20F94BF1520E030E048EC72
:10AD600052E460917A0670917B0680917C06909106
:10AD70007D060F94173A20E030EB4AE156E40F9439
:10AD8000083E0F947B3F1F92E3EF8E2EE0E29E2E53
:10AD9000F0EFAF2EF7E4BF2E6B0118E5E12E1DE4B6
:10ADA000F12E00E010E024E539ED4FEF5FEF6AE7A8
:10ADB00076E08FEE98E00E94EB2C0F9080919F053B
:10ADC000882309F4A4CF7BCF9A81923009F0DDC0AB
:10ADD0006092470910924B0910924A091092490952
:10ADE000109248098091A0058230D9F080917502B7
:10ADF000882309F44ECF11E08091A005823009F03C
:10AE000010E060917E0670917F068091800690919F
:10AE100081060E94651F00E09C014FEE58E0642D02
:10AE200090CF80913F0910923F098823F9F20F9447
:10AE3000BF1520E030E048EC52E460917E0670914E
:10AE40007F0680918006909181060F94173A20E04A
:10AE500030EB4AE156E40F94083E0F947B3F1F927B
:10AE600033EF832E30E2932E40EFA42E47E4B42E2E
:10AE70006B0118E5E12E1DE4F12E00E010E024E561
:10AE800039ED4FEF5FEF6EE776E08FEE98E00E94CE
:10AE9000EB2C0F9080919F05882309F4A7CF0FCF4B
:10AEA0005092470910924B0910924A091092490991
:10AEB000109248098091A0058330D9F080917502E5
:10AEC000882309F4E6CE11E08091A005833009F0D3
:10AED00010E06091820670918306809184069091C3
:10AEE00085060E94651F00E09C014FEE58E0672D2B
:10AEF00028CF80913F0910923F098823F9F20F94DF
:10AF0000BF1520E030E048EC52E460918206709179
:10AF1000830680918406909185060F94173A20E06D
:10AF200030E048E453E40F94083E0F947B3F1F92B7
:10AF300083EF882E80E2982E90EFA92E97E4B92E09
:10AF40006B0110EBE12E14E0F12E00E010E028E39D
:10AF50003FEF4FEF5FEF62E876E08FEE98E00E9400
:10AF6000EB2C0F9080919F05882309F4A7CFA7CEE3
:10AF700080913F0910923F09882391F00E94D92BBC
:10AF800080919F05882361F09ACE8A81833009F4ED
:10AF900087CF843009F07DCE8091A005843041F3C5
:10AFA00080917502882309F474CE89ED9BE29F930A
:10AFB0008F938EE399E09F938F938B818F9381E0A2
:10AFC0009091A005943009F080E08F930E947D2538
:10AFD0000F900F900F900F900F900F905ACE5F929E
:10AFE0006F927F928F929F92AF92BF92CF92DF9299
:10AFF000EF92FF920F931F93CF93DF9361E081E075
:10B000000E943223C091A10525E0722E7C0ED1E072
:10B01000DC1B6C2E6194C11134C01091A00511236A
:10B02000A1F080917502882349F081E0111180E040
:10B0300024E041E159E0662D0F941E15CF5F7C128C
:10B04000EACF82E080939E050CC080913F09109268
:10B050003F09882331F30E946C2E80919F0588233D
:10B0600001F3DF91CF911F910F91FF90EF90DF904F
:10B07000CF90BF90AF909F908F907F906F905F9098
:10B080000895C130D9F65090A00581E0581609F412
:10B0900047C080917502882389F211E0511210E0B7
:10B0A000C0908606D0908706E0908806F0908906CA
:10B0B00020E030E0A901C701B6010F94B1392DEBB2
:10B0C00037E346E055EB87FD04C02DEB37E346E060
:10B0D00055E3C701B6010F94083E6B017C0120E0E7
:10B0E00030E0A9010F94B13920E030E040E05FEB9F
:10B0F00087FD04C020E030E040E05FE3C701B60117
:10B100000F94083E0F94743FCB010E9492BD00E063
:10B110009C0147EE58E06D2F812F0E9420488ECF72
:10B1200080913F0910923F09882309F4B2CF6091C2
:10B1300086067091870680918806909189060F9403
:10B140007B3F1F92912C812C8AEEA82E87E4B82E8B
:10B150006B011AE0E12EF12C00E010E020E030E07D
:10B16000A90166E876E087EE98E00E94EB2C0F904C
:10B1700080919F05882309F48CCF73CF2F923F9243
:10B180004F925F926F927F928F929F92AF92BF92F7
:10B19000CF92DF92EF92FF920F931F93CF93DF93A3
:10B1A00000D000D01F921F92CDB7DEB72091470983
:10B1B000288761E081E00E9432233091A1053F831E
:10B1C000E8858E2F90E0880F991F9C01275E314FF4
:10B1D0003C832B8336E0E39FC0011124FC01EC503B
:10B1E000FA4FFA83E9839C012E503A4F79015F8030
:10B1F00035E0432E450C11E0312E3518252C2194D5
:10B20000FE82ED82570134E0A30EB11C49EDC42E3D
:10B210004BE2D42E85E0782E75184701E2E08E0EC1
:10B22000911C82E0682E6518FF81F11161C0112325
:10B23000D9F08091A0051816BCF040913B095091BF
:10B240003C0960913D0970913E094F5F5F4F6F4F20
:10B250007F4F40933B0950933C0960933D097093A5
:10B260003E098F5F8093A00580917502882341F08D
:10B27000EB81FC816591749143E0822D0F949314CE
:10B28000F501808180933609FF81F23009F080C09A
:10B2900028852093470910924B0910924A09109271
:10B2A0004909109248098091A005823009F45DC0D7
:10B2B00080917502882391F011E08091A005823081
:10B2C00009F010E0809136090E942ABE00E09C013E
:10B2D00047E059E0662D812F0E94204810E02F8121
:10B2E0002F5F2F834212A0CF86E080939E0519C066
:10B2F0002F81213029F61091A005113031F0809175
:10B300007502811127C010E0BBCF80913F091092D8
:10B310003F098823A1F30E946C2E80919F0588230A
:10B3200071F328960FB6F894DEBF0FBECDBFDF9144
:10B33000CF911F910F91FF90EF90DF90CF90BF9032
:10B34000AF909F908F907F906F905F904F903F90C5
:10B350002F90089581E0113009F080E024E041E170
:10B3600059E0632D0F941E15CECF80913F091092A6
:10B370003F09882309F49CCF65EE70E287E099E0ED
:10B380000F94A41780919F05882309F491CFC9CF0A
:10B390003F81333091F58091A0058330C1F08091D9
:10B3A0007502882309F49ACF11E08091A0058330BB
:10B3B00009F010E0ED81FE81808191810E9492BDB3
:10B3C00063E0651900E09C0140E059E084CF809182
:10B3D0003F0910923F09882311F310E000E025EFA8
:10B3E00030E045E050E0B70180E099E00F94CC16E2
:10B3F00080919F05882399F294CFFF81F43091F5D5
:10B400008091A0058430B9F080917502882309F4F9
:10B4100065CF11E08091A005843009F010E0F401BF
:10B42000808191810E9492BD64E0651900E09C01D9
:10B430004CEF58E050CF80913F0910923F0988238C
:10B4400019F310E000E024E630E045E050E06981C7
:10B450007A818CEF98E00F94CC1680919F05882319
:10B4600099F25FCFFF81F53009F039CF8091A005C7
:10B470008530E1F080917502882309F42FCFDF92A7
:10B48000CF928EE399E09F938F937F9281E090918A
:10B49000A005953009F080E08F930E947D250F90E4
:10B4A0000F900F900F900F900F9018CF80913F0941
:10B4B00010923F098823F1F20E94D92B80919F05B9
:10B4C0008823C1F22ECF5F926F927F928F929F92CC
:10B4D000AF92BF92CF92DF92EF92FF920F931F93A2
:10B4E000CF93DF93CDB7DEB760970FB6F894DEBF8A
:10B4F0000FBECDBF80E1ECE8F2E0DE0111960190D5
:10B500000D928A95E1F761E081E00E943223D090AC
:10B51000A1059D2C65E0862E8D0C7D2C719473E029
:10B52000672ED11012C01091A005112309F4CEC0CE
:10B5300080917502882349F081E0111180E024E0B8
:10B540004CE358E0672D0F941E15AA24A394B12C48
:10B550005D2C5918DA102FC08FEF8A0D80934709A0
:10B5600010924B0910924A09109249091092480909
:10B570008091A0058D1509F4CDC0809175028823B6
:10B58000D1F011E08091A0058D1110E0F501EE0FD2
:10B59000FF1FEE0FFF1FEB5AF64F60A171A182A1B2
:10B5A00093A10E94F52700E09C014CEE57E0652D29
:10B5B000812F0E942048CA2C81E08A0D9FEFA91A92
:10B5C000B90A94E0A916B10429F68D112CC0609235
:10B5D000470910924B0910924A091092490910929A
:10B5E00048098091A0058D1509F4BEC080917502AF
:10B5F0008823C9F0BD2CB91811E08091A0058D11E8
:10B6000010E0609185097091860980918709909179
:10B6100088090E94F52700E09C014CEE57E06B2D55
:10B62000812F0E94204882E08C0D8D1122C08091D4
:10B63000A0058D1509F4B6C0809175028823C9F064
:10B64000BD2CB91811E08091A0058D1110E060911A
:10B6500095097091960980919709909198090E9497
:10B66000F52700E09C014FED57E06B2D812F0E94E4
:10B67000204883E08C0D8D1121C08091A0058D158F
:10B6800009F4ADC0809175028823C1F011E080916A
:10B69000A0058D1110E06091990970919A0980912F
:10B6A0009B0990919C090E94F52700E09C014EECBB
:10B6B00057E06D2D6919812F0E942048D3948D1079
:10B6C00030CF84E08C0D80939E050EC080913F09A1
:10B6D00010923F09882309F42BCF0E946C2E809191
:10B6E0009F05882309F424CF60960FB6F894DEBF37
:10B6F0000FBECDBFDF91CF911F910F91FF90EF90C3
:10B70000DF90CF90BF90AF909F908F907F906F9081
:10B710005F90089580913F0910923F09882309F4B2
:10B720002CCF0F94BF15B501660F771F660F771FDB
:10B73000FB01349781E090E08C0F9D1FE80FF91F0B
:10B74000E080F180028113816B58764F20E030E079
:10B7500040E85FE38CEE97E00F94CB1580919F0556
:10B76000882309F40ACFC0CF80913F0910923F0986
:10B77000882309F43BCF0F94BF15E12C1CE3F12E75
:10B780000CE116E420E030E040E85FE365E879E0B2
:10B790008CEE97E00F94CB1580919F05882309F4D8
:10B7A00025CFA2CF80913F0910923F09882309F449
:10B7B00043CF0F94BF15E12C1CE3F12E0CE116E4EE
:10B7C00020E030E0A90165E979E08FED97E00F9482
:10B7D000CB1580919F05882309F42ECF85CF8091CA
:10B7E0003F0910923F09882309F44CCF0F94BF15ED
:10B7F000E12C1CE3F12E0CE116E420E030E0A9017D
:10B8000069E979E08EEC97E00F94CB1580919F0564
:10B81000882309F437CF68CF2F923F924F925F92DF
:10B820006F927F928F929F92AF92BF92CF92DF9250
:10B83000EF92FF920F931F93CF93DF93CDB7DEB7B5
:10B840002C970FB6F894DEBF0FBECDBFC09059093C
:10B85000D0905A09E0905B09F0905C0980915D09F5
:10B8600090915E09A0915F09B09160098C159D05CA
:10B87000AE05BF0510F4D701C601C0905509D090A0
:10B880005609E0905709F0905809BC01CD016C159C
:10B890007D058E059F0510F4C701B6010F94B639DA
:10B8A0002B013C0161E081E00E9432232091A1053F
:10B8B0002C872E83822F8B5F8D8387E0821B8F8363
:10B8C00086E0821B888785E0821B898784E0821B53
:10B8D0008A8783E0821B8B8742E0242E221A322E35
:10B8E00031942C85211140C01091A0051123B9F08D
:10B8F00080917502882349F081E0111180E024E0F5
:10B900004CE358E0632D0F941E159C859F5F9C8728
:10B910002D812913E6CF88E080939E050CC080918D
:10B920003F0910923F09882319F30E946C2E8091E1
:10B930009F058823E9F22C960FB6F894DEBF0FBE60
:10B94000CDBFDF91CF911F910F91FF90EF90DF90CE
:10B95000CF90BF90AF909F908F907F906F905F90AF
:10B960004F903F902F9008958C85813009F081C0D1
:10B970008091A0058130F9F080917502882329F229
:10B9800011E08091A005813009F010E060918909F3
:10B9900070918A0980918B0990918C090E94F527FA
:10B9A00061E02E81621B00E09C014BE258E0812F98
:10B9B0000E942048AACF80913F0910923F09882316
:10B9C000D9F20F94BF152AE037ED43E25DE3C301DE
:10B9D000B2010F94173A4B015C0120E030E040E0E7
:10B9E0005FE40F94B13987FD05C0812C912CA12C07
:10B9F0003FE4B32E2AE037ED43E25DE3609189092D
:10BA000070918A0980918B0990918C090F94173A53
:10BA100020E030E040E85FE30F94073E0F947B3F67
:10BA200069837A838B839C83C501B4010F94743F2F
:10BA30007B018C0121E0E21AF108010911091F9232
:10BA4000912C812C22E0A22E28E4B22EC980DA802B
:10BA500021E030E040E050E069E879E08BE298E0F6
:10BA60000E94EB2C0F9080919F05882309F484CFCE
:10BA700062CF8C85823009F0A6C18091A00582300A
:10BA8000D9F080917502882309F43FCF11E08091AD
:10BA9000A005823009F010E060918D0970918E0947
:10BAA00080918F09909190090E94F52700E09C01F8
:10BAB0004DE158E0622D7BCF80913F0910923F0904
:10BAC0008823F9F20F94BF156091610970916209A2
:10BAD00080916309909164090F94B6397B018C01C0
:10BAE00020E030E048EC52E46DE879E08DE198E048
:10BAF0000F94CB1580919F05882319F21CCF80915C
:10BB0000A0058330D9F080917502882309F4FDCE19
:10BB100011E08091A005833009F010E06091910957
:10BB20007091920980919309909194090E94F52750
:10BB300000E09C0140E158E06B8539CF80913F09DE
:10BB400010923F098823F9F20F94BF152AE037EDD0
:10BB500043E25DE3C301B2010F94173A4B015C016C
:10BB600020E030E040E05FE40F94B13987FD05C08C
:10BB7000812C912CA12C9FE4B92E2AE037ED43E2D1
:10BB80005DE3609191097091920980919309909180
:10BB900094090F94173A20E030E040E85FE30F94F7
:10BBA000073E0F947B3F69837A838B839C83C50117
:10BBB000B4010F94743F7B018C0121E0E21AF1087B
:10BBC000010911091F92912C812C82E0A82E88E492
:10BBD000B82EC980DA8021E030E040E050E061E931
:10BBE00079E080E198E00E94EB2C0F9080919F0516
:10BBF000882309F488CF9FCE1092470910924B09F1
:10BC000010924A0910924909109248098091A005A2
:10BC10008430E9F080917502882309F476CE11E032
:10BC20008091A005843009F010E060915509709171
:10BC3000560980915709909158090F94B6390E947E
:10BC4000D22700E09C0144E058E06A85B0CE8091A4
:10BC50003F0910923F098823E9F20F94BF150CE7C2
:10BC600018E224E630E040E050E065E579E084E069
:10BC700098E00F94541680919F05882359F25BCE6B
:10BC800081E08093470910924B0910924A09109263
:10BC90004909109248098091A0058530E9F080910A
:10BCA0007502882309F431CE11E08091A00585301A
:10BCB00009F010E06091590970915A0980915B096F
:10BCC00090915C090F94B6390E94D22700E09C0144
:10BCD00044E058E069856BCE80913F0910923F099E
:10BCE0008823E9F20F94BF150AE718E224E630E052
:10BCF00040E050E069E579E084E098E00F94541664
:10BD000080919F05882359F216CE82E080934709DF
:10BD100010924B0910924A09109249091092480951
:10BD20008091A0058630E9F080917502882309F49E
:10BD3000ECCD11E08091A005863009F010E0609113
:10BD40005D0970915E0980915F09909160090F947F
:10BD5000B6390E94D22700E09C0144E058E0688593
:10BD600026CE80913F0910923F098823E9F20F9473
:10BD7000BF1508E718E22AE030E040E050E06DE54A
:10BD800079E084E098E00F94541680919F05882311
:10BD900059F2D1CD80913F0910923F09882339F1A2
:10BDA0000F94BF1506E718E224E630E040E050E0CB
:10BDB00061E679E088EF97E00F94541680919F0533
:10BDC0008823A9F0B8CD8C85833009F498CE8430CF
:10BDD00009F412CF853009F453CF863009F495CF9A
:10BDE000873009F092CD8091A005873099F280913B
:10BDF0007502882309F489CD11E08091A005873070
:10BE000009F010E060916109709162098091630905
:10BE1000909164090F94B6390E94D22700E09C01EA
:10BE200048EF57E06F81C3CD2F923F924F925F92C0
:10BE30006F927F928F929F92AF92BF92CF92DF923A
:10BE4000EF92FF920F931F93CF93DF9300D01F9237
:10BE50001F92CDB7DEB761E081E00E94322380916E
:10BE6000A1058C838A83982F9B5F9983E82FE195A6
:10BE7000EB8384E0482EFC814F1A8C81811114C021
:10BE80009091A0059D83992309F489C08091750242
:10BE9000882351F081E0ED81E11180E024E04CE362
:10BEA00058E06B810F941E1565E5662E69E0762ECD
:10BEB000F1E0FD833C803A942C808A81281A9C8191
:10BEC000ED819E1328C03092470910924B091092C1
:10BED0004A0910924909109248098091A0058917D2
:10BEE00009F483C0809175028823A9F011E0809144
:10BEF000A005FD818F1310E0F3016489758986899F
:10BF000097890E94052100E09C0141E358E0622DE1
:10BF1000812F0E9420485D80F4E06F0E711C81E04B
:10BF2000850D8D83843059F69C81943069F5E3E06A
:10BF3000E093470910924B0910924A09109249095F
:10BF4000109248098091A005843009F48CC080913A
:10BF500075028823C9F0F1E0FD838091A00584304B
:10BF600009F01D82609175097091760980917709B9
:10BF7000909178090E94052100E09C0141E358E07E
:10BF8000642D8D810E9420488C818F5F8C839981E4
:10BF9000981373CF5394539450929E050EC0809182
:10BFA0003F0910923F09882309F470CF0E946C2E3C
:10BFB00080919F05882309F469CF0F900F900F900F
:10BFC0000F900F90DF91CF911F910F91FF90EF9005
:10BFD000DF90CF90BF90AF909F908F907F906F90A9
:10BFE0005F904F903F902F90089580913F0910925D
:10BFF0003F09882309F476CF0F94BF1520E030E085
:10C0000040E251E4F30164897589868997890F9428
:10C01000173A20E030E048E452E40F94073E0F94D2
:10C020007B3F1F9234E7832E38E2932E46EFA42EF7
:10C0300047E4B42E6B0114E6E12E16E8F12E01E080
:10C0400010E022E330E040E050E0B3016C5E7F4F4F
:10C0500081E398E00E94EB2C0F9080919F0588234C
:10C0600009F440CFAACF80913F0910923F0988235D
:10C0700009F46DCF0F94BF1520E030E040E251E4A9
:10C08000609175097091760980917709909178098E
:10C090000F94173A20E030E048E452E40F94073E52
:10C0A0000F947B3F1F9282E7882E88E2982E96EFAE
:10C0B000A92E97E4B92E6B0114E6E12E16E8F12EB5
:10C0C00001E010E022E330E040E050E065E779E095
:10C0D00081E398E00E94EB2C0F9080919F058823CC
:10C0E00009F435CF6ACF2F923F924F925F926F92B1
:10C0F0007F928F929F92AF92BF92CF92DF92EF92F8
:10C10000FF920F931F93CF93DF9300D000D0CDB752
:10C11000DEB761E081E00E9432232091A1052D83EA
:10C120002E83322F3B5F398381E0922F821B8A83DB
:10C1300091959B8382E0821B8C83FD81F11185C1E7
:10C140001091A005112309F459C18091750288232B
:10C1500049F081E0111180E024E04CE358E06B816C
:10C160000F941E158091F105882309F437C2FD81D3
:10C17000F23029F58091A005823009F4A2C18091A6
:10C1800075028823E1F011E08091A005823009F06A
:10C1900010E0E091510924E0E29FF0011124E75101
:10C1A000FA4F60817181828193810E94E62100E0D3
:10C1B0009C0144E957E06C81812F0E942048712C3A
:10C1C000612C13E0312E2D803E81231A8D81831145
:10C1D0002EC06092470910924B0910924A091092A2
:10C1E0004909109248098091A0059D81891709F499
:10C1F000B1C1809175028823D1F011E08091A00532
:10C20000831110E0F301EE0FFF1FEE0FFF1FE75148
:10C21000FA4F60817181828193810E94E62100E062
:10C220009C0148E857E0622D812F0E942048FFEFD3
:10C230006F1A7F0A24E032128AC115E03D81131380
:10C2400029C08091A005811709F4CAC180917502A7
:10C25000882301F16D809E81691A772473948091FF
:10C26000A005ED818E13712CE091510928E0E29F29
:10C27000F0011124E752FA4F60817181828193812C
:10C280000E94362800E09C014EE757E0662D872D7E
:10C290000E94204844244394410E712C612C3D801F
:10C2A0003E81331A8D8184112FC06092470910920C
:10C2B0004B0910924A09109249091092480980913D
:10C2C000A0059D81891709F4AAC180917502882370
:10C2D000D9F011E08091A005841110E0F30133E062
:10C2E000EE0FFF1F3A95E1F7E752FA4F6081718137
:10C2F000828193810E94362800E09C0145E757E047
:10C30000632D812F0E942048542C44244394450CD3
:10C310006A94672809F07FC1FD814F1228C080917F
:10C32000A0058F1709F496C1809175028823F9F052
:10C330007D803E81731A11E08091A0059D81891353
:10C3400010E0E091510928E0E29FF0011124E7524A
:10C35000FA4F64817581868197810E94362800E0BA
:10C360009C014DE657E0672D812F0E942048539491
:10C370005394712C612C4D803E81431A8D8185111F
:10C380002FC06092470910924B0910924A091092EF
:10C390004909109248098091A0059D81891709F4E7
:10C3A00078C1809175028823D9F011E08091A005B1
:10C3B000851110E0F30183E0EE0FFF1F8A95E1F78E
:10C3C000E752FA4F64817581868197810E943628F1
:10C3D00000E09C0146E657E0642D812F0E94204832
:10C3E00053946A94672809F050C1FD81FF5FFD8373
:10C3F00029812F13A2CE50929E050EC080913F0935
:10C4000010923F09882309F4A0CE0E946C2E8091DF
:10C410009F05882309F499CE26960FB6F894DEBFBF
:10C420000FBECDBFDF91CF911F910F91FF90EF9085
:10C43000DF90CF90BF90AF909F908F907F906F9044
:10C440005F904F903F902F9008952D81213009F0FB
:10C4500089CE8091A0058130D1F08091750288232A
:10C4600009F480CE81E09091A005913009F080E040
:10C470009091F10522EC37E0911102C02EEB37E0EC
:10C4800001E04EE957E06A810E9420486BCE80911E
:10C49000F10590913F0910923F099923F1F23D81F6
:10C4A00083278093F10583E080937502E7EEF1E73F
:10C4B000EF2B11F00E94E77180919F05882369F2AC
:10C4C000ABCF80913F0910923F09882309F457CEE2
:10C4D0000F94BF156090510924E0629E3001112431
:10C4E000C30187519A4F3C0120E030E04AE754E411
:10C4F000FC0160817181828193810F94173A20E061
:10C5000030E84BEB54E40F94073E0F947B3F1F92AF
:10C5100007EE802E01E7902E8AE1A82E88E4B82E3F
:10C520006B0116EDE12E16E0F12E00E010E02CED8F
:10C5300035E040E050E0B30184E997E00E94EB2C45
:10C540000F9080919F05882309F419CE65CFB4E040
:10C550003B2E3CCE80913F0910923F09882309F47D
:10C5600048CE0F94BF15C301880F991F880F991FDC
:10C57000FC01E751FA4F2F0120E030E04AE754E494
:10C5800060817181828193810F94173A20E030E8B5
:10C590004BEB54E40F94073E0F947B3F1F92E7EE62
:10C5A0008E2EE1E79E2EFAE1AF2EF8E4BF2E6B014E
:10C5B00016EDE12E16E0F12E00E010E02CED35E056
:10C5C00040E050E0B20188E897E00E94EB2C0F9029
:10C5D00080919F05882309F40CCE1ECF12E02ECE49
:10C5E00080913F0910923F09882309F42FCE0F94C0
:10C5F000BF156091510988E0689FB001112467520E
:10C600007A4F8EE797E00F946A1780919F058823F1
:10C6100009F41CCE01CF66246394712C43CE809123
:10C620003F0910923F09882309F44FCE0F94BF159C
:10C63000B30143E0660F771F4A95E1F767527A4FDF
:10C6400085E797E00F946A1780919F05882309F486
:10C650003CCEE2CE80913F0910923F09882309F435
:10C6600063CE0F94BF156091510928E0629FB0011D
:10C67000112463527A4F8DE697E00F946A178091E8
:10C680009F05882309F450CEC7CE66246394712C8D
:10C6900075CE80913F0910923F09882309F481CE1D
:10C6A0000F94BF15B30193E0660F771F9A95E1F7DA
:10C6B00063527A4F86E697E00F946A1780919F0540
:10C6C000882309F46ECEA8CE2F923F924F925F92AC
:10C6D0006F927F928F929F92AF92BF92CF92DF9292
:10C6E000EF92FF920F931F93CF93DF9300D0CDB7BC
:10C6F000DEB761E081E00E9432232091A1052A8308
:10C700002B5F298384E09A81891B8B8323E0522E3F
:10C71000352C391A82E0782E791A81E0682E691A50
:10C72000292E21942A8121113DC01091A0051123A9
:10C73000B9F080917502882349F081E0111180E001
:10C7400024E04CE358E0622D0F941E152A812F5FE0
:10C750002A8389812813E6CF85E080939E050CC04B
:10C7600080913F0910923F09882319F30E946C2E93
:10C7700080919F058823E9F20F900F900F90DF9131
:10C78000CF911F910F91FF90EF90DF90CF90BF90CE
:10C79000AF909F908F907F906F905F904F903F9061
:10C7A0002F9008958A81813071F59091A005913084
:10C7B000B9F080917502882349F281E0913009F047
:10C7C00080E090916D0622EC37E0911102C02EEBD3
:10C7D00037E001E045EC57E0662D0E942048B6CFD7
:10C7E00080913F0910923F09882319F380916D06CB
:10C7F0002A81822780936D065092750280919F0551
:10C800008823B9F2B9CF8A81823009F098C080912B
:10C81000A0058230C1F080917502882309F496CF7B
:10C8200011E08091A005823009F010E0809118029B
:10C83000909119020E9492BD00E09C0147EB57E0E5
:10C84000672D812FCACF80913F0910923F0988231D
:10C8500011F310E000E025EF30E050E040E068E147
:10C8600072E087EB97E00F94CC1680919F058823A8
:10C8700091F282CF8091A0058330B9F0809175024A
:10C88000882309F463CF11E08091A005833009F07B
:10C8900010E080911602909117020E9492BD00E074
:10C8A0009C0140EB57E0632DCCCF80913F09109263
:10C8B0003F09882319F310E000E025EF30E050E055
:10C8C00040E066E172E080EB97E00F94CC16809137
:10C8D0009F05882399F250CF80913F0910923F091C
:10C8E0008823C9F120E030E048EC52E46091120264
:10C8F0007091130280911402909115020F94173ACF
:10C900000F947B3F1F92912C812C80EFA82E87E4FF
:10C91000B82E6B0118EEE12E13E0F12E00E010E0CE
:10C9200020E030E0A90162E172E088EA97E00E942D
:10C93000EB2C0F9080919F05882369F01DCF9A8181
:10C94000933009F497CF943009F000CF4090A005C0
:10C9500094E0491609F280917502882309F4F6CE15
:10C96000609112027091130280911402909115024D
:10C970000E94651F9C0181E094E0491280E000E084
:10C9800048EA57E06B8129CFE5E4F6E183AF64AF75
:10C990006FEF7FEFCA010C947FC72F923F924F92A7
:10C9A0005F926F927F928F929F92AF92BF92CF923F
:10C9B000DF92EF92FF920F931F93CF93DF9300D0FC
:10C9C00000D01F921F92CDB7DEB710924509E091BB
:10C9D0001712F0911812309721F0199581110F94C8
:10C9E0008E1080913F0910923F09882319F120E0B1
:10C9F00040E070E060E08EE89BE30E9493230E9499
:10CA0000DE3F28960FB6F894DEBF0FBECDBFDF9194
:10CA1000CF911F910F91FF90EF90DF90CF90BF903B
:10CA2000AF909F908F907F906F905F904F903F90CE
:10CA30002F90089580919705882309F434C260915E
:10CA4000470670914806072E000C880B990B0F942F
:10CA5000B83911E0209143063091440640914506D3
:10CA6000509146060F94684018160CF010E0609143
:10CA70005E0670915F06072E000C880B990B0F94D1
:10CA8000B8399B01AC0160915A0670915B068091A8
:10CA90005C0690915D060F94B13987FD12600E948B
:10CAA0003BC88111146010932E0520916D0F3091B9
:10CAB0006E0F40916F0F5091700F609176027091E0
:10CAC000770280917802909179020F94083E4B0191
:10CAD0005C012091710F3091720F4091730F509152
:10CAE000740F60917A0270917B0280917C02909128
:10CAF0007D020F94083E6D837E838F8398872091FB
:10CB0000750F3091760F4091770F5091780F6091AB
:10CB10007E0270917F0280918002909181020F9439
:10CB2000083E2B013C0120E030E040E251E40F944C
:10CB3000173A20E030E048EC52E40F94173A6B01CA
:10CB40007C0120E030E0A901C301B2010F94B139AA
:10CB500020E030E040EA50EC87FD04C020E030E007
:10CB600040EA50E4C701B6010F94083E20E030E0EF
:10CB700040E251E40F94023F0F94743F2B013C01BB
:10CB800080E277FE09C07094609450944094411CF8
:10CB9000511C611C711C8DE28093A20560E220E1B2
:10CBA000421627E25206610471048CF0C301B201FF
:10CBB00020E137E240E050E00F94C63DCA01B901E0
:10CBC0002AE030E040E050E00F94C63D605D6093A5
:10CBD000A30560E238EE431633E0530661047104A6
:10CBE0008CF0C301B20128EE33E040E050E00F9436
:10CBF000C63DCA01B9012AE030E040E050E00F94A0
:10CC0000C63D605D6093A405C301B20124E630E037
:10CC100040E050E00F94C63D6AE0C62ED12CE12CD6
:10CC2000F12CCA01B901A70196010F94C63D605DC0
:10CC30006093A505C301B201A70196010F94C63DFB
:10CC4000162FCA01B901A70196010F94C63D112301
:10CC500009F4F6C08EE28093A605605D6093A70597
:10CC6000105D1093A80562EA75E086E295E00F94E6
:10CC7000ED4120E030E0A901C501B4010F94B139C4
:10CC800020E030E040E05FEB87FD04C020E030E0D2
:10CC900040E05FE3C501B4010F94083E0F94743F78
:10CCA000CB010E9413BDBC0181E295E00F94ED41E0
:10CCB00020E030E0A9016D817E818F8198850F94FD
:10CCC000B13920E030E040E05FEB87FD04C020E0B8
:10CCD00030E040E05FE36D817E818F8198850F9425
:10CCE000083E0F94743FCB010E9413BDBC018CE140
:10CCF00095E00F94ED418091A21714E683FD29C0C1
:10CD00000E9473CD882309F4ADC080919A17909149
:10CD10009B17A0919C17B0919D170097A105B10595
:10CD200009F4A0C0BC01CD016D597F4F8F4F9F4FBB
:10CD300024E630E040E050E00F94A43D60919E175F
:10CD400070919F178091A0179091A1170F94A43D07
:10CD5000122F0E94E4BA4B015C01062F80910F0252
:10CD60008117A1F010930F0288E4189FB0011124DD
:10CD700090E080E00F94B6392AE037ED43E25CE3BF
:10CD80000F94173A0F947B3F60931B0580910E021E
:10CD9000081709F488C080920E02C501B40120E191
:10CDA0003EE040E050E00F94A43DC22E732EE22EF0
:10CDB000F32E5CE3252E312C412C512CC501B401FE
:10CDC000A20191010F94A43D062F672ECA01B9015B
:10CDD000A20191010F94A43D162FD72E90E8891639
:10CDE00091E5990691E0A906B104F0F1C501B401FD
:10CDF00020E831E541E050E00F94A43D5901DF9275
:10CE00001F93C70168E170E00F9434419F938F93A3
:10CE10003F932F938FE796E09F938F938BE095E05E
:10CE20009F938F930F9448390FB6F894DEBF0FBECF
:10CE3000CDBF89E0BAE0AB16B10470F588E02CC034
:10CE4000662351F08EE28093A605605D6093A7058E
:10CE500080E28093A80507CF80E28093A7058093A6
:10CE6000A605F6CF10E075CFE114F10409F087C2F2
:10CE70006F920F93DF921F9383E796E09F938F93B8
:10CE80008BE095E09F938F930F9448390FB6F894F9
:10CE9000DEBF0FBECDBF85E0982F990F990F891B7C
:10CEA000855A80930A050E94F224D82E81E00E94C0
:10CEB000AA3F80912E05982F947042E102E082FFF4
:10CEC00002C048E00CE080917D16843180F48091AE
:10CED0007F16841760F0992309F471C28BE197E003
:10CEE0007C0123E060E589E496E10F94852680913A
:10CEF0007D168431B8F480917F16823098F0DD2061
:10CF000009F460C28091D205882309F45BC28FEDD9
:10CF100096E07C0102E123E042E068E689E496E1E4
:10CF20000F94852680917D168C3108F0EAC02FE39E
:10CF3000222E26E0322E1FE0B12CA12C39E0432E08
:10CF4000512C612C712C4CE1C42E3A2DD101149638
:10CF50008D919D910D90BC91A02D8D839E83AF836B
:10CF6000B887F1018084918480917D16843118F511
:10CF700080917F168830F8F062E2A11001C068E06D
:10CF8000F501E855FD4F208180912E0590E002C00B
:10CF9000959587953A95E2F7F501EE0FFF1F80FF13
:10CFA00014C2EB55F94FE590F4900CE048E089E4A9
:10CFB00096E10F94852680917D168830B0F4D110CB
:10CFC0000BC025E02A9DF0012B9DF00D1124E25E9F
:10CFD000F94F8481811109C097FEFAC14DE956E0ED
:10CFE00067E087EF810F0E94C46480917D168C31C9
:10CFF000C8F480917F168431A8F020E030E040E052
:10D000005FE36D817E818F8198850F94083E0F9438
:10D01000743F77FF08C24DE956E06CE187EF810F5E
:10D020000E94C4643FEFA31AB30A87E1280E311CA3
:10D03000165E133409F089CF809032069090330643
:10D04000A0903406B090350680917D16883090F41B
:10D05000D11004C080912C0681110CC0809136063D
:10D060009091370697FF09C24DE956E067E081E5E8
:10D070000E94C46480917D168C31B0F480917F163B
:10D08000843190F020E030E040E05FE3C501B4017E
:10D090000F94083E0F94743F77FF1DC24DE956E090
:10D0A0006CE181E50E94C46480917D168C3148F565
:10D0B00080917F16843128F18091D205882309F16F
:10D0C000E4E68E9FC001112481589F4F6FEF70E0FE
:10D0D0000F944841CB010E9492BD27E62093801611
:10D0E0002CE1209381160E94AD4285E290E0A0E001
:10D0F000B0E089839A83AB83BC83CE0101960E9402
:10D1000067400E9473CD882379F180917D16843326
:10D1100058F580917F168A3238F107E028E04AE21C
:10D120006AE289E496E10F94C72305E022E04CE22D
:10D1300062E389E496E10F94C72324E04AE061E3C7
:10D140008AE20F948D2360914B1670914C1682E306
:10D15000809365168BE28093661625E636E142E3FE
:10D1600089E496E10F94452280917D16853350F431
:10D1700080917F16813330F024E04AE461E386E356
:10D180000F948D2380917D16843368F480917F16EF
:10D19000823348F002E020911B0542E367E389E413
:10D1A00096E10F94C72380917D16803378F48091A7
:10D1B0007F16883258F080910A058093801680E3AC
:10D1C000809381168BE095E00E94AD4280917D16A0
:10D1D000883208F06FC080917F168D3108F46AC0E4
:10D1E0002BE040E86DE180E00F948D2380917D1667
:10D1F000873208F05FC080917F168F3108F45AC0E3
:10D2000088E590E0A0E0B0E089839A83AB83BC839B
:10D2100083E08093801616E210938116CE0101966A
:10D220000E9467408BE08093801610938116DD206A
:10D2300009F480C181E295E00E94AD4289E590E069
:10D24000A0E0B0E089839A83AB83BC8388E28093BB
:10D25000801616E210938116CE0101960E94674057
:10D2600080E38093801610938116DD2009F48AC133
:10D270008CE195E00E94AD428AE590E0A0E0B0E04C
:10D2800089839A83AB83BC838DE48093801616E2F6
:10D2900010938116CE0101960E94674085E5809328
:10D2A000801610938116DD2009F494C186E295E082
:10D2B0000E94AD4280917D168333A8F580917F1640
:10D2C0008B3288F183E00E94AA3F86E090E0A0E0E4
:10D2D000B0E089839A83AB83BC8383E0809380161C
:10D2E00013E310938116CE0101960E94674081E0FE
:10D2F0000E94AA3F80912002909121020E9492BD3B
:10D300002CE020938016109381160E94AD4285E296
:10D3100090E0A0E0B0E089839A83AB83BC83CE0128
:10D3200001960E94674080917D16813408F069CB98
:10D3300080917F16863308F464CB109280168EE3BA
:10D340008093811689E192E10E94A724182F60E85A
:10D3500070E089E192E10E94DDC780E2C82ED12C05
:10D36000E12CF12C153108F04CCBC982DA82EB822A
:10D37000FC82CE0101960E9467401F5FF3CFF4E666
:10D38000EF16F10438F4DF921F937F92CF9287E675
:10D3900096E074CDDF921F937F92CF928DE596E059
:10D3A0009F938F938BE095E09F938F930F944839D1
:10D3B0000FB6F894DEBF0FBECDBF86E06DCD85E120
:10D3C00097E08ECD89EA96E0A4CDEF55F94FEBCDED
:10D3D000C4010E9492BDFC01808193E0803229F457
:10D3E000818192E0803209F491E0892F880F880FC3
:10D3F000392F381B832F810F8093801687E080930D
:10D400008116A3E0B0E0A91BB109CD018E0F9F1FCB
:10D410000E94AD4249825A826B827C82CE01019683
:10D420000E946740E2CDCB010E9492BDFC01808149
:10D4300093E0803229F4818192E0803209F491E016
:10D44000892F880F880FB92FB81B8B2F810F8093DE
:10D450008016C092811623E030E0291B3109C901F2
:10D460008E0F9F1F0E94AD4249825A826B827C823E
:10D47000CE0101960E946740D5CD0E9492BDFC016D
:10D48000808193E0803229F4818192E0803209F436
:10D4900091E0892F880F880FA92FA81B8A2F865A01
:10D4A0008093801687E08093811623E030E0291B6B
:10D4B0003109CF01820F931F0E94AD4289E090E0B5
:10D4C000A0E0B0E089839A83AB83BC83CE01019650
:10D4D0000E946740CFCDCB010E9492BDFC018081AC
:10D4E00093E0803229F4818192E0803209F491E066
:10D4F000892F880F880FB92FB81B8B2F865A8093DE
:10D5000080168CE18093811623E030E0291B3109DD
:10D51000CF01820F931F0E94AD4289E090E0A0E00E
:10D52000B0E089839A83AB83BC83CE0101960E94CD
:10D530006740BACD0F94171180FF19C001E215E0C2
:10D54000D8018D918D01882309F478CE8F320CF0AB
:10D550008FE3082E000C990BAA0BBB0B89839A83CF
:10D56000AB83BC83CE0101960E946740E9CF8091D6
:10D57000E40880FD5FCE6FEF7FEF88E996E00E94C0
:10D580007FC75CCE0F94171181FF19C00CE115E025
:10D59000F80181918F01882309F46ECE8F320CF04F
:10D5A0008FE3082E000C990BAA0BBB0B89839A837F
:10D5B000AB83BC83CE0101960E946740E9CF809186
:10D5C000E40881FD55CE6FEF7FEF88E996E00E9479
:10D5D0007FC752CE0F94171182FF19C006E215E0E3
:10D5E000D8018D918D01882309F464CE8F320CF01F
:10D5F0008FE3082E000C990BAA0BBB0B89839A832F
:10D60000AB83BC83CE0101960E946740E9CF809135
:10D61000E40882FD4BCE6FEF7FEF80E996E00E9439
:10D620007FC748CECF93DF93FC0125AD211104C005
:10D6300021E025AF0F944922C0914B16D0914C1692
:10D64000E0917A16F0917B1682E01995E0917A16B6
:10D65000F0917B1681E0199530E020E044E1BE01B5
:10D6600089E496E10F9445222CE736E147E1BE01BB
:10D6700089E496E10F944522E0917A16F0917B16A9
:10D6800080E0DF91CF9119944F925F926F927F92D9
:10D690008F929F92AF92BF92CF92DF92EF92FF92C2
:10D6A0001F93CF93DF93CDB7DEB760970FB6F89493
:10D6B000DEBF0FBECDBF0F941E1D6B017C0180919C
:10D6C00010028F3F09F44DC00F941E1D809030054D
:10D6D00090903105A0903205B09033056819790912
:10D6E0008A099B0997FD3DC08091091690910A1601
:10D6F0008F5F8F708917A9F18091100240E050E090
:10D7000065E073E4843050F424E0829FF00111243A
:10D71000E655FD4F40815181628173814D875E875F
:10D720006F87788B19821A821B821C821D821E824F
:10D730001F82188619861A861B861C8640912F0523
:10D74000833011F0409151099E012F5F3F4FBE0180
:10D75000635F7F4F86E792E00E94ACA68FEF8093D5
:10D7600010020E94603E8091FF0382FF33C08091CF
:10D770003B05811131C091E090933B0580914F09A9
:10D78000892780933F0910924F0983E080937502A7
:10D790001092FF030F941E1D6C507E4F8F4F9F4FB2
:10D7A00060933E0570933F0580934005909341053B
:10D7B00068E873E182E090E00E948D2B16E0115042
:10D7C00059F00E94312B62E070E080E090E00F940D
:10D7D000911CF5CF10923B058091FB039091FC03C7
:10D7E000A091FD03B091FE03A7019601281B390B00
:10D7F0004A0B5B0BDA01C901B7FF05C080919405A4
:10D80000882309F4BDC1D701C6018C599F4FAF4F82
:10D81000BF4F8093FB039093FC03A093FD03B09351
:10D82000FE0360913C05062E000C770B77FF03C0CA
:10D8300071956195710990913C0580913A05981315
:10D8400065C0633008F062C010923C0580913C05D1
:10D8500080933A05653008F06BC080913F098111D3
:10D86000E9C080914316909144168D5C944641F432
:10D8700080911102882309F4EFC081508093110236
:10D880000E943C958090CE059090CF05A090D00549
:10D89000B090D10581110E944995D501C4013AE0AB
:10D8A000B695A795979587953A95D1F7009741E05A
:10D8B000A407B10520F08FEF9FEFA0E0B0E09695B0
:10D8C0008795209175022111D9C0309194053111AD
:10D8D00086C180914316909144168D5C944609F45C
:10D8E00065C180914009811161C180913605909197
:10D8F0003705A0913805B0913905C81AD90AEA0A46
:10D90000FB0AF7FC61C10E945E2D5EC18DEF860FA0
:10D91000823008F09BCF80913C0591E087FD9FEF1E
:10D92000892F880F880F890F80933C0565E08ECF83
:10D930008091450921E030E040E050E0882309F47F
:10D9400056C08090410990904209A0904309B09040
:10D95000440981149104A104B104E9F170E090E05C
:10D9600080E00F94B63920E030E040EA50E40F94B4
:10D97000023F2B013C01C701B601681979098A09E8
:10D980009B090F94B6399B01AC01C301B2010F94FE
:10D99000023F20E030E04AE754E40F94173A4B018D
:10D9A0005C0120E030E040EA52E40F94684024E655
:10D9B00030E040E050E087FF12C020E030E040EF70
:10D9C00051E4C501B4010F9468402AE030E040E022
:10D9D00050E087FF04C021E030E040E050E0C0921A
:10D9E0004109D0924209E0924309F0924409A09182
:10D9F0003C050A2E000CBB0B0F94F03D25E030E0F7
:10DA000040E050E00F94C63D80913B0990913C0965
:10DA1000A0913D09B0913E09820F931FA41FB51F2D
:10DA200080933B0990933C09A0933D09B0933E0934
:10DA300010923C05D701C6018856954CAF4FBF4F99
:10DA40008093360590933705A0933805B093390538
:10DA500081E08093750205CF8CE080931102809164
:10DA6000340590913505009729F00197909335057D
:10DA70008093340581E08093750202CF009741F0D6
:10DA800040913405509135054817590708F021CFCA
:10DA900080919405811112C0223038F0243008F4AE
:10DAA00041C0243011F41092750285E496E10E9481
:10DAB000126B81E0809397058093940583E00E9428
:10DAC000AA3F81E080936916E0914316F0914416D5
:10DAD00019951092970580919405811127C0109295
:10DAE0003F0980914316909144168D5C944609F04D
:10DAF000F8CE0F941E1DDC01CB018C199D09AE09D7
:10DB0000BF098090340590903505B12CA12C881662
:10DB10009906AA06BB0608F0DCCE909335058093E3
:10DB20003405D7CE81E080937502BFCF89E496E1BA
:10DB30000F94E72491E0811101C090E09093940547
:10DB4000882369F280914316909144168D5C944627
:10DB5000B9F40F941E1DDC01CB018C199D09AE098F
:10DB6000BF09C0903405D0903505F12CE12CC816C2
:10DB7000D906EA06FB0620F4909335058093340518
:10DB800060960FB6F894DEBF0FBECDBFDF91CF9188
:10DB90001F91FF90EF90DF90CF90BF90AF909F903C
:10DBA0008F907F906F905F904F90089548E9C40EDA
:10DBB0004AE3D41EE11CF11CC0923605D092370511
:10DBC000E0923805F0923905809194058111D8CF03
:10DBD000809175028130A1F610927502D1CF009725
:10DBE00009F46CCF4DCF3F924F925F926F927F922C
:10DBF0008F929F92AF92BF92CF92DF92EF92FF925D
:10DC00000F931F93CF93DF93CDB7DEB7EB970FB68C
:10DC1000F894DEBF0FBECDBF8FEF80931B028091C3
:10DC20009705882369F18091A21700E010E084FF36
:10DC300023C089E894E10E945F808BE1E9E8F4E188
:10DC4000DE01919601900D928A95E1F710E000E0D7
:10DC5000BE016F5F7F4FCE0181960F946C0E181638
:10DC60003CF4CE0101960E94F579080F111DF0CF0A
:10DC7000CE0181960E9464800093950510939605CD
:10DC800061E081E00E9432231091A105412E85E0E0
:10DC9000582E510E312E319491E1A92E9FE1B92ECB
:10DCA00024E1822E2DE0922E81E0682E611A11115E
:10DCB00011C00091A005002329F1809175028823ED
:10DCC00049F081E0011180E024E049E15DE0632D4D
:10DCD0000F941E158091A21786FD59C084FF57C06E
:10DCE000113009F052C00091A005013079F1809106
:10DCF0007502811138C082E01F5F5112D8CF809326
:10DD00009E050CC080913F0910923F098823A9F21B
:10DD10000E946C2E80919F05882379F2EB960FB6B6
:10DD2000F894DEBF0FBECDBFDF91CF911F910F9151
:10DD3000FF90EF90DF90CF90BF90AF909F908F902B
:10DD40007F906F905F904F903F90089580913F0932
:10DD500010923F09882359F20E94111F80919F055C
:10DD6000882329F2DBCFBF92AF929F928F926F925E
:10DD700081E0013009F080E08F930E947D250F90B3
:10DD80000F900F900F900F900F9082E001C081E0F4
:10DD900090917502992309F4AFCF082FD12CC12C93
:10DDA000712E7418802FE0909505F0909605CE1492
:10DDB000DF0408F0A1CF0113A9C081E0E81AF1083F
:10DDC000EC18FD0889E894E10E945F808BE1E9E8A6
:10DDD000F4E1DE01919601900D928A95E1F7F12C24
:10DDE000BE016F5F7F4FCE0181960F946C0E1816A7
:10DDF0007CF4CE0101960E94F579882389F3EF1017
:10DE00006BC0BE016F5F7F4F89E79FE00E94127A6F
:10DE1000CE0181960E9464808091A217F090A005A7
:10DE200085FF79C0F11263C080913F0910923F09CC
:10DE3000882309F45CC019821C8280918C1464EAE6
:10DE400074E1882311F069E874E121E049E75FE0BB
:10DE5000CE0101960E946A80882309F43FC08BE1BD
:10DE6000FE013196A9E8B4E101900D928A95E1F79F
:10DE70008091A2178F7B8093A217A0919717AA3049
:10DE800080F481E08A0F809397178BE18A9FD001FD
:10DE90001124A757B94EE9E8F4E101900D928A9553
:10DEA000E1F7CE0101960E9464801092A10582E004
:10DEB00090E0A0E0B0E080933B0990933C09A093F0
:10DEC0003D09B0933E0981E080939F05109294052F
:10DED00083E08093750222CFF39482CF0E940FD803
:10DEE00069E77FE08EEF9CE00F94E226DACF809125
:10DEF0007502882359F0EE24E394F112E12C6E2D83
:10DF0000872D0E94733F41E0811116C08FEFC81A20
:10DF1000D80A0F5F47CFF116A1F0809175028823D0
:10DF2000A9F3EE24E394F112E12C6E2D872D0E94CB
:10DF3000733F882359F340E0672D8E2D0F944014D2
:10DF4000E5CF80913F0910923F09882331F381EE9C
:10DF500096E20E947D2480919F058823F1F2DECE17
:10DF6000DC01680F791F90E080E02D91E92FFF27F9
:10DF7000E227EE0FFF1FE656FB4D25913491982FB7
:10DF80008827822793276A177B0779F708950F93CD
:10DF90001F93CF93DF93CDB7DEB760970FB6F8949A
:10DFA000DEBF0FBECDBF8C01DC01ED91FC91028084
:10DFB000F381E02DBE016F5F7F4F1995882309F42F
:10DFC00064C08981807CC9F56F81637070E0762FB1
:10DFD0006627770F770F8885B4E08B9FC0011124E7
:10DFE000682B792B89858295869586958370682B19
:10DFF0006F5F7F4F90E080E02A852370220F3B8582
:10E0000037FB332730F9232B3E813F70230F332713
:10E01000331F2750310904C0660F771F881F991FCF
:10E020002A95D2F760960FB6F894DEBF0FBECDBF2B
:10E03000DF91CF911F910F910895803419F5688574
:10E040006695669570E090E080E0CB0177276627C3
:10E050002A85622B098510E0102F0027012E000C65
:10E06000220B330B602B712B822B932B6F5F7F4F17
:10E070008F4F9F4F4AE0660F771F881F991F4A9561
:10E08000D1F7D0CF8BE0F801848360E070E0CB0162
:10E09000C9CF0895FC0182810895CF93DF93E09169
:10E0A000390687E1E89FF0011124E15CF94FC08552
:10E0B000D18581E0CE31D105C4F020E030E040E0F0
:10E0C0005FE364817581868197810F94083E0F9488
:10E0D000743F6C1B7D0B77FF03C0719561957109CF
:10E0E00081E0633071050CF080E0DF91CF910895FD
:10E0F000FC0190E1AFEAB7E001900D929A95E1F74B
:10E100000895BC012091A0073091A1074091A0077C
:10E110005091A1072417350731F481E026173707FE
:10E1200009F080E008959A01F1CFEF92FF920F93EA
:10E130001F93E0920306F0920406009305061093E5
:10E1400006066093070670930806809309069FEF02
:10E15000FF27621B730B840B30F4809570956195DB
:10E16000790B890B992790930E08A6E06A9F00927D
:10E170000208512DEE277A9F500DE11D8A9FE00D78
:10E1800050930308E0930408AFE06A9F00920608EA
:10E19000512DEE277A9F500DE11D8A9FE00D50937F
:10E1A0000708E0930808AAE06A9F00920A08512D28
:10E1B000EE277A9F500DE11D8A9FE00D50930B08CA
:10E1C000E0930C081F910F91FF90EF90089580E06D
:10E1D00008959F92AF92BF92CF92DF92EF92FF92FB
:10E1E0000F931F93CF93DF9300D01F921F92CDB751
:10E1F000DEB7EBEBF6E10027BB27462F572FA82F02
:10E20000AA2341F4A52F542FB85FAA2319F4A52FF0
:10E210005527B85FA03138F45295A295452F4F701D
:10E22000507FA42BBC5FA03428F4550FAA1F550FB4
:10E23000AA1FBE5FA03818F4550FAA1FB395550F3B
:10E24000AA1FEA0FF01F449151E0AA27B85081F1AC
:10E25000C8F0B0FF02C0440F551FB1FF04C0440F07
:10E26000551F440F551FB2FF06C052954295142FFB
:10E270001F70407F512BB3FF1BC0A52F542F442785
:10E280000C945871B195B0FF02C055954795B1FFF8
:10E2900004C05595479555954795B2FF05C05295D1
:10E2A000407F4295452B5F70B3FF02C0452F552735
:10E2B000DD24CC24BB24B2E0649FD018C108B00A8E
:10E2C000B00B749FC018B108B00B849FB018B1098F
:10E2D000659FC018B108B00B759FB018B109859F34
:10E2E000B0196A9FB018B1097A9FB0194D9DA12C41
:10E2F00099243327992722275D9DA00C911C301F5C
:10E30000901F201FAD9D900C311D901F201F4C9D14
:10E31000A00C911C301F901F201F5C9D900C311D84
:10E32000901F201FAC9D300D911D201F4B9D900C08
:10E33000311D901F201F5B9D300D911D201FAB9D37
:10E34000900D211D4B9F300D911D201F5B9F900D47
:10E35000211DAB9F200DB1E0BB24CC24DD24639FA5
:10E36000D018C108B00AB00B739FC018B108B00B29
:10E37000839FB018B109699FC018B108B00B799F8D
:10E38000B018B109899FB019629FB018B109729F86
:10E39000B019D61AC70AB80A20F0B1E03B0F901F97
:10E3A000201F1124792F632F90E0822F0F900F9060
:10E3B0000F900F900F90DF91CF911F910F91FF90D1
:10E3C000EF90DF90CF90BF90AF909F9008957F9295
:10E3D0008F929F92AF92BF92CF92DF92EF92FF9275
:10E3E0000F931F93CF93DF937090F105C6EBD5E0A9
:10E3F00092E2C92E92E0D92E26E2E22E22E0F22EFF
:10E4000009EE15E0772009F45EC0F8018080918064
:10E41000A280B38020E030E0A901C501B4010F94CF
:10E42000B139882309F44FC020E030E040E05FE3D9
:10E43000C501B4010F94173A9B01AC010F94173A30
:10E440002BED3FE049E450E40F94173A9B01AC01F7
:10E4500060E070E080E89FE30F94023F4B015C01B5
:10E4600089929992A992B992F601619171916F0185
:10E47000072E000C880B990B0F94B8392AE037ED62
:10E4800043E25CE30F94173AA50194010F94173A05
:10E49000F70161937193819391937F010C5F1F4FFB
:10E4A000F5E0CE3BDF0709F0ADCFDF91CF911F91B3
:10E4B0000F91FF90EF90DF90CF90BF90AF909F9023
:10E4C0008F907F900895812C912C80E8A82E8FE367
:10E4D000B82EC6CFFC01908193FB882780F993FF6B
:10E4E0000E94E770811102C081E0089580E00895E4
:10E4F000CF92DF92EF92FF920F931F93CF93DF9310
:10E50000E82FF0E0EF01CC0FDD1FCC0FDD1F461729
:10E5100039F0823009F049C0C12CD12C760117C0E6
:10E520008230D1F3A09151098A2F90E0DC01AA0F2B
:10E53000BB1FA80FB91FAE0FBF1FAA0FBB1FAA0F8B
:10E54000BB1FA259B94FCD90DD90ED90FC908F018B
:10E55000000F111F000F111FF801E059FB4E25910C
:10E56000359145915491C95CDD4FC701B6010F94B7
:10E57000083E6A837B838C839D83F801EC59FB4EB4
:10E580002591359145915491C701B6010F94083EEC
:10E590006E877F87888B998BDF91CF911F910F9129
:10E5A000FF90EF90DF90CF90089550E0DA01AA0F2E
:10E5B000BB1FA40FB51FAE0FBF1FAA0FBB1FAA0F13
:10E5C000BB1FA259B94F862F90E0BC01660F771F81
:10E5D000680F791FE60FF71FEE0FFF1FEE0FFF1FEB
:10E5E000E259F94F20813181428153816D917D91B2
:10E5F0008D919C910F94073E6B017C01C95CDD4FAE
:10E60000AC019B016A817B818C819D810F94083EC6
:10E610006A837B838C839D83A70196016E857F85AA
:10E6200088899989B3CFCF93DF93EC018D810E94C4
:10E63000CFDD60E08B81DF91CF910D945D18AF92BB
:10E64000BF92DF92EF92FF920F931F93CF93DF93CE
:10E6500000D000D0CDB7DEB77C01D62E122F032F0D
:10E66000B42EA52E0E9413730F942A1D1E821D82A4
:10E670008D2D80648983AA82BB820C831D838E01C9
:10E680000F5F1F4FCE010696D801E0E02D91F0E01C
:10E69000EE0FFF1FE227E656FC4DE491A817B907DD
:10E6A000A9F7EE0FE160EE83580186E0A80EB11CD9
:10E6B000F80181918F010E94C3DD0A151B05C1F786
:10E6C000FCE0DF1202C00E94C8DD10E00E94C8DD3D
:10E6D000F701868387FF04C01F3F11F01F5FF6CF4D
:10E6E00026960FB6F894DEBF0FBECDBFDF91CF9157
:10E6F0001F910F91FF90EF90DF90BF90AF90089522
:10E7000061E0FC0183810F945D188FEF0C94C3DDF1
:10E710000F931F93CF938C010E9413730F942A1DA4
:10E72000C82F882371F08DEF0E94C3DD0F942A1D3E
:10E73000C82FC8010E9480738C2FCF911F910F9119
:10E74000089582E1F8018483F4CF8F929F92AF9273
:10E75000BF92CF92DF92EF92FF920F931F93CF93CE
:10E76000DF93EC016A017B01590120E030E0A9014F
:10E7700067E30E941F73A501980167E1CE010E9423
:10E780001F73811127C08F81833039F089E0CC0C51
:10E79000DD1CEE1CFF1C8A95D1F7A701960169E1EB
:10E7A000CE010E941F7311E0882319F010E087E06A
:10E7B0008C83CE010E948073812FDF91CF911F91B6
:10E7C0000F91FF90EF90DF90CF90BF90AF909F9010
:10E7D0008F90089589E08C8310E0EBCFEF92FF9249
:10E7E0000F931F93CF93DF93EC01E62E8A0160E035
:10E7F00072E0CA010E94B06FF82E892FEEBCF801BA
:10E8000098013E5F0DB407FEFDCF90819EBD0DB413
:10E8100007FEFDCF91819EBD3296E217F30791F777
:10E820000DB407FEFDCF0E94C3DD8F2D0E94C3DD16
:10E830000E94C8DD8E838F71853069F083E18C83FF
:10E84000CE010E94807380E0DF91CF911F910F91E4
:10E85000FF90EF90089581E0F7CF0F931F93CF9330
:10E86000DF93EC018B010E9413730F942A1D811119
:10E870000CC085E18C8310E0CE010E948073812F53
:10E88000DF91CF911F910F910895A8016CEFCE01F8
:10E890000E94EE73182F882361F3EECF0F931F931E
:10E8A000CF93DF93EC0189018F81833039F089E0C8
:10E8B000440F551F661F771F8A95D1F79A01AB0148
:10E8C00068E1CE010E941F7381112AC0A8016EEF7A
:10E8D000CE010E94EE73182F8823B1F00F942A1DE9
:10E8E000182F8823D1F020E030E0A9016DE0CE019F
:10E8F0000E941F73882321F086E18C8310E004C0FE
:10E900000E94C8DD8111F8CFCE010E948073812F53
:10E91000DF91CF911F910F91089587E18C83F4CF00
:10E9200086E0EBCF1F93CF93DF93EC010E9413732C
:10E9300020E030E0A9016CE0CE010E941F7311E0DD
:10E94000882319F010E083E08C83CE010E9480734D
:10E95000812FDF91CF911F9108951F93CF93DF9364
:10E96000EC018F81833039F089E0440F551F661F19
:10E97000771F8A95D1F79A01AB0162E1CE010E941F
:10E980001F7311E0882319F010E085E08C83CE011D
:10E990000E948073812FDF91CF911F9108958F92F4
:10E9A0009F92AF92BF92CF92DF92FF920F931F93ED
:10E9B000CF93DF93EC018B016A010F941E1D4B0175
:10E9C0005C012CE2820E21E0921EA11CB11C0E946F
:10E9D000C8DD8E838F3F61F40F941E1D681979097D
:10E9E0008A099B0997FDF3CF81E18C8310E028C051
:10E9F0008E3F09F040C0C60101972FEF2EBDF801F0
:10EA00004FEF0DB407FEFDCF2EB521934EBD9F01F4
:10EA1000201B310B28173907A0F30DB407FEFDCFDB
:10EA20002EB5800F911FFC0120830E94C8DDF82EB7
:10EA30000E94C8DDB82E80915502811111C011E0ED
:10EA4000CE010E948073812FDF91CF911F910F9192
:10EA5000FF90DF90CF90BF90AF909F908F900895E0
:10EA6000B601C8010E94B06F3F2D2B2D821793076E
:10EA700031F38BE1BACF8FE0B8CF0F931F93CF93D1
:10EA8000DF93EC018B010E94137340E052E0B80168
:10EA9000CE01DF91CF911F910F910C94CF74AF9263
:10EAA000BF92CF92DF92EF92FF920F931F93CF937B
:10EAB000DF93EC016A017B0159018F81833039F0CA
:10EAC00089E0CC0CDD1CEE1CFF1C8A95D1F713E00D
:10EAD00004E0A701960161E1CE010E941F73882323
:10EAE00079F00C83CE010E9480731150E1F020E098
:10EAF00030E0A9016CE0CE010E941F731C82E9CFB7
:10EB000040E052E0B501CE010E94CF74882351F35A
:10EB1000DF91CF911F910F91FF90EF90DF90CF90F9
:10EB2000BF90AF90089580E0F3CF8F929F92AF9205
:10EB3000BF92CF92DF92EF92FF920F931F93CF93EA
:10EB4000DF93EC01162F1F821C824B830F941E1D36
:10EB50006B017C0120EDC20E27E0D21EE11CF11CEE
:10EB6000A89561E08B810F945D1861E08B810F9413
:10EB70002C1B209A289A219A2398229A81E00E949D
:10EB8000CFDD85E08D830E94CFDD0AE08FEF0E940C
:10EB9000C3DD0150D9F7A89520E030E0A90160E07D
:10EBA000CE010E941F738E83813081F00F941E1D51
:10EBB0006C197D098E099F0997FDEECF81E08C834A
:10EBC000CE010E9480731A8280E078C021E030E09C
:10EBD00040E050E06BE3CE010E941F7391E0813072
:10EBE00009F090E090935502A8952AEA31E040E0C0
:10EBF00050E068E0CE010E941F73853041F581E04E
:10EC00008F83A8958F81812C912C5401823029F417
:10EC1000812C912CA12C80E4B82E20E030E0A901B9
:10EC200067E3CE010E941F73A501940169E2CE0142
:10EC30000E941F738E838823F1F00F941E1D6C19A0
:10EC40007D098E099F0997FDE8CF8AE0B8CF04E0DF
:10EC50000E94C8DD8E830150D9F78A3A11F482E010
:10EC6000CFCF0F941E1D6C197D098E099F0997FD4A
:10EC7000BCCF82E0A4CF8F818230C1F420E030E0AD
:10EC8000A9016AE3CE010E941F73882311F088E076
:10EC900096CF0E94C8DD807C803C11F483E08F8396
:10ECA0000E94C8DD0E94C8DD0E94C8DDCE010E941E
:10ECB000807381E08A83173070F41D83DF91CF91D8
:10ECC0001F910F91FF90EF90DF90CF90BF90AF908A
:10ECD0009F908F90089588E18C8376CF0F931F9338
:10ECE000CF93DF93EC018B0120E030E0A90169E0D4
:10ECF0000E941F7381110AC040E150E0B801CE01AB
:10ED0000DF91CF911F910F910C94CF7480E18C8390
:10ED1000CE010E94807380E0DF91CF911F910F910F
:10ED200008950F930091020621E0022725E537E0C0
:10ED30004CE050E0BC0183E597E00E9461CE0F916A
:10ED400008950F930091020621E0022725E537E0A0
:10ED500041E050E0BC0183E597E00E9461CE0F9155
:10ED600008950F930091020621E0022725E537E080
:10ED700041E050E0BC0183E597E00E9461CE0F9135
:10ED800008950F930091020621E0022725E537E060
:10ED900048E050E0BC0183E597E00E9461CE0F910E
:10EDA00008950F930091020621E0022725E537E040
:10EDB0004CE050E0BC0183E597E00E9461CE0F91EA
:10EDC00008950F930091020621E0022725E537E020
:10EDD00044E050E0BC0183E597E00E9461CE0F91D2
:10EDE00008950F9301E025E537E041E050E0BC01D4
:10EDF00083E597E00E9461CE0F9108950F93AB01D8
:10EE00000091020621E0022725E537E0BC0183E5F9
:10EE100097E00E9461CE0F91089525E537E04CE020
:10EE200050E0BC0183E597E00C9494DA25E537E0E7
:10EE300041E050E0BC0183E597E00C9494DA25E5CD
:10EE400037E041E050E0BC0183E597E00C9494DAB0
:10EE500025E537E04CE050E0BC0183E597E00C94F9
:10EE600094DA25E537E044E050E0BC0183E597E023
:10EE70000C9494DACF93C82FCB010E94ACCE85E3DB
:10EE800094E10E94ACCE86E294E1CC2311F08BE2B7
:10EE900094E1CF910C9409DB2F923F924F925F92B5
:10EEA0006F927F928F929F92AF92BF92CF92DF929A
:10EEB000EF92FF920F931F93CF93DF93CDB7DEB7FF
:10EEC0006C970FB6F894DEBF0FBECDBF8C015B010F
:10EED0005A834983FC01E95BFF4F208031804280E7
:10EEE00053802D823E824F825886C201B1010F9419
:10EEF000B6396B017C01D5012D913D914D915C910D
:10EF00000F94173A0F94E63E2B013C01E981FA81F8
:10EF10002081318142815381C701B6010F94173A94
:10EF20000F94E63E4B015C01C301B2010F947B3F9D
:10EF30006D877E878F87988B68377105810591056E
:10EF400048F438E7232E312C412C512C2D863E8657
:10EF50004F86588AC501B4010F947B3F698B7A8B29
:10EF60008B8B9C8B683771058105910548F428E7E8
:10EF7000222E312C412C512C298A3A8A4B8A5C8AC8
:10EF8000F801ED5AFF4F80809180A280B380D801B4
:10EF900095962D903D904D905C90989729863A8655
:10EFA0004B865C86C501B4010F94B8396D8B7E8B9E
:10EFB0008F8B988F89288A288B2809F49CC1A701F8
:10EFC0009601C701B6010F94173A69837A838B8340
:10EFD0009C836D857E858F8598890F94B6399B01BA
:10EFE000AC010F94173A698F7A8F8B8F9C8F2D8984
:10EFF0003E894F89588D60E070E080E09FE30F9478
:10F00000023F4B015C01298D3A8D4B8D5C8D6981EE
:10F010007A818B819C810F94073EA50194010F9406
:10F02000173A6B017C010F94E63E0F947B3F1B0166
:10F030002C0169897A898B899C890F94B6399B0147
:10F04000AC010F94173A9B01AC0169817A818B81E5
:10F050009C810F94073EA50194010F94173A4B0130
:10F060005C010F94AA3F0F947B3F69837A838B8363
:10F070009C83DC01CB01820D931DA41DB51D298548
:10F080003A854B855C85281B390B4A0B5B0BDA01F3
:10F09000C901B7FF61C069857A858B859C850F940E
:10F0A000B639A70196010F94083EA50194010F946B
:10F0B000073E20E030E040E05FE30F94173A0F9402
:10F0C000E63E6B017C0120E030E0A9010F9468402E
:10F0D00018161CF0C12CD12C7601C701B6010F9473
:10F0E0007B3F1B012C0149855A856B857C85421528
:10F0F00053056405750510F41A012B0169857A859D
:10F100008B859C85621973098409950969837A83C3
:10F110008B839C83C201B1010F94B6396B017C01D2
:10F120002D893E894F89588DCA01B9010F94083E37
:10F130009B01AC01C701B6010F94173A298D3A8D96
:10F140004B8D5C8D0F94083E0F94B6400F947B3F1F
:10F150006D837E838F8398876D817E818F81988573
:10F160002D853E854F855889621B730B840B950B4B
:10F170000F94B6392D893E894F89588D0F94023FDF
:10F1800020E034E244EF59E40F94173A0F947B3FA8
:10F190006B017C016D817E818F81988529893A89F7
:10F1A0004B895C89621B730B840B950B0F94B639EA
:10F1B0002D893E894F89588D0F94023F20E034E21B
:10F1C00044EF59E40F94173A0F947B3F4B015C01D5
:10F1D0003FE6C316D104E104F10408F094C0F6013F
:10F1E000EE0FFF1FEE0FFF1FE150FB4E8591959133
:10F1F000A591B4913C01AD8BB9874FE6841691047B
:10F20000A104B10408F087C0F401EE0FFF1FEE0F58
:10F21000FF1FE150FB4E4591559165917491342F3C
:10F22000252FCB01D8019A962D923D924D925C925A
:10F230009D9795964D915D916D917C9198972980C0
:10F240003A804B805C8042195309640975099E9687
:10F250004D935D936D937C93D197F801E55BFF4FE0
:10F260002D843E844F84588820823182428253828A
:10F27000D696CD92DD92ED92FC92D997F80182AEAE
:10F2800093AEA4AEB5AEFE96608271822D882282C6
:10F2900039843382349630832183828393832D8013
:10F2A0003E804F805884D2962D923D924D925C9232
:10F2B000D5973D9629883A884B885C882082318290
:10F2C000428253826C960FB6F894DEBF0FBECDBF5C
:10F2D000DF91CF911F910F91FF90EF90DF90CF9032
:10F2E000BF90AF909F908F907F906F905F904F9066
:10F2F0003F902F90089519821A821B821C82212C24
:10F30000312C210129CFC701B6010E94E9703B01D0
:10F310008D8B998772CFC501B4010E94E970362F99
:10F32000272F80CF8091A21784FF04C08460877F3D
:10F330008093A2170895CF92DF92EF92FF920F93DE
:10F340001F93CF93DF93CDB7DEB7EDB6FEB6DC01EA
:10F350000D900020E9F79D01281B390B285F3F4FD6
:10F36000EDB7FEB7E21BF30B0FB6F894FEBF0FBE6E
:10F37000EDBF0DB71EB70F5F1F4F9F938F9380E1B7
:10F3800097E29F938F931F930F930F9448396801CF
:10F39000F4E0CF0ED11C0F900F900F900F900F90B4
:10F3A0000F90D6018D916D01882349F0082E000C35
:10F3B000990B0F94B141F60131978083F2CF6BE046
:10F3C00077E2C8010F94E838C8010E94E12B0FB61C
:10F3D000F894FEBE0FBEEDBEDF91CF911F910F914D
:10F3E000FF90EF90DF90CF900895FC01938591FFFF
:10F3F00002C080E00895987121E0903109F020E08A
:10F400008091A21720FB85F98093A217903141F0DB
:10F410008085873471F781E091859E3751F3089597
:10F4200081E0FDCFFC0120E03EE2DB014D91BD011A
:10F43000403249F0283011F430833196DB011197C6
:10F440004C91408331962F5F2B3079F710820895CD
:10F45000CF9380914D14C1E08823C9F080914E1460
:10F4600090914F1440914514509146146091471467
:10F4700070914814DC01ED91FC910288F389E02D34
:10F4800025E432E11995C82F811104C0C0E08C2F0A
:10F49000CF9108954091491450914A1460914B14B2
:10F4A00070914C144115510561057105B9F08091B9
:10F4B0004E1490914F14DC01ED91FC910288F38978
:10F4C000E02D25E432E11995882301F310924914C7
:10F4D00010924A1410924B1410924C1410924D1426
:10F4E000D6CFCF92DF92EF92FF92CF936B017C0148
:10F4F000C42F8091451490914614A0914714B09167
:10F5000048148C159D05AE05BF0529F10E94287A87
:10F51000811108C0C0E08C2FCF91FF90EF90DF9059
:10F52000CF90089580914E1490914F14DC01ED918D
:10F53000FC910088F189E02D25E432E1B701A601B4
:10F540001995882339F3C0924514D0924614E0925D
:10F550004714F0924814CC2321F081E080934D149D
:10F56000DACFC1E0D8CF4F925F926F927F928F92A5
:10F570009F92AF92BF92CF92DF92EF92FF920F9342
:10F580001F93CF93DF93EC01423051056105710564
:10F5900090F480E0DF91CF911F910F91FF90EF9059
:10F5A000DF90CF90BF90AF909F908F907F906F90A3
:10F5B0005F904F90089589859A85AB85BC850196AB
:10F5C000A11DB11D84179507A607B70710F38F89F2
:10F5D0008031C9F5852E962EA72EBB248B899C8958
:10F5E000AD89BE89880E991EAA1EBB1E280139014D
:10F5F0006A017B0141E0C501B4010E94717A882350
:10F6000041F29F89903181F5DD24EE24FF24F6013B
:10F61000EE0FFF1FEB5BFD4E118300839A89923042
:10F6200008F4B8CF4D815E816F817885840E951E78
:10F63000A61EB71E8092491490924A14A0924B14B1
:10F64000B0924C14A7CF803209F0A3CF8B899C894C
:10F65000AD89BE894A015B01E7E0B694A79497940F
:10F660008794EA95D1F7BECFE894C7F8DD24EE245D
:10F67000FF24F601EE0FFF1FEE0FFF1FEB5BFD4EA9
:10F680004082518262827382C9CFCF92DF92EF9221
:10F69000FF920F931F93CF93DF93FC018185928597
:10F6A000A385B4850196A11DB11D84179507A607F2
:10F6B000B70750F480E0DF91CF911F910F91FF9039
:10F6C000EF90DF90CF90089587898031A9F5BB270F
:10F6D000A72F962F852FC388D488E588F6888C0DB0
:10F6E0009D1DAE1DBF1DE9016A017B018F01409187
:10F6F0004514509146146091471470914814841732
:10F700009507A607B70749F5F8018789803169F59C
:10F71000B701A601552766277727440F551F4B5B76
:10F720005D4EFA0180819181B0E0A0E088839983E9
:10F73000AA83BB8381E0BFCF803209F0BBCFC388EF
:10F74000D488E588F688DB01CA01C7E0B695A7959D
:10F7500097958795CA95D1F7C2CF40E0BC01CD01FE
:10F760000E94717A8111D0CFA5CFB701A6014F7742
:10F77000552766277727440F551F440F551F4B5BAE
:10F780005D4EFA0180819181A281B381BF70CECF9D
:10F790004F925F926F927F92AF92BF92CF92DF9221
:10F7A000EF92FF920F931F93CF93DF9300D01F929E
:10F7B000CDB7DEB78C0149835A836B837C835901B3
:10F7C000C12CD12C7601412C82E0582E612C712C59
:10F7D00049815A816B817C819E012F5F3F4FC80117
:10F7E0000E94457B882319F1F8018585A3019201C8
:10F7F00004C0220F331F441F551F8A95D2F7DA0128
:10F80000C901C80ED91EEA1EFB1E49815A816B81AF
:10F810007C8187898031F1F481E0483F5F4F610549
:10F820007105B0F2F501C082D182E282F3820F90BD
:10F830000F900F900F90DF91CF911F910F91FF903C
:10F84000EF90DF90CF90BF90AF907F906F905F90E0
:10F850004F90089581E0483F5F4F6F4F7F4008F41D
:10F86000B7CFE0CF0F931F93CF93DF93FC0123819A
:10F87000222331F080E0DF91CF911F910F91089505
:10F880008B01EC01FB018789803139F582E08B83A4
:10F890001D8A1E8A1F8A188E808D918DB0E0A0E08F
:10F8A00025E0880F991FAA1FBB1F2A95D1F7898BC6
:10F8B0009A8BAB8BBC8B1A8F098F81E0898318865A
:10F8C00019861A861B861C821D821E821F82188A38
:10F8D0001C861D861E861F86CECF803259F683E099
:10F8E0008B83428D538D648D758D4D8B5E8B6F8BAD
:10F8F000788F9E012F5E3F4FC8010E94C87B811107
:10F90000DACFB8CF8F929F92AF92BF92CF92DF9211
:10F91000EF92FF920F931F93CF93DF93EC018B81B4
:10F9200081110EC080E0DF91CF911F910F91FF9068
:10F93000EF90DF90CF90BF90AF909F908F90089501
:10F9400009891A892B893C89041715072607370767
:10F9500048F34A015B01823031F488869986AA8691
:10F96000BB8681E0E0CF81149104A104B10449F485
:10F97000188619861A861B861C821D821E821F828B
:10F98000F0CF088519852A853B85E98DFA8D858517
:10F9900090E00996B901A801415051096109710926
:10F9A000082E04C076956795579547950A94D2F727
:10F9B00075016401E1E0CE1AD108E108F10804C044
:10F9C000F694E794D794C7948A95D2F7C416D506CF
:10F9D000E606F70620F0012B022B032B11F58D898B
:10F9E0009E89AF89B88D8C839D83AE83BF838E0142
:10F9F0000C5F1F4FC114D104E104F10409F4ADCF31
:10FA00004C815D816E817F819801898D9A8D0E94E4
:10FA1000457B91E0C91AD108E108F1088111EACFCC
:10FA200081CFC41AD50AE60AF70AE1CF2F923F9296
:10FA30004F925F926F927F928F929F92AF92BF92FE
:10FA4000CF92DF92EF92FF920F931F93CF93DF93AA
:10FA5000EC014B017A018B81811115C08FEF9FEF73
:10FA6000DF91CF911F910F91FF90EF90DF90CF909A
:10FA7000BF90AF909F908F907F906F905F904F90CE
:10FA80003F902F900895898180FFE8CF89899A89D6
:10FA9000AB89BC89488559856A857B85841B950B14
:10FAA000A60BB70BA70170E060E084179507A607C7
:10FAB000B70708F47C0167011E0124E0220E311C07
:10FAC000C114D10409F4A9C0488559856A857B858C
:10FAD0005A0181E0B822898D9A8D2A013B0129E0E3
:10FAE00076946794579447942A95D1F72B81FC011B
:10FAF000223081F5628D738D848D958D640D751D19
:10FB0000861D971D00E012E00A191B09C016D106D8
:10FB100008F486010115E2E01E0771F440904514D7
:10FB20005090461460904714709048146415750501
:10FB30008605970509F04EC040E00E94717A88233F
:10FB400009F48CCFB5016B5B7D4EA801C4010F9405
:10FB5000C64152C0148111501421A114B10471F492
:10FB600011110CC0452B462B472B51F58D899E89D1
:10FB7000AF89B88D8C839D83AE83BF83E98DFA8D69
:10FB80004C805D806E807F8022E0421A51086108BF
:10FB90007108858504C0440C551C661C771C8A9529
:10FBA000D2F786859785A089B189480E591E6A1EAD
:10FBB0007B1EC301B201610F711D811D911DA2CF7A
:10FBC0004C815D816E817F8191010E94457B811115
:10FBD000D5CF44CFA0914E14B0914F14ED91FC912C
:10FBE00011970088F189E02D9401AB01BC01CD0192
:10FBF0001995882309F432CF800E911E8885998546
:10FC0000AA85BB85800F911FA11DB11D888799878B
:10FC1000AA87BB87C01AD10A53CFC70121CFCF9380
:10FC2000DF93EC01462F41706C857D858E859F8525
:10FC30000E94717A882351F0888920E2829FC00156
:10FC400011248B5B9D4EDF91CF91089590E080E071
:10FC5000FACFCF93DF93EC018B81882349F189811F
:10FC600087FF22C061E0CE010E940F7EFC01892B3C
:10FC7000F9F08081853EE1F08B81823040F4898902
:10FC80009A89AB89BC89848F958FA68FB78F8D8910
:10FC90009E89938F828F8D899E89AF89B88DB58B10
:10FCA000A48B89818F778983DF91CF910C94287AF7
:10FCB00081E0888380E0DF91CF910895CF93DF9337
:10FCC000EC010E94297E1B82DF91CF910895109252
:10FCD0009A068091A2178F778093A2170E9473CD06
:10FCE000882321F080E594E10C945E7E0895CF9303
:10FCF000C091A217C2FF10C0C7FD0EC00E9473CDF5
:10FD000080FBC7F9C093A2178091A2178F7E8064F1
:10FD10008093A217CF9108950E94677EF5CFCF936D
:10FD2000DF938091A2178F7E8093A2178091A714F2
:10FD3000882321F084EA94E10E945E7E8091A317DB
:10FD40009091A417DC01ED91FC910190F081E02DE0
:10FD500045E360E01995811112C00E940FD88FEF22
:10FD600096E20E94ACCE8091A21784FF34C00F941B
:10FD7000022783E080937502DF91CF910895C091AF
:10FD8000A317D091A41761E0CE010F94DA0A811174
:10FD90000BC060E0CE010F94DA0A811105C00E9409
:10FDA0000BD88BEE96E2DDCF6BE674E184EA94E14A
:10FDB0000E94327C811105C00E940BD88AED96E228
:10FDC000D0CF8091A21780618093A2170E940FD894
:10FDD0008EEC96E2C6CF80913509882351F261E01E
:10FDE0008EEB96E20E941D3B0E945E2DC2CFCF9308
:10FDF000DF93EB01FC012381211104C080E0DF913E
:10FE0000CF9108952250223028F48FE288831982FE
:10FE100081E0F5CF60E00E940F7E009779F3DC016E
:10FE200060E080E09EE22D91203299F0883031F43C
:10FE30009E01260F311DF90190836F5F9E01260FF1
:10FE4000311DAD0141505109FA014081F901408352
:10FE50006F5F8F5F8B3039F7FE01E60FF11D108267
:10FE6000D7CFCF93DF93EC01CB01E881F98160819B
:10FE700071810E94F77E28813981D901ED91FC9131
:10FE8000AA81BB818C919081992359F08936C8F45D
:10FE9000CF010196F901918380838C918F5F8C93C0
:10FEA000EACF893670F48FE28083E881F98180811E
:10FEB0009181019691838083EA81FB8180818F5FAC
:10FEC0008083DF91CF9108953F924F925F926F921E
:10FED0007F928F929F92AF92BF92CF92DF92EF92DA
:10FEE000FF920F931F93CF93DF93CDB7DEB72C977D
:10FEF0000FB6F894DEBF0FBECDBF5C01DC01599692
:10FF00008D909C90F40181859285A385B4859C0198
:10FF1000AD012F5F3F4F4F4F5F4F29873A874B8788
:10FF20005C87D50114964D905D906D907C901797ED
:10FF3000411451046104710409F459C0BFEF4B1A14
:10FF40005B0A6B0A7B0A312C730162011D821E82DF
:10FF50001F821886F40181859285A385B4852D8141
:10FF60003E814F815885281739074A075B0708F0FB
:10FF700056C089859A85AB85BC858C159D05AE05D7
:10FF8000BF0550F482E0C82ED12CE12CF12C92E078
:10FF9000492E512C612C712C9E012F5F3F4FB701D0
:10FFA000A601C4010E94457B8823C9F189819A81F9
:10FFB000AB81BC81892B8A2B8B2B01F12601370168
:10FFC0009FEF491A590A690A790A2D813E814F81AA
:10FFD00058852F5F3F4F4F4F5F4F2D833E834F8399
:10FFE00058873FEFC31AD30AE30AF30AB3CF40801E
:10FFF00051806280738033243394A6CFC414D50417
:020000021000EC
:10000000E604F70411F70FEF1FEF2FEF3FE0B70102
:10001000A601C4010E94B37A782E81111AC0712CF6
:10002000872D2C960FB6F894DEBF0FBECDBFDF91A3
:10003000CF911F910F91FF90EF90DF90CF90BF90E5
:10004000AF909F908F907F906F905F904F903F9078
:100050000895F501448155816681778141155105E7
:100060006105710539F097018601C4010E94B37AD8
:100070008823A9F2D5011496CD92DD92ED92FC92DF
:100080001797332051F0D701C6010196A11DB11D6C
:10009000F40180839183A283B383F50185899689D6
:1000A000A789B08D892B8A2B8B2B09F0B9CFC58AF4
:1000B000D68AE78AF08E818180688183B1CF40E063
:1000C00050E0BA010C94827CFC01238121110C9434
:1000D0005E7E08952F923F924F925F926F927F9231
:1000E0008F929F92AF92BF92CF92DF92EF92FF9248
:1000F0000F931F93CF93DF93CDB7DEB7C454D109CD
:100100000FB6F894DEBF0FBECDBF7C014B015A0184
:10011000222E19821C821C8E1F8E6115710511F40E
:1001200010E0B3C1DC0113968C918111F9CFFA0173
:1001300080818B018F32D1F4DB0113968C91139760
:100140008250823060F059966D917C91CE014C9630
:100150000E94327C8E01045E1F4F882309F3C50183
:100160005C010196F50120812F32D1F39E012F5FB2
:100170003F4F6901290130E2332E2496CFAE2497F8
:100180002596DFAE25973E013CE1630E711C229659
:100190003FAE229721963FAE21973FAE3EAE3DAE99
:1001A0003CAE3BAE3AAE39AE38AE3FAA950190E0D8
:1001B00047E0D9018D91882361F18F3251F18E3260
:1001C00039F44A3009F4ACCF98E04AE09D01F1CF10
:1001D000EAE9F6E22491222321F031968213FACF44
:1001E0009FCF491708F49CCF813208F499CF8F37FD
:1001F00009F496CF3FE9380F3A3108F420EEE7E3EF
:10020000F0E0EC0FFD1FE90FF11D820F80839F5F6F
:10021000DDCF8FA9803209F483CF5901D9018C91A8
:100220002F5F3F4F8F32C9F38823A9F008151905B6
:1002300019F0C8010E945E7E24969FAD24972596F2
:100240008FAD25974C145D0411F4962D872D8601F2
:10025000C92ED82E9CCFF801818D928DD7015A9648
:100260009C938E935997C8010E945F80C12CF8011E
:1002700080859185A285B385418952896389748976
:1002800084179507A607B70708F053C025E0B69571
:10029000A795979587952A95D1F7F82FFF70DF2EB0
:1002A000D80113968C91823008F43ACF41E050E0A7
:1002B000BE016E5B7F4FC8010E94167D019709F059
:1002C0002FCFF80180859185A285B3854F96A11D1A
:1002D000B11D80879187A287B387F0E2DF9EB001CE
:1002E00011246B5B7D4E6115710509F419CFDB019B
:1002F0008C91882341F0853E09F04DC0CC2029F037
:10030000CC24C394B4CFC1100EC0809145149091F9
:100310004614A0914714B0914814F701848795873B
:10032000A687B787D08ADB018C918111E9CFCC24D5
:10033000C394822D8274823409F0F2CECC2009F469
:10034000C7C0F701D08861E0C7010E940F7E009707
:1003500009F4E6CE20E2DC011D922A95E9F72BE0B4
:10036000FE01F796DC0101900D922A95E1F721E25A
:1003700038E2FC01318B208B40E058E057874687FC
:10038000338B228B318F208F578B468B0E94287A9C
:1003900081110AC0C5CE4BE050E0CE01C7960F9444
:1003A000B941892B09F063CF2D2D30E0F901B5E07B
:1003B000EE0FFF1FBA95E1F7DF01AB5BBD4E1B9659
:1003C0008C91817121F0822D827109F020C1D701B9
:1003D00059968D919C915A9740914514509146148D
:1003E00060914714709148141C964D935D936D93E2
:1003F0007C931F975096DC925097EB5BFD4E848860
:100400009588B12CA12C54019924882455968D925D
:100410009D92AD92BC925897428D538D70E060E0F2
:10042000482959296A297B2955964D935D936D93E7
:100430007C935897A5E0220F331FAA95E1F7D901C5
:10044000AB5BBD4E1B962C91287109F0D2C0848DF8
:10045000958DA68DB78DF701818B928BA38BB48B75
:1004600081E08383822D8F70F7018183148215824E
:1004700016821782108611861286138611E024FEDA
:1004800004C0C7010F94290C182FCE014C960E946E
:100490006480CE0101960E946480812FCC5BDF4F87
:1004A0000FB6F894DEBF0FBECDBFDF91CF911F9185
:1004B0000F91FF90EF90DF90CF90BF90AF909F9003
:1004C0008F907F906F905F904F903F902F90089506
:1004D000D80113968C911397823009F421CE51964E
:1004E0008D919D910D90BC91A02D803E9F4FAF416D
:1004F000B10508F015CEC8010E94647F882309F475
:100500000FCE0E94287A882309F40ACED801599682
:10051000ED91FC915A9714968D909D90AD90BC9062
:100520001797B2E08B1A9108A108B108858504C01D
:10053000880C991CAA1CBB1C8A95D2F786859785C6
:10054000A089B189880E991EAA1EBB1E81E08093E6
:100550004D148092451490924614A0924714B09284
:100560004814E5E4F2E180E092E0DF019C011D9295
:1005700021503040E1F7DD24D394D8015996ED9114
:10058000FC918481D816C0F480914E1490914F1440
:10059000DC01ED91FC910288F389E02D25E432E144
:1005A000B501A4014D0D511D611D711D19958823C3
:1005B00009F4B6CDD394E1CF258580E092E0A0E0A8
:1005C000B0E004C0880F991FAA1FBB1F2A95D2F75D
:1005D000F8014189528963897489840F951FA61F88
:1005E000B71F818B928BA38BB48B85E492E1D12CC6
:1005F000B1CE203161F497012F5E3F4F0E94C87B3E
:10060000882329F084E0D70113968C932BCFD70150
:1006100013961C9285CD0F931F93CF93DF93CDB785
:10062000DEB7EB970FB6F894DEBF0FBECDBF8C01DF
:1006300089E894E10E945F808BE1E9E8F4E1DE0162
:10064000919601900D928A95E1F7BE016F5F7F4F01
:10065000CE0181960F946C0E1816A4F4CE0101966B
:100660000E94F579882389F3BE016F5F7F4F89E788
:100670009FE00E94127A69E77FE0C8010F94CF41A2
:10068000892B19F7CE0181960E946480EB960FB6F4
:10069000F894DEBF0FBECDBFDF91CF911F910F91B8
:1006A00008958F929F92AF92BF92CF92DF92EF9276
:1006B000FF920F931F93CF93DF93DC0170E0FB0158
:1006C000EE0FFF1FEF5BFC4F20813181615C7C4F9F
:1006D000FB019081D92E80E0E82EF12CB7016D0D41
:1006E000711D75956795611119C0F9013296659173
:1006F0007491072E000C880B990B0F94B839DF9179
:10070000CF911F910F91FF90EF90DF90CF90BF900E
:10071000AF909F908F900895D62EE0CF681711F07C
:10072000D6120CC0492F4150550BFA01EE0FFF1F96
:10073000EE0FFF1F3296E20FF31FD9CFAB014150EE
:100740005109440F551F440F551FF901E40FF51FC0
:1007500005911491FA013496E20FF31FC591D491DB
:10076000A017B107C8F2862FCA17DB0708F4B4CF69
:10077000FA013296E20FF31FE590F490FA013696F3
:10078000E20FF31FC590D490A01BB10BBD0190E008
:1007900080E00F94B6394B015C01B6016E197F09F8
:1007A000072E000C880B990B0F94B8399B01AC01F4
:1007B000C501B4010F94173A4B015C01C01BD10B6A
:1007C000BE0190E080E00F94B6399B01AC01C501F9
:1007D000B4010F94023F4B015C01B701FF0C880B81
:1007E000990B0F94B8399B01AC01C501B4010F946A
:1007F000083E85CF8F929F92AF92BF92CF92DF92A9
:10080000EF92FF92CF936B017C01C42F20E030E088
:10081000A9010F94B13987FF07C08DE20E949FCED6
:10082000F7FAF094F7F8F0942BE037ED43EA5BE346
:10083000C23021F02FE632E143E05AE3C701B601AE
:100840000F94083E6B017C010F947B3F4B015C01D0
:100850000F94B6399B01AC01C701B6010F94073E56
:100860006B017C01C501B4010F94C00D8EE20E94A2
:100870009FCEC150E8F020E030E040E251E4C701F3
:10088000B6010F94173A6B017C010F947B3F4B012B
:100890005C010F94C00DC501B4010F94B6399B01E2
:1008A000AC01C701B6010F94073E6B017C01E1CF9B
:1008B000CF91FF90EF90DF90CF90BF90AF909F903F
:1008C0008F900895EF92FF920F931F93CF93DF9332
:1008D000C82F7B018A01D2E48F3F09F0D4E580E282
:1008E0000E949FCE8D2F0E949FCEC7FD04C080E343
:1008F0008C0F0E949FCE8AE30E949FCEF7016081F9
:1009000071818281938142E00E94FA8387E693E2BB
:100910000E94ACCEF801608171818281938142E0B6
:100920000E94FA8362E070E080E090E0DF91CF9176
:100930001F910F91FF90EF900D94911CEF92FF92F9
:100940000F931F93CF93DF9300D000D01F921F927D
:10095000CDB7DEB7082F17E1189FC00111249C0105
:10096000215C394F7901F90160857185072E000CF2
:10097000880B990B0F94B8396D837E838F8398878A
:10098000F70184819581A681B78189839A83AB839E
:10099000BC83AE014B5F5F4FBE016F5F7F4F80E84E
:1009A0000E9462846091360670913706072E000C13
:1009B000880B990B0F94B8396D837E838F8398874A
:1009C0008091320690913306A0913406B09135069D
:1009D00089839A83AB83BC83AE014B5F5F4FBE01BB
:1009E0006F5F7F4F8FEF0E94628460914706709126
:1009F0004806072E000C880B990B0F94B8396D83AD
:100A00007E838F8398878091430690914406A091BE
:100A10004506B091460689839A83AB83BC83AE01B9
:100A20004B5F5F4FBE016F5F7F4F80E00E9462842B
:100A300060915E0670915F06072E000C880B990B83
:100A40000F94B8396D837E838F83988780915A067F
:100A500090915B06A0915C06B0915D0689839A83B4
:100A6000AB83BC83AE014B5F5F4FBE016F5F7F4FB7
:100A700081E00E946284609138060F3F31F00103EB
:100A8000F0011124E15CF94F628570E082E793E2A6
:100A90000E9487DA6091380670E08DE693E20E944A
:100AA00087DA60E08AE693E20E94A2D68AE30E9497
:100AB0009FCE6091490670E090E080E00F942A0E8E
:100AC00061E08AE693E20E94A2D68AE30E949FCE6A
:100AD0006091600670E090E080E00F942A0E289606
:100AE0000FB6F894DEBF0FBECDBFDF91CF911F913F
:100AF0000F91FF90EF9008950F930FB70F93009110
:100B00006E000D7F00936E0078940F930BB70F93D8
:100B10000CB70F921F922F933F934F935F936F9356
:100B20007F938F939F93AF93BF93EF93FF93112482
:100B30000E94CB95FF91EF91BF91AF919F918F91C3
:100B40007F916F915F914F913F912F911F900F90E7
:100B50000CBF0F910BBF0F910260F89400936E00D1
:100B60000F910FBF0F911895EF92FF920F931F9364
:100B7000CF93DF9310926D0660E090E080E00E94DA
:100B8000DCCCCFE3D6E01A8661E090E080E00E9402
:100B9000DCCC19A22C9802E011E0F8018081807170
:100BA000C0E0D1E088838EE2E82E86E0F82EF701DF
:100BB000118610860E9422C6F7011286F8018081F4
:100BC00080728883DF91CF911F910F91FF90EF90FA
:100BD00008958F929F92AF92BF92CF92DF92EF9241
:100BE000FF920F931F93CF93DF93B0E4A0E06A2F9F
:100BF00070E0AB014B0F511D55954795411119C040
:100C0000E1EDF8E365917491072E000C880B990BC8
:100C10000F94B839DF91CF911F910F91FF90EF9012
:100C2000DF90CF90BF90AF909F908F900895B42F9A
:100C3000E0CFA41711F0B41303C0EDECF9E3E2CF59
:100C40009A0121503109220F331F220F331FF9015E
:100C5000E153F74CE590F490F901ED52F74CC59152
:100C6000D4918E159F0518F3A42FC817D90708F43F
:100C7000BECFF901EF52F74C05911491F901EB52F7
:100C8000F74CC590D4908E199F09BC0190E080E08C
:100C90000F94B6394B015C01B601601B710B072E36
:100CA000000C880B990B0F94B8399B01AC01C5015E
:100CB000B4010F94173A4B015C01CE19DF09BE0154
:100CC00090E080E00F94B6399B01AC01C501B401FE
:100CD0000F94023F6B017C01B801110F880B990B37
:100CE0000F94B8399B01AC01C701B6010F94083EBF
:100CF00091CF80910B06882339F060918316709113
:100D0000841680918516089560E070E080E0089573
:100D10002F923F924F925F926F927F928F929F920B
:100D2000AF92BF92CF92DF92EF92FF920F931F93F9
:100D3000CF93DF93CDB7DEB765970FB6F894DEBFDC
:100D40000FBECDBF8F836B8B20916D062E871092C7
:100D50006D0637E1839FF0011124E15CF94F848136
:100D60009581A681B7818F87988BA98BBA8B1092BA
:100D70003A0681E080937402212C312C21011B82E0
:100D80001C821D821E821A869CE39B87ACE1AC8785
:100D9000B6E4BD87612C10E000E82FEB2A831982AE
:100DA000AF01485F5F4F59874887CF0104969D8BFD
:100DB0008C8BA885B9856D917C91072E000C880BD2
:100DC000990B0F94B8396B017C01262D312F402FE0
:100DD0005A810F94B1398823A9F0EC89FD892081CB
:100DE000318142815381FB89B601C701F1117DC078
:100DF0000F94B139881F8827881F89836C2C1D2D7B
:100E00000E2DFA820F941E1D6B017C01DC01CB01BB
:100E10002B813C814D815E81821B930BA40BB50B12
:100E2000B7FD10C0D701C60188519C4FAF4FBF4FCF
:100E30008B839C83AD83BE838F810E949E848AE0D6
:100E40000E949FCE80E00E94EADD0F941E1D6093F9
:100E50003B0670933C0680933D0690933E06AC891A
:100E6000BD89AC9011969C90119712968C90129718
:100E700013967C90B981B1116FC0662D712F802FB0
:100E80009A810F94743F6B016A2D792D882D972DCF
:100E90000F94743F4B016F85788989899A890F94E3
:100EA000743FCB01A601B4010E949DCB80917402D6
:100EB0008823F9F0A885B9856D917C91072E000CE7
:100EC000880B990B0F94B8399B01AC01EC89FD8913
:100ED0006081718182819381F981FF23C1F10F9437
:100EE000684018160CF465CF04C00F94B13987FF21
:100EF00028C0209174022983222331F010927402B9
:100F00000F948E100E944B272E8520936D068981A9
:100F100065960FB6F894DEBF0FBECDBFDF91CF91BF
:100F20001F910F91FF90EF90DF90CF90BF90AF9007
:100F30009F908F907F906F905F904F903F902F90F9
:100F400008956C2C1D2D0E2DFA8219825BCF0F9403
:100F5000B13987FD2ECFCDCF211431044104510486
:100F600041F0D701C60182199309A409B509B7FD5B
:100F70009DCF2A2D392D482D572D6A857B858C854F
:100F80009D850F94073E20E030E040EC5FE30F9436
:100F9000B13987FDAECF16012701E0E62E0EEAEE4D
:100FA0003E1E411C511CAA869B868C867D867ECF68
:100FB00012988D5F21E030E001C0220F8A95EAF798
:100FC0008091BF07822B8093BF070895CF92DF9255
:100FD000EF92FF92CF93DF93EC01C880D980EA8033
:100FE000FB8083EB92E20E94ACCEC701B6010F9466
:100FF0002A0ECC80DD80EE80FF8083E49CE30E949B
:10100000ACCEC701B6010F942A0EC884D984EA84F5
:10101000FB848FE39CE30E94ACCEC701B6010F9422
:101020002A0E8AE0DF91CF91FF90EF90DF90CF9072
:101030000C949FCE0F930FB70F9300916E000F93F8
:101040000D7F00936E0000916F000D7F00936F0085
:101050000F930BB70F930CB70F921F922F933F93E1
:101060004F935F936F937F938F939F93AF93BF93B0
:10107000EF93FF9311240E9418A8FF91EF91BF9165
:10108000AF919F918F917F916F915F914F913F9120
:101090002F911F900F900CBF0F910BBF0F9102600B
:1010A000F89400936F000F9100936E000F910FBFA3
:1010B0000F91189500008091E50880FF27C0899A5C
:1010C0008FEF809358078091E50881FF22C08F9AA7
:1010D0008FEF809359078091E50882FF1DC08091B2
:1010E0000B0180958270809309018FEF80935A07DE
:1010F00080915C079091E50893FF17C0811113C0A0
:10110000169A8FEF80935B0700000895899881E01D
:10111000D8CF8F9881E0DDCF80910B0182708093D2
:10112000090181E0E3CF4398ECCF811103C0169809
:1011300081E0E8CF439AFCCFAF92BF92CF92DF928B
:10114000EF92FF921F93CF93DF9340EC50E070E05B
:1011500060E08FEA95E10F94CE218FEAA82E85E119
:10116000B82E11E0F50113AF43E051E860E070E103
:10117000C5010F940222C0E2D3E0F501D2AFC1AFA6
:10118000C12CD12CE12C9FE3F92EC586D686E786AB
:10119000F08A60E273E0C5010F940F2164E0C5019D
:1011A0000F942E09C5010F94E61160E8C5010F9454
:1011B000C72044E25EE06DE078ECC5010F94B221F7
:1011C000C5010F94DA1168EC70E080E090E00F94B4
:1011D000911C40EC50E070E060E083E795E10F94F3
:1011E000CE2123E7A22E25E1B22EF50113AF43E075
:1011F00051E860E070E1C5010F940222F501D2AF21
:10120000C1AFC586D686E786F08A60E273E0C50185
:101210000F940F2164E0C5010F942E09C5010F94AE
:10122000E61160E8C5010F94C72044E25EE06DE07E
:1012300078ECC5010F94B221C5010F94DA1168EC66
:1012400070E080E090E00F94911C40EC50E070E082
:1012500060E087E395E10F94CE2137E3A32E35E1DB
:10126000B32EF50113AF43E051E860E070E1C50132
:101270000F940222F501D2AFC1AFC586D686E786AC
:10128000F08A60E273E0C5010F940F2164E0C501AC
:101290000F942E09C5010F94E61160E8C5010F9463
:1012A000C72044E25EE06DE078ECC5010F94B22106
:1012B000C5010F94DA1168EC70E080E090E00F94C3
:1012C000911C40EC50E070E060E08BEF94E10F94F3
:1012D000CE214BEFA42E44E1B42EF50113AF43E031
:1012E00051E860E070E1C5010F940222F501D2AF30
:1012F000C1AFC586D686E786F08A60E273E0C50195
:101300000F940F2164E0C5010F942E09C5010F94BD
:10131000E61160E8C5010F94C72044E25EE06DE08D
:1013200078ECC5010F94B221C5010F94DA1168EC75
:1013300070E080E090E00F94911C40EC50E070E091
:1013400060E08FEB94E10F94CE215FEBA52E54E18A
:10135000B52EF50113AF43E051E860E070E1C5013F
:101360000F940222F501D2AFC1AFC586D686E786BB
:10137000F08A60E273E0C5010F940F2164E0C501BB
:101380000F942E09C5010F94E61160E8C5010F9472
:10139000C72044E25EE06DE078ECC5010F94B22115
:1013A000C5010F94DA1168EC70E080E090E00F94D2
:1013B000911CDF91CF911F91FF90EF90DF90CF9024
:1013C000BF90AF900C945A8893E0980F21E030E0E2
:1013D00002C0220F331F9A95E2F720953095909125
:1013E000BF0729232093BF07882321F0813021F0F4
:1013F00081E00895129AFCCF479AFACF80E00E94CC
:10140000E48981E00C94E489882319F0813021F08B
:10141000089580E00C94D88747988091BF07806139
:101420008093BF070895813089F070F0823081F099
:1014300021E030E001C0220F8A95EAF78091BF07D2
:10144000822B8093BF0708955F98F2CF8A98F0CFE0
:1014500090910801917090930601EACF0F931F932A
:10146000CF93DF93C82F41E06DE979E10E946FD9F6
:101470008C2F0E948ED985E999E10E94ACCE8DED2A
:1014800098E10E9409DB41E063E879E18C2F0E943A
:101490006FD98C2F0E948ED986E699E10E94ACCE3E
:1014A0008C2F0E9415DA8C2F0F9432128C2F0E94F1
:1014B00010D68C2F0E943AD68C2F0E94EED58C2FFE
:1014C0000E94B6D58C2F0E9494D58C2F0E94E4D90F
:1014D00041E065EF78E18C2F0E946FD902EF15E0B3
:1014E000D0E08C2F0E948ED96D2F8CEE98E10E9457
:1014F00074D6F80160817181072E000C880B990B5E
:101500000F94B839AB01BC0189EE98E10E94A4CFD9
:10151000F80162817381072E000C880B990B0F94E0
:10152000B839AB01BC0186EE98E10E94A4CFF80166
:101530006481758183EE98E10E9404DB0A5F1F4F8E
:10154000D13009F098C06FEF8C2F0E9493D98C2F67
:101550000E9484D641E063E279E18C2F0E946FD92A
:101560008C2F0E948ED980E199E10E94ACCE6091CF
:10157000E8157091E9158EE499E10E947BDA60919B
:10158000AC157091AD158FE09CE30E947BDA609101
:101590007015709171158CE09CE30E947BDA8AE0F3
:1015A0000E949FCE8C2F0E948ED980E199E10E94EB
:1015B000ACCE60913415709135158DE199E10E94A2
:1015C00004DB8C2F0E948ED980E199E10E94ACCE81
:1015D0006091F8147091F91487E199E10E9404DB9D
:1015E0008AE00E949FCE41E061E579E18C2F0E9464
:1015F0006FD9D091EA151091AE1500917215D111E5
:101600003CC0111141C001113FC0809136158823A3
:1016100091F0C11102C00E940FD88AE399E10E94A3
:10162000ACCE80E20E949FCE89E499E10E94ACCECC
:101630008AE00E949FCE8091FA14882391F0C11114
:1016400002C00E940FD88AE399E10E94ACCE80E2EA
:101650000E949FCE84E499E10E94ACCE8AE00E9471
:101660009FCE8C2F0E94C7DB8C2FDF91CF911F91D3
:101670000F910C948ED6D1E034CFCC2349F08AE37D
:1016800099E10E94ACCE0CC08AE399E1C1110AC075
:101690000E940FD88AE399E10E94ACCEDD2321F0AD
:1016A0008EE499E10E94ACCE112321F08FE09CE3FF
:1016B0000E94ACCE002321F08CE09CE30E94ACCED3
:1016C0008AE00E949FCEA1CF8F929F92AF92BF924D
:1016D000DF92EF92FF920F931F93CF93DF93CDB7DB
:1016E000DEB7C658D1090FB6F894DEBF0FBECDBF26
:1016F000C358DF4F188219821A821B82CD57D040FF
:101700008091EF039091F003A091F103B091F20367
:10171000CF57DF4F88839983AA83BB83C158D040BA
:1017200084E690E0909354078093530710925607F5
:10173000109255071092570725E537E044E050E036
:10174000BE016F577F4F83E597E00E9494DA809146
:101750005307909154070296909354078093530730
:10176000109256071092550781E0CA57DF4F8883C1
:10177000C658D040CE018A579F4F0E941F7725E55B
:1017800037E048E450E065E579E083E597E00E94C2
:1017900094DA80E1E4ECF2E08E010F5F1F4FD80194
:1017A00001900D928A95E1F725E537E040E150E0A0
:1017B000B80183E597E00E9494DA8EEF95E00E94ED
:1017C000317786EE98E00E9428778AE796E00E94BB
:1017D00028777E018DE6E80EF11C8FEFD7018C9300
:1017E000C7010E941F7719821A821B821C82C801BE
:1017F0000E94317719821A821B821C82C8010E94C2
:101800003177C358DF4F188219821A821B82CD5755
:10181000D04083E0F70180838983CE0183589F4FB6
:101820000E943177C7010E941F77C8010E941F776D
:101830005AE0D52EDA94DD2031F0CE0183589F4F47
:101840000E943177F7CF8CE0D8011D928A95E9F795
:10185000C8010E942877C358DF4F188219821A8264
:101860001B82CD57D0404AE0D42EDA94DD2031F0EF
:10187000CE0183589F4F0E943177F7CF83E0CB573B
:10188000DF4F8883C558D040EA968FAFEA97CE01E4
:101890008B579F4F0E941F77CE0187589F4F0E9402
:1018A0001F7788E0F701982F11929A95E9F7D801F0
:1018B0001D928A95E9F725E537E048E050E0B70149
:1018C00083E597E00E9494DA25E537E048E050E0B0
:1018D000B80183E597E00E9494DAC358DF4F18827D
:1018E00019821A821B82CD57D0403AE0A32EB12C28
:1018F000B1E0AB1AB10831F0CE0183589F4F0E947E
:101900003177F6CF19828FEFF7018083C8010E94EB
:101910001677C7010E941F7780E1D8011D928A9532
:10192000E9F725E537E040E150E0B80183E597E0CD
:101930000E9494DA1982C8010E94167725E537E0E3
:101940004CE050E062EF75E083E597E00E9494DAA6
:1019500092E0D92E812C912C20E8A22E2FE3B22EDA
:10196000198A1A8A1B8A1C8A8D869E86AF86B88A37
:1019700080914A0690914B06A0914C06B0914D067D
:1019800089839A83AB83BC832CEA35EC47E25EE320
:1019900060914E0670914F068091500690915106CD
:1019A0000F94023F6D837E838F8398872CEA35ECFA
:1019B00047E25EE3609152067091530680915406AF
:1019C000909155060F94173A69877A878B879C8781
:1019D00025E537E044E150E0B80183E597E00E9457
:1019E00094DAB1E0DB12C5C184E190E09A83898387
:1019F00025E537E042E050E0B80183E597E00E943A
:101A000094DA8CE0E4EDF2E0D80101900D928A9531
:101A1000E1F7C8010E940D778CE0E4EDF2E0D80117
:101A200001900D928A95E1F7C8010E940D77198205
:101A3000C8010E941F7780912E028983C8010E94ED
:101A40001F778FEF8983C8010E941F7785E0E0EE42
:101A5000F2E0D80101900D928A95E1F725E537E093
:101A600045E050E0B80183E597E00E9494DA1982DE
:101A7000C8010E94167780E2E5EEF2E0D8010190FD
:101A80000D928A95E1F725E537E040E250E0B80194
:101A900083E597E00E9494DAF7011082C7010E9463
:101AA000167781EF95E00E94167725E537E048E04C
:101AB00050E069EE75E083E597E00E9494DAC35840
:101AC000DF4F188219821A821B82CD57D040CE0177
:101AD00083589F4F0E943177CE0183589F4F0E94B9
:101AE0003177FE0137968AE0DF011D928A95E9F78A
:101AF0008091E8159091E9159A8389838091AC15BE
:101B00009091AD159C838B83809170159091711588
:101B10009E838D8380913415909135159A8B898B96
:101B20008091F8149091F9149C8B8B8B25E537E00C
:101B300044E150E0B80183E597E00E9494DA88E23E
:101B4000E5E0F3E0D80101900D928A95E1F725E5F3
:101B500037E048E250E0B80183E597E00E9494DA6C
:101B600080E1D82EF8018D2D11928A95E9F725E5AF
:101B700037E040E150E0B80183E597E00E9494DA55
:101B80001A8219828091EA1581709091AE1590FBAE
:101B900081F99091721590FB82F989838A819091E5
:101BA000361590FB80F99091FA1490FB81F98A83A5
:101BB00025E537E042E050E0B80183E597E00E9478
:101BC00094DAC358DF4F188219821A821B82CD57CC
:101BD000D040CE0183589F4F0E943177CE01835869
:101BE0009F4F0E943177D8011D92DA94E9F725E5DD
:101BF00037E040E150E0B80183E597E00E9494DAD5
:101C00008CE6F80111928A95E9F725E537E04CE674
